
STM32F429I-DISCO.elf:     file format elf32-littlearm

Sections:
Idx Name          Size      VMA       LMA       File off  Algn
  0 .isr_vector   000001ac  08000000  08000000  00010000  2**0
                  CONTENTS, ALLOC, LOAD, READONLY, DATA
  1 .text         0001e434  080001b0  080001b0  000101b0  2**4
                  CONTENTS, ALLOC, LOAD, READONLY, CODE
  2 .rodata       00003608  0801e5e8  0801e5e8  0002e5e8  2**3
                  CONTENTS, ALLOC, LOAD, READONLY, DATA
  3 FontFlashSection 000007fa  08021bf0  08021bf0  00031bf0  2**2
                  CONTENTS, ALLOC, LOAD, READONLY, DATA
  4 FontSearchFlashSection 00000028  080223ec  080223ec  000323ec  2**2
                  CONTENTS, ALLOC, LOAD, READONLY, DATA
  5 TextFlashSection 00000028  08022414  08022414  00032414  2**2
                  CONTENTS, ALLOC, LOAD, READONLY, DATA
  6 ExtFlashSection 000bb800  0802243c  0802243c  0003243c  2**2
                  CONTENTS, ALLOC, LOAD, READONLY, DATA
  7 .ARM.extab    00000000  080ddc3c  080ddc3c  000f02d0  2**0
                  CONTENTS
  8 .ARM          00000008  080ddc3c  080ddc3c  000edc3c  2**2
                  CONTENTS, ALLOC, LOAD, READONLY, DATA
  9 .preinit_array 00000000  080ddc44  080ddc44  000f02d0  2**0
                  CONTENTS, ALLOC, LOAD, DATA
 10 .init_array   00000014  080ddc44  080ddc44  000edc44  2**2
                  CONTENTS, ALLOC, LOAD, DATA
 11 .fini_array   00000008  080ddc58  080ddc58  000edc58  2**2
                  CONTENTS, ALLOC, LOAD, DATA
 12 .data         000002d0  20000000  080ddc60  000f0000  2**2
                  CONTENTS, ALLOC, LOAD, DATA
 13 .bss          00012604  200002d0  080ddf30  000f02d0  2**3
                  ALLOC
 14 ._user_heap_stack 00001404  200128d4  080ddf30  000f28d4  2**0
                  ALLOC
 15 .ARM.attributes 00000030  00000000  00000000  000f02d0  2**0
                  CONTENTS, READONLY
 16 TouchGFX_Framebuffer 00070800  d0000000  d0000000  00100000  2**2
                  ALLOC
 17 .debug_line   0004a41b  00000000  00000000  000f0300  2**0
                  CONTENTS, READONLY, DEBUGGING, OCTETS
 18 .debug_info   000993bb  00000000  00000000  0013a71b  2**0
                  CONTENTS, READONLY, DEBUGGING, OCTETS
 19 .debug_abbrev 0001259c  00000000  00000000  001d3ad6  2**0
                  CONTENTS, READONLY, DEBUGGING, OCTETS
 20 .debug_aranges 000029c8  00000000  00000000  001e6078  2**3
                  CONTENTS, READONLY, DEBUGGING, OCTETS
 21 .debug_str    0010af6c  00000000  00000000  001e8a40  2**0
                  CONTENTS, READONLY, DEBUGGING, OCTETS
 22 .debug_ranges 000042c8  00000000  00000000  002f39b0  2**3
                  CONTENTS, READONLY, DEBUGGING, OCTETS
 23 .debug_loc    0002983e  00000000  00000000  002f7c78  2**0
                  CONTENTS, READONLY, DEBUGGING, OCTETS
 24 .debug_macro  000306c2  00000000  00000000  003214b6  2**0
                  CONTENTS, READONLY, DEBUGGING, OCTETS
 25 .comment      000000cf  00000000  00000000  00351b78  2**0
                  CONTENTS, READONLY
 26 .debug_frame  00008800  00000000  00000000  00351c48  2**2
                  CONTENTS, READONLY, DEBUGGING, OCTETS

Disassembly of section .text:

080001b0 <__do_global_dtors_aux>:
 80001b0:	b510      	push	{r4, lr}
 80001b2:	4c05      	ldr	r4, [pc, #20]	; (80001c8 <__do_global_dtors_aux+0x18>)
 80001b4:	7823      	ldrb	r3, [r4, #0]
 80001b6:	b933      	cbnz	r3, 80001c6 <__do_global_dtors_aux+0x16>
 80001b8:	4b04      	ldr	r3, [pc, #16]	; (80001cc <__do_global_dtors_aux+0x1c>)
 80001ba:	b113      	cbz	r3, 80001c2 <__do_global_dtors_aux+0x12>
 80001bc:	4804      	ldr	r0, [pc, #16]	; (80001d0 <__do_global_dtors_aux+0x20>)
 80001be:	f3af 8000 	nop.w
 80001c2:	2301      	movs	r3, #1
 80001c4:	7023      	strb	r3, [r4, #0]
 80001c6:	bd10      	pop	{r4, pc}
 80001c8:	200002d0 	.word	0x200002d0
 80001cc:	00000000 	.word	0x00000000
 80001d0:	0801e5cc 	.word	0x0801e5cc

080001d4 <frame_dummy>:
 80001d4:	b508      	push	{r3, lr}
 80001d6:	4b03      	ldr	r3, [pc, #12]	; (80001e4 <frame_dummy+0x10>)
 80001d8:	b11b      	cbz	r3, 80001e2 <frame_dummy+0xe>
 80001da:	4903      	ldr	r1, [pc, #12]	; (80001e8 <frame_dummy+0x14>)
 80001dc:	4803      	ldr	r0, [pc, #12]	; (80001ec <frame_dummy+0x18>)
 80001de:	f3af 8000 	nop.w
 80001e2:	bd08      	pop	{r3, pc}
 80001e4:	00000000 	.word	0x00000000
 80001e8:	200002d4 	.word	0x200002d4
 80001ec:	0801e5cc 	.word	0x0801e5cc

080001f0 <strlen>:
 80001f0:	4603      	mov	r3, r0
 80001f2:	f813 2b01 	ldrb.w	r2, [r3], #1
 80001f6:	2a00      	cmp	r2, #0
 80001f8:	d1fb      	bne.n	80001f2 <strlen+0x2>
 80001fa:	1a18      	subs	r0, r3, r0
 80001fc:	3801      	subs	r0, #1
 80001fe:	4770      	bx	lr

08000200 <memchr>:
 8000200:	f001 01ff 	and.w	r1, r1, #255	; 0xff
 8000204:	2a10      	cmp	r2, #16
 8000206:	db2b      	blt.n	8000260 <memchr+0x60>
 8000208:	f010 0f07 	tst.w	r0, #7
 800020c:	d008      	beq.n	8000220 <memchr+0x20>
 800020e:	f810 3b01 	ldrb.w	r3, [r0], #1
 8000212:	3a01      	subs	r2, #1
 8000214:	428b      	cmp	r3, r1
 8000216:	d02d      	beq.n	8000274 <memchr+0x74>
 8000218:	f010 0f07 	tst.w	r0, #7
 800021c:	b342      	cbz	r2, 8000270 <memchr+0x70>
 800021e:	d1f6      	bne.n	800020e <memchr+0xe>
 8000220:	b4f0      	push	{r4, r5, r6, r7}
 8000222:	ea41 2101 	orr.w	r1, r1, r1, lsl #8
 8000226:	ea41 4101 	orr.w	r1, r1, r1, lsl #16
 800022a:	f022 0407 	bic.w	r4, r2, #7
 800022e:	f07f 0700 	mvns.w	r7, #0
 8000232:	2300      	movs	r3, #0
 8000234:	e8f0 5602 	ldrd	r5, r6, [r0], #8
 8000238:	3c08      	subs	r4, #8
 800023a:	ea85 0501 	eor.w	r5, r5, r1
 800023e:	ea86 0601 	eor.w	r6, r6, r1
 8000242:	fa85 f547 	uadd8	r5, r5, r7
 8000246:	faa3 f587 	sel	r5, r3, r7
 800024a:	fa86 f647 	uadd8	r6, r6, r7
 800024e:	faa5 f687 	sel	r6, r5, r7
 8000252:	b98e      	cbnz	r6, 8000278 <memchr+0x78>
 8000254:	d1ee      	bne.n	8000234 <memchr+0x34>
 8000256:	bcf0      	pop	{r4, r5, r6, r7}
 8000258:	f001 01ff 	and.w	r1, r1, #255	; 0xff
 800025c:	f002 0207 	and.w	r2, r2, #7
 8000260:	b132      	cbz	r2, 8000270 <memchr+0x70>
 8000262:	f810 3b01 	ldrb.w	r3, [r0], #1
 8000266:	3a01      	subs	r2, #1
 8000268:	ea83 0301 	eor.w	r3, r3, r1
 800026c:	b113      	cbz	r3, 8000274 <memchr+0x74>
 800026e:	d1f8      	bne.n	8000262 <memchr+0x62>
 8000270:	2000      	movs	r0, #0
 8000272:	4770      	bx	lr
 8000274:	3801      	subs	r0, #1
 8000276:	4770      	bx	lr
 8000278:	2d00      	cmp	r5, #0
 800027a:	bf06      	itte	eq
 800027c:	4635      	moveq	r5, r6
 800027e:	3803      	subeq	r0, #3
 8000280:	3807      	subne	r0, #7
 8000282:	f015 0f01 	tst.w	r5, #1
 8000286:	d107      	bne.n	8000298 <memchr+0x98>
 8000288:	3001      	adds	r0, #1
 800028a:	f415 7f80 	tst.w	r5, #256	; 0x100
 800028e:	bf02      	ittt	eq
 8000290:	3001      	addeq	r0, #1
 8000292:	f415 3fc0 	tsteq.w	r5, #98304	; 0x18000
 8000296:	3001      	addeq	r0, #1
 8000298:	bcf0      	pop	{r4, r5, r6, r7}
 800029a:	3801      	subs	r0, #1
 800029c:	4770      	bx	lr
 800029e:	bf00      	nop

080002a0 <__aeabi_drsub>:
 80002a0:	f081 4100 	eor.w	r1, r1, #2147483648	; 0x80000000
 80002a4:	e002      	b.n	80002ac <__adddf3>
 80002a6:	bf00      	nop

080002a8 <__aeabi_dsub>:
 80002a8:	f083 4300 	eor.w	r3, r3, #2147483648	; 0x80000000

080002ac <__adddf3>:
 80002ac:	b530      	push	{r4, r5, lr}
 80002ae:	ea4f 0441 	mov.w	r4, r1, lsl #1
 80002b2:	ea4f 0543 	mov.w	r5, r3, lsl #1
 80002b6:	ea94 0f05 	teq	r4, r5
 80002ba:	bf08      	it	eq
 80002bc:	ea90 0f02 	teqeq	r0, r2
 80002c0:	bf1f      	itttt	ne
 80002c2:	ea54 0c00 	orrsne.w	ip, r4, r0
 80002c6:	ea55 0c02 	orrsne.w	ip, r5, r2
 80002ca:	ea7f 5c64 	mvnsne.w	ip, r4, asr #21
 80002ce:	ea7f 5c65 	mvnsne.w	ip, r5, asr #21
 80002d2:	f000 80e2 	beq.w	800049a <__adddf3+0x1ee>
 80002d6:	ea4f 5454 	mov.w	r4, r4, lsr #21
 80002da:	ebd4 5555 	rsbs	r5, r4, r5, lsr #21
 80002de:	bfb8      	it	lt
 80002e0:	426d      	neglt	r5, r5
 80002e2:	dd0c      	ble.n	80002fe <__adddf3+0x52>
 80002e4:	442c      	add	r4, r5
 80002e6:	ea80 0202 	eor.w	r2, r0, r2
 80002ea:	ea81 0303 	eor.w	r3, r1, r3
 80002ee:	ea82 0000 	eor.w	r0, r2, r0
 80002f2:	ea83 0101 	eor.w	r1, r3, r1
 80002f6:	ea80 0202 	eor.w	r2, r0, r2
 80002fa:	ea81 0303 	eor.w	r3, r1, r3
 80002fe:	2d36      	cmp	r5, #54	; 0x36
 8000300:	bf88      	it	hi
 8000302:	bd30      	pophi	{r4, r5, pc}
 8000304:	f011 4f00 	tst.w	r1, #2147483648	; 0x80000000
 8000308:	ea4f 3101 	mov.w	r1, r1, lsl #12
 800030c:	f44f 1c80 	mov.w	ip, #1048576	; 0x100000
 8000310:	ea4c 3111 	orr.w	r1, ip, r1, lsr #12
 8000314:	d002      	beq.n	800031c <__adddf3+0x70>
 8000316:	4240      	negs	r0, r0
 8000318:	eb61 0141 	sbc.w	r1, r1, r1, lsl #1
 800031c:	f013 4f00 	tst.w	r3, #2147483648	; 0x80000000
 8000320:	ea4f 3303 	mov.w	r3, r3, lsl #12
 8000324:	ea4c 3313 	orr.w	r3, ip, r3, lsr #12
 8000328:	d002      	beq.n	8000330 <__adddf3+0x84>
 800032a:	4252      	negs	r2, r2
 800032c:	eb63 0343 	sbc.w	r3, r3, r3, lsl #1
 8000330:	ea94 0f05 	teq	r4, r5
 8000334:	f000 80a7 	beq.w	8000486 <__adddf3+0x1da>
 8000338:	f1a4 0401 	sub.w	r4, r4, #1
 800033c:	f1d5 0e20 	rsbs	lr, r5, #32
 8000340:	db0d      	blt.n	800035e <__adddf3+0xb2>
 8000342:	fa02 fc0e 	lsl.w	ip, r2, lr
 8000346:	fa22 f205 	lsr.w	r2, r2, r5
 800034a:	1880      	adds	r0, r0, r2
 800034c:	f141 0100 	adc.w	r1, r1, #0
 8000350:	fa03 f20e 	lsl.w	r2, r3, lr
 8000354:	1880      	adds	r0, r0, r2
 8000356:	fa43 f305 	asr.w	r3, r3, r5
 800035a:	4159      	adcs	r1, r3
 800035c:	e00e      	b.n	800037c <__adddf3+0xd0>
 800035e:	f1a5 0520 	sub.w	r5, r5, #32
 8000362:	f10e 0e20 	add.w	lr, lr, #32
 8000366:	2a01      	cmp	r2, #1
 8000368:	fa03 fc0e 	lsl.w	ip, r3, lr
 800036c:	bf28      	it	cs
 800036e:	f04c 0c02 	orrcs.w	ip, ip, #2
 8000372:	fa43 f305 	asr.w	r3, r3, r5
 8000376:	18c0      	adds	r0, r0, r3
 8000378:	eb51 71e3 	adcs.w	r1, r1, r3, asr #31
 800037c:	f001 4500 	and.w	r5, r1, #2147483648	; 0x80000000
 8000380:	d507      	bpl.n	8000392 <__adddf3+0xe6>
 8000382:	f04f 0e00 	mov.w	lr, #0
 8000386:	f1dc 0c00 	rsbs	ip, ip, #0
 800038a:	eb7e 0000 	sbcs.w	r0, lr, r0
 800038e:	eb6e 0101 	sbc.w	r1, lr, r1
 8000392:	f5b1 1f80 	cmp.w	r1, #1048576	; 0x100000
 8000396:	d31b      	bcc.n	80003d0 <__adddf3+0x124>
 8000398:	f5b1 1f00 	cmp.w	r1, #2097152	; 0x200000
 800039c:	d30c      	bcc.n	80003b8 <__adddf3+0x10c>
 800039e:	0849      	lsrs	r1, r1, #1
 80003a0:	ea5f 0030 	movs.w	r0, r0, rrx
 80003a4:	ea4f 0c3c 	mov.w	ip, ip, rrx
 80003a8:	f104 0401 	add.w	r4, r4, #1
 80003ac:	ea4f 5244 	mov.w	r2, r4, lsl #21
 80003b0:	f512 0f80 	cmn.w	r2, #4194304	; 0x400000
 80003b4:	f080 809a 	bcs.w	80004ec <__adddf3+0x240>
 80003b8:	f1bc 4f00 	cmp.w	ip, #2147483648	; 0x80000000
 80003bc:	bf08      	it	eq
 80003be:	ea5f 0c50 	movseq.w	ip, r0, lsr #1
 80003c2:	f150 0000 	adcs.w	r0, r0, #0
 80003c6:	eb41 5104 	adc.w	r1, r1, r4, lsl #20
 80003ca:	ea41 0105 	orr.w	r1, r1, r5
 80003ce:	bd30      	pop	{r4, r5, pc}
 80003d0:	ea5f 0c4c 	movs.w	ip, ip, lsl #1
 80003d4:	4140      	adcs	r0, r0
 80003d6:	eb41 0101 	adc.w	r1, r1, r1
 80003da:	3c01      	subs	r4, #1
 80003dc:	bf28      	it	cs
 80003de:	f5b1 1f80 	cmpcs.w	r1, #1048576	; 0x100000
 80003e2:	d2e9      	bcs.n	80003b8 <__adddf3+0x10c>
 80003e4:	f091 0f00 	teq	r1, #0
 80003e8:	bf04      	itt	eq
 80003ea:	4601      	moveq	r1, r0
 80003ec:	2000      	moveq	r0, #0
 80003ee:	fab1 f381 	clz	r3, r1
 80003f2:	bf08      	it	eq
 80003f4:	3320      	addeq	r3, #32
 80003f6:	f1a3 030b 	sub.w	r3, r3, #11
 80003fa:	f1b3 0220 	subs.w	r2, r3, #32
 80003fe:	da0c      	bge.n	800041a <__adddf3+0x16e>
 8000400:	320c      	adds	r2, #12
 8000402:	dd08      	ble.n	8000416 <__adddf3+0x16a>
 8000404:	f102 0c14 	add.w	ip, r2, #20
 8000408:	f1c2 020c 	rsb	r2, r2, #12
 800040c:	fa01 f00c 	lsl.w	r0, r1, ip
 8000410:	fa21 f102 	lsr.w	r1, r1, r2
 8000414:	e00c      	b.n	8000430 <__adddf3+0x184>
 8000416:	f102 0214 	add.w	r2, r2, #20
 800041a:	bfd8      	it	le
 800041c:	f1c2 0c20 	rsble	ip, r2, #32
 8000420:	fa01 f102 	lsl.w	r1, r1, r2
 8000424:	fa20 fc0c 	lsr.w	ip, r0, ip
 8000428:	bfdc      	itt	le
 800042a:	ea41 010c 	orrle.w	r1, r1, ip
 800042e:	4090      	lslle	r0, r2
 8000430:	1ae4      	subs	r4, r4, r3
 8000432:	bfa2      	ittt	ge
 8000434:	eb01 5104 	addge.w	r1, r1, r4, lsl #20
 8000438:	4329      	orrge	r1, r5
 800043a:	bd30      	popge	{r4, r5, pc}
 800043c:	ea6f 0404 	mvn.w	r4, r4
 8000440:	3c1f      	subs	r4, #31
 8000442:	da1c      	bge.n	800047e <__adddf3+0x1d2>
 8000444:	340c      	adds	r4, #12
 8000446:	dc0e      	bgt.n	8000466 <__adddf3+0x1ba>
 8000448:	f104 0414 	add.w	r4, r4, #20
 800044c:	f1c4 0220 	rsb	r2, r4, #32
 8000450:	fa20 f004 	lsr.w	r0, r0, r4
 8000454:	fa01 f302 	lsl.w	r3, r1, r2
 8000458:	ea40 0003 	orr.w	r0, r0, r3
 800045c:	fa21 f304 	lsr.w	r3, r1, r4
 8000460:	ea45 0103 	orr.w	r1, r5, r3
 8000464:	bd30      	pop	{r4, r5, pc}
 8000466:	f1c4 040c 	rsb	r4, r4, #12
 800046a:	f1c4 0220 	rsb	r2, r4, #32
 800046e:	fa20 f002 	lsr.w	r0, r0, r2
 8000472:	fa01 f304 	lsl.w	r3, r1, r4
 8000476:	ea40 0003 	orr.w	r0, r0, r3
 800047a:	4629      	mov	r1, r5
 800047c:	bd30      	pop	{r4, r5, pc}
 800047e:	fa21 f004 	lsr.w	r0, r1, r4
 8000482:	4629      	mov	r1, r5
 8000484:	bd30      	pop	{r4, r5, pc}
 8000486:	f094 0f00 	teq	r4, #0
 800048a:	f483 1380 	eor.w	r3, r3, #1048576	; 0x100000
 800048e:	bf06      	itte	eq
 8000490:	f481 1180 	eoreq.w	r1, r1, #1048576	; 0x100000
 8000494:	3401      	addeq	r4, #1
 8000496:	3d01      	subne	r5, #1
 8000498:	e74e      	b.n	8000338 <__adddf3+0x8c>
 800049a:	ea7f 5c64 	mvns.w	ip, r4, asr #21
 800049e:	bf18      	it	ne
 80004a0:	ea7f 5c65 	mvnsne.w	ip, r5, asr #21
 80004a4:	d029      	beq.n	80004fa <__adddf3+0x24e>
 80004a6:	ea94 0f05 	teq	r4, r5
 80004aa:	bf08      	it	eq
 80004ac:	ea90 0f02 	teqeq	r0, r2
 80004b0:	d005      	beq.n	80004be <__adddf3+0x212>
 80004b2:	ea54 0c00 	orrs.w	ip, r4, r0
 80004b6:	bf04      	itt	eq
 80004b8:	4619      	moveq	r1, r3
 80004ba:	4610      	moveq	r0, r2
 80004bc:	bd30      	pop	{r4, r5, pc}
 80004be:	ea91 0f03 	teq	r1, r3
 80004c2:	bf1e      	ittt	ne
 80004c4:	2100      	movne	r1, #0
 80004c6:	2000      	movne	r0, #0
 80004c8:	bd30      	popne	{r4, r5, pc}
 80004ca:	ea5f 5c54 	movs.w	ip, r4, lsr #21
 80004ce:	d105      	bne.n	80004dc <__adddf3+0x230>
 80004d0:	0040      	lsls	r0, r0, #1
 80004d2:	4149      	adcs	r1, r1
 80004d4:	bf28      	it	cs
 80004d6:	f041 4100 	orrcs.w	r1, r1, #2147483648	; 0x80000000
 80004da:	bd30      	pop	{r4, r5, pc}
 80004dc:	f514 0480 	adds.w	r4, r4, #4194304	; 0x400000
 80004e0:	bf3c      	itt	cc
 80004e2:	f501 1180 	addcc.w	r1, r1, #1048576	; 0x100000
 80004e6:	bd30      	popcc	{r4, r5, pc}
 80004e8:	f001 4500 	and.w	r5, r1, #2147483648	; 0x80000000
 80004ec:	f045 41fe 	orr.w	r1, r5, #2130706432	; 0x7f000000
 80004f0:	f441 0170 	orr.w	r1, r1, #15728640	; 0xf00000
 80004f4:	f04f 0000 	mov.w	r0, #0
 80004f8:	bd30      	pop	{r4, r5, pc}
 80004fa:	ea7f 5c64 	mvns.w	ip, r4, asr #21
 80004fe:	bf1a      	itte	ne
 8000500:	4619      	movne	r1, r3
 8000502:	4610      	movne	r0, r2
 8000504:	ea7f 5c65 	mvnseq.w	ip, r5, asr #21
 8000508:	bf1c      	itt	ne
 800050a:	460b      	movne	r3, r1
 800050c:	4602      	movne	r2, r0
 800050e:	ea50 3401 	orrs.w	r4, r0, r1, lsl #12
 8000512:	bf06      	itte	eq
 8000514:	ea52 3503 	orrseq.w	r5, r2, r3, lsl #12
 8000518:	ea91 0f03 	teqeq	r1, r3
 800051c:	f441 2100 	orrne.w	r1, r1, #524288	; 0x80000
 8000520:	bd30      	pop	{r4, r5, pc}
 8000522:	bf00      	nop

08000524 <__aeabi_ui2d>:
 8000524:	f090 0f00 	teq	r0, #0
 8000528:	bf04      	itt	eq
 800052a:	2100      	moveq	r1, #0
 800052c:	4770      	bxeq	lr
 800052e:	b530      	push	{r4, r5, lr}
 8000530:	f44f 6480 	mov.w	r4, #1024	; 0x400
 8000534:	f104 0432 	add.w	r4, r4, #50	; 0x32
 8000538:	f04f 0500 	mov.w	r5, #0
 800053c:	f04f 0100 	mov.w	r1, #0
 8000540:	e750      	b.n	80003e4 <__adddf3+0x138>
 8000542:	bf00      	nop

08000544 <__aeabi_i2d>:
 8000544:	f090 0f00 	teq	r0, #0
 8000548:	bf04      	itt	eq
 800054a:	2100      	moveq	r1, #0
 800054c:	4770      	bxeq	lr
 800054e:	b530      	push	{r4, r5, lr}
 8000550:	f44f 6480 	mov.w	r4, #1024	; 0x400
 8000554:	f104 0432 	add.w	r4, r4, #50	; 0x32
 8000558:	f010 4500 	ands.w	r5, r0, #2147483648	; 0x80000000
 800055c:	bf48      	it	mi
 800055e:	4240      	negmi	r0, r0
 8000560:	f04f 0100 	mov.w	r1, #0
 8000564:	e73e      	b.n	80003e4 <__adddf3+0x138>
 8000566:	bf00      	nop

08000568 <__aeabi_f2d>:
 8000568:	0042      	lsls	r2, r0, #1
 800056a:	ea4f 01e2 	mov.w	r1, r2, asr #3
 800056e:	ea4f 0131 	mov.w	r1, r1, rrx
 8000572:	ea4f 7002 	mov.w	r0, r2, lsl #28
 8000576:	bf1f      	itttt	ne
 8000578:	f012 437f 	andsne.w	r3, r2, #4278190080	; 0xff000000
 800057c:	f093 4f7f 	teqne	r3, #4278190080	; 0xff000000
 8000580:	f081 5160 	eorne.w	r1, r1, #939524096	; 0x38000000
 8000584:	4770      	bxne	lr
 8000586:	f032 427f 	bics.w	r2, r2, #4278190080	; 0xff000000
 800058a:	bf08      	it	eq
 800058c:	4770      	bxeq	lr
 800058e:	f093 4f7f 	teq	r3, #4278190080	; 0xff000000
 8000592:	bf04      	itt	eq
 8000594:	f441 2100 	orreq.w	r1, r1, #524288	; 0x80000
 8000598:	4770      	bxeq	lr
 800059a:	b530      	push	{r4, r5, lr}
 800059c:	f44f 7460 	mov.w	r4, #896	; 0x380
 80005a0:	f001 4500 	and.w	r5, r1, #2147483648	; 0x80000000
 80005a4:	f021 4100 	bic.w	r1, r1, #2147483648	; 0x80000000
 80005a8:	e71c      	b.n	80003e4 <__adddf3+0x138>
 80005aa:	bf00      	nop

080005ac <__aeabi_ul2d>:
 80005ac:	ea50 0201 	orrs.w	r2, r0, r1
 80005b0:	bf08      	it	eq
 80005b2:	4770      	bxeq	lr
 80005b4:	b530      	push	{r4, r5, lr}
 80005b6:	f04f 0500 	mov.w	r5, #0
 80005ba:	e00a      	b.n	80005d2 <__aeabi_l2d+0x16>

080005bc <__aeabi_l2d>:
 80005bc:	ea50 0201 	orrs.w	r2, r0, r1
 80005c0:	bf08      	it	eq
 80005c2:	4770      	bxeq	lr
 80005c4:	b530      	push	{r4, r5, lr}
 80005c6:	f011 4500 	ands.w	r5, r1, #2147483648	; 0x80000000
 80005ca:	d502      	bpl.n	80005d2 <__aeabi_l2d+0x16>
 80005cc:	4240      	negs	r0, r0
 80005ce:	eb61 0141 	sbc.w	r1, r1, r1, lsl #1
 80005d2:	f44f 6480 	mov.w	r4, #1024	; 0x400
 80005d6:	f104 0432 	add.w	r4, r4, #50	; 0x32
 80005da:	ea5f 5c91 	movs.w	ip, r1, lsr #22
 80005de:	f43f aed8 	beq.w	8000392 <__adddf3+0xe6>
 80005e2:	f04f 0203 	mov.w	r2, #3
 80005e6:	ea5f 0cdc 	movs.w	ip, ip, lsr #3
 80005ea:	bf18      	it	ne
 80005ec:	3203      	addne	r2, #3
 80005ee:	ea5f 0cdc 	movs.w	ip, ip, lsr #3
 80005f2:	bf18      	it	ne
 80005f4:	3203      	addne	r2, #3
 80005f6:	eb02 02dc 	add.w	r2, r2, ip, lsr #3
 80005fa:	f1c2 0320 	rsb	r3, r2, #32
 80005fe:	fa00 fc03 	lsl.w	ip, r0, r3
 8000602:	fa20 f002 	lsr.w	r0, r0, r2
 8000606:	fa01 fe03 	lsl.w	lr, r1, r3
 800060a:	ea40 000e 	orr.w	r0, r0, lr
 800060e:	fa21 f102 	lsr.w	r1, r1, r2
 8000612:	4414      	add	r4, r2
 8000614:	e6bd      	b.n	8000392 <__adddf3+0xe6>
 8000616:	bf00      	nop

08000618 <__aeabi_dmul>:
 8000618:	b570      	push	{r4, r5, r6, lr}
 800061a:	f04f 0cff 	mov.w	ip, #255	; 0xff
 800061e:	f44c 6ce0 	orr.w	ip, ip, #1792	; 0x700
 8000622:	ea1c 5411 	ands.w	r4, ip, r1, lsr #20
 8000626:	bf1d      	ittte	ne
 8000628:	ea1c 5513 	andsne.w	r5, ip, r3, lsr #20
 800062c:	ea94 0f0c 	teqne	r4, ip
 8000630:	ea95 0f0c 	teqne	r5, ip
 8000634:	f000 f8de 	bleq	80007f4 <__aeabi_dmul+0x1dc>
 8000638:	442c      	add	r4, r5
 800063a:	ea81 0603 	eor.w	r6, r1, r3
 800063e:	ea21 514c 	bic.w	r1, r1, ip, lsl #21
 8000642:	ea23 534c 	bic.w	r3, r3, ip, lsl #21
 8000646:	ea50 3501 	orrs.w	r5, r0, r1, lsl #12
 800064a:	bf18      	it	ne
 800064c:	ea52 3503 	orrsne.w	r5, r2, r3, lsl #12
 8000650:	f441 1180 	orr.w	r1, r1, #1048576	; 0x100000
 8000654:	f443 1380 	orr.w	r3, r3, #1048576	; 0x100000
 8000658:	d038      	beq.n	80006cc <__aeabi_dmul+0xb4>
 800065a:	fba0 ce02 	umull	ip, lr, r0, r2
 800065e:	f04f 0500 	mov.w	r5, #0
 8000662:	fbe1 e502 	umlal	lr, r5, r1, r2
 8000666:	f006 4200 	and.w	r2, r6, #2147483648	; 0x80000000
 800066a:	fbe0 e503 	umlal	lr, r5, r0, r3
 800066e:	f04f 0600 	mov.w	r6, #0
 8000672:	fbe1 5603 	umlal	r5, r6, r1, r3
 8000676:	f09c 0f00 	teq	ip, #0
 800067a:	bf18      	it	ne
 800067c:	f04e 0e01 	orrne.w	lr, lr, #1
 8000680:	f1a4 04ff 	sub.w	r4, r4, #255	; 0xff
 8000684:	f5b6 7f00 	cmp.w	r6, #512	; 0x200
 8000688:	f564 7440 	sbc.w	r4, r4, #768	; 0x300
 800068c:	d204      	bcs.n	8000698 <__aeabi_dmul+0x80>
 800068e:	ea5f 0e4e 	movs.w	lr, lr, lsl #1
 8000692:	416d      	adcs	r5, r5
 8000694:	eb46 0606 	adc.w	r6, r6, r6
 8000698:	ea42 21c6 	orr.w	r1, r2, r6, lsl #11
 800069c:	ea41 5155 	orr.w	r1, r1, r5, lsr #21
 80006a0:	ea4f 20c5 	mov.w	r0, r5, lsl #11
 80006a4:	ea40 505e 	orr.w	r0, r0, lr, lsr #21
 80006a8:	ea4f 2ece 	mov.w	lr, lr, lsl #11
 80006ac:	f1b4 0cfd 	subs.w	ip, r4, #253	; 0xfd
 80006b0:	bf88      	it	hi
 80006b2:	f5bc 6fe0 	cmphi.w	ip, #1792	; 0x700
 80006b6:	d81e      	bhi.n	80006f6 <__aeabi_dmul+0xde>
 80006b8:	f1be 4f00 	cmp.w	lr, #2147483648	; 0x80000000
 80006bc:	bf08      	it	eq
 80006be:	ea5f 0e50 	movseq.w	lr, r0, lsr #1
 80006c2:	f150 0000 	adcs.w	r0, r0, #0
 80006c6:	eb41 5104 	adc.w	r1, r1, r4, lsl #20
 80006ca:	bd70      	pop	{r4, r5, r6, pc}
 80006cc:	f006 4600 	and.w	r6, r6, #2147483648	; 0x80000000
 80006d0:	ea46 0101 	orr.w	r1, r6, r1
 80006d4:	ea40 0002 	orr.w	r0, r0, r2
 80006d8:	ea81 0103 	eor.w	r1, r1, r3
 80006dc:	ebb4 045c 	subs.w	r4, r4, ip, lsr #1
 80006e0:	bfc2      	ittt	gt
 80006e2:	ebd4 050c 	rsbsgt	r5, r4, ip
 80006e6:	ea41 5104 	orrgt.w	r1, r1, r4, lsl #20
 80006ea:	bd70      	popgt	{r4, r5, r6, pc}
 80006ec:	f441 1180 	orr.w	r1, r1, #1048576	; 0x100000
 80006f0:	f04f 0e00 	mov.w	lr, #0
 80006f4:	3c01      	subs	r4, #1
 80006f6:	f300 80ab 	bgt.w	8000850 <__aeabi_dmul+0x238>
 80006fa:	f114 0f36 	cmn.w	r4, #54	; 0x36
 80006fe:	bfde      	ittt	le
 8000700:	2000      	movle	r0, #0
 8000702:	f001 4100 	andle.w	r1, r1, #2147483648	; 0x80000000
 8000706:	bd70      	pople	{r4, r5, r6, pc}
 8000708:	f1c4 0400 	rsb	r4, r4, #0
 800070c:	3c20      	subs	r4, #32
 800070e:	da35      	bge.n	800077c <__aeabi_dmul+0x164>
 8000710:	340c      	adds	r4, #12
 8000712:	dc1b      	bgt.n	800074c <__aeabi_dmul+0x134>
 8000714:	f104 0414 	add.w	r4, r4, #20
 8000718:	f1c4 0520 	rsb	r5, r4, #32
 800071c:	fa00 f305 	lsl.w	r3, r0, r5
 8000720:	fa20 f004 	lsr.w	r0, r0, r4
 8000724:	fa01 f205 	lsl.w	r2, r1, r5
 8000728:	ea40 0002 	orr.w	r0, r0, r2
 800072c:	f001 4200 	and.w	r2, r1, #2147483648	; 0x80000000
 8000730:	f021 4100 	bic.w	r1, r1, #2147483648	; 0x80000000
 8000734:	eb10 70d3 	adds.w	r0, r0, r3, lsr #31
 8000738:	fa21 f604 	lsr.w	r6, r1, r4
 800073c:	eb42 0106 	adc.w	r1, r2, r6
 8000740:	ea5e 0e43 	orrs.w	lr, lr, r3, lsl #1
 8000744:	bf08      	it	eq
 8000746:	ea20 70d3 	biceq.w	r0, r0, r3, lsr #31
 800074a:	bd70      	pop	{r4, r5, r6, pc}
 800074c:	f1c4 040c 	rsb	r4, r4, #12
 8000750:	f1c4 0520 	rsb	r5, r4, #32
 8000754:	fa00 f304 	lsl.w	r3, r0, r4
 8000758:	fa20 f005 	lsr.w	r0, r0, r5
 800075c:	fa01 f204 	lsl.w	r2, r1, r4
 8000760:	ea40 0002 	orr.w	r0, r0, r2
 8000764:	f001 4100 	and.w	r1, r1, #2147483648	; 0x80000000
 8000768:	eb10 70d3 	adds.w	r0, r0, r3, lsr #31
 800076c:	f141 0100 	adc.w	r1, r1, #0
 8000770:	ea5e 0e43 	orrs.w	lr, lr, r3, lsl #1
 8000774:	bf08      	it	eq
 8000776:	ea20 70d3 	biceq.w	r0, r0, r3, lsr #31
 800077a:	bd70      	pop	{r4, r5, r6, pc}
 800077c:	f1c4 0520 	rsb	r5, r4, #32
 8000780:	fa00 f205 	lsl.w	r2, r0, r5
 8000784:	ea4e 0e02 	orr.w	lr, lr, r2
 8000788:	fa20 f304 	lsr.w	r3, r0, r4
 800078c:	fa01 f205 	lsl.w	r2, r1, r5
 8000790:	ea43 0302 	orr.w	r3, r3, r2
 8000794:	fa21 f004 	lsr.w	r0, r1, r4
 8000798:	f001 4100 	and.w	r1, r1, #2147483648	; 0x80000000
 800079c:	fa21 f204 	lsr.w	r2, r1, r4
 80007a0:	ea20 0002 	bic.w	r0, r0, r2
 80007a4:	eb00 70d3 	add.w	r0, r0, r3, lsr #31
 80007a8:	ea5e 0e43 	orrs.w	lr, lr, r3, lsl #1
 80007ac:	bf08      	it	eq
 80007ae:	ea20 70d3 	biceq.w	r0, r0, r3, lsr #31
 80007b2:	bd70      	pop	{r4, r5, r6, pc}
 80007b4:	f094 0f00 	teq	r4, #0
 80007b8:	d10f      	bne.n	80007da <__aeabi_dmul+0x1c2>
 80007ba:	f001 4600 	and.w	r6, r1, #2147483648	; 0x80000000
 80007be:	0040      	lsls	r0, r0, #1
 80007c0:	eb41 0101 	adc.w	r1, r1, r1
 80007c4:	f411 1f80 	tst.w	r1, #1048576	; 0x100000
 80007c8:	bf08      	it	eq
 80007ca:	3c01      	subeq	r4, #1
 80007cc:	d0f7      	beq.n	80007be <__aeabi_dmul+0x1a6>
 80007ce:	ea41 0106 	orr.w	r1, r1, r6
 80007d2:	f095 0f00 	teq	r5, #0
 80007d6:	bf18      	it	ne
 80007d8:	4770      	bxne	lr
 80007da:	f003 4600 	and.w	r6, r3, #2147483648	; 0x80000000
 80007de:	0052      	lsls	r2, r2, #1
 80007e0:	eb43 0303 	adc.w	r3, r3, r3
 80007e4:	f413 1f80 	tst.w	r3, #1048576	; 0x100000
 80007e8:	bf08      	it	eq
 80007ea:	3d01      	subeq	r5, #1
 80007ec:	d0f7      	beq.n	80007de <__aeabi_dmul+0x1c6>
 80007ee:	ea43 0306 	orr.w	r3, r3, r6
 80007f2:	4770      	bx	lr
 80007f4:	ea94 0f0c 	teq	r4, ip
 80007f8:	ea0c 5513 	and.w	r5, ip, r3, lsr #20
 80007fc:	bf18      	it	ne
 80007fe:	ea95 0f0c 	teqne	r5, ip
 8000802:	d00c      	beq.n	800081e <__aeabi_dmul+0x206>
 8000804:	ea50 0641 	orrs.w	r6, r0, r1, lsl #1
 8000808:	bf18      	it	ne
 800080a:	ea52 0643 	orrsne.w	r6, r2, r3, lsl #1
 800080e:	d1d1      	bne.n	80007b4 <__aeabi_dmul+0x19c>
 8000810:	ea81 0103 	eor.w	r1, r1, r3
 8000814:	f001 4100 	and.w	r1, r1, #2147483648	; 0x80000000
 8000818:	f04f 0000 	mov.w	r0, #0
 800081c:	bd70      	pop	{r4, r5, r6, pc}
 800081e:	ea50 0641 	orrs.w	r6, r0, r1, lsl #1
 8000822:	bf06      	itte	eq
 8000824:	4610      	moveq	r0, r2
 8000826:	4619      	moveq	r1, r3
 8000828:	ea52 0643 	orrsne.w	r6, r2, r3, lsl #1
 800082c:	d019      	beq.n	8000862 <__aeabi_dmul+0x24a>
 800082e:	ea94 0f0c 	teq	r4, ip
 8000832:	d102      	bne.n	800083a <__aeabi_dmul+0x222>
 8000834:	ea50 3601 	orrs.w	r6, r0, r1, lsl #12
 8000838:	d113      	bne.n	8000862 <__aeabi_dmul+0x24a>
 800083a:	ea95 0f0c 	teq	r5, ip
 800083e:	d105      	bne.n	800084c <__aeabi_dmul+0x234>
 8000840:	ea52 3603 	orrs.w	r6, r2, r3, lsl #12
 8000844:	bf1c      	itt	ne
 8000846:	4610      	movne	r0, r2
 8000848:	4619      	movne	r1, r3
 800084a:	d10a      	bne.n	8000862 <__aeabi_dmul+0x24a>
 800084c:	ea81 0103 	eor.w	r1, r1, r3
 8000850:	f001 4100 	and.w	r1, r1, #2147483648	; 0x80000000
 8000854:	f041 41fe 	orr.w	r1, r1, #2130706432	; 0x7f000000
 8000858:	f441 0170 	orr.w	r1, r1, #15728640	; 0xf00000
 800085c:	f04f 0000 	mov.w	r0, #0
 8000860:	bd70      	pop	{r4, r5, r6, pc}
 8000862:	f041 41fe 	orr.w	r1, r1, #2130706432	; 0x7f000000
 8000866:	f441 0178 	orr.w	r1, r1, #16252928	; 0xf80000
 800086a:	bd70      	pop	{r4, r5, r6, pc}

0800086c <__aeabi_ddiv>:
 800086c:	b570      	push	{r4, r5, r6, lr}
 800086e:	f04f 0cff 	mov.w	ip, #255	; 0xff
 8000872:	f44c 6ce0 	orr.w	ip, ip, #1792	; 0x700
 8000876:	ea1c 5411 	ands.w	r4, ip, r1, lsr #20
 800087a:	bf1d      	ittte	ne
 800087c:	ea1c 5513 	andsne.w	r5, ip, r3, lsr #20
 8000880:	ea94 0f0c 	teqne	r4, ip
 8000884:	ea95 0f0c 	teqne	r5, ip
 8000888:	f000 f8a7 	bleq	80009da <__aeabi_ddiv+0x16e>
 800088c:	eba4 0405 	sub.w	r4, r4, r5
 8000890:	ea81 0e03 	eor.w	lr, r1, r3
 8000894:	ea52 3503 	orrs.w	r5, r2, r3, lsl #12
 8000898:	ea4f 3101 	mov.w	r1, r1, lsl #12
 800089c:	f000 8088 	beq.w	80009b0 <__aeabi_ddiv+0x144>
 80008a0:	ea4f 3303 	mov.w	r3, r3, lsl #12
 80008a4:	f04f 5580 	mov.w	r5, #268435456	; 0x10000000
 80008a8:	ea45 1313 	orr.w	r3, r5, r3, lsr #4
 80008ac:	ea43 6312 	orr.w	r3, r3, r2, lsr #24
 80008b0:	ea4f 2202 	mov.w	r2, r2, lsl #8
 80008b4:	ea45 1511 	orr.w	r5, r5, r1, lsr #4
 80008b8:	ea45 6510 	orr.w	r5, r5, r0, lsr #24
 80008bc:	ea4f 2600 	mov.w	r6, r0, lsl #8
 80008c0:	f00e 4100 	and.w	r1, lr, #2147483648	; 0x80000000
 80008c4:	429d      	cmp	r5, r3
 80008c6:	bf08      	it	eq
 80008c8:	4296      	cmpeq	r6, r2
 80008ca:	f144 04fd 	adc.w	r4, r4, #253	; 0xfd
 80008ce:	f504 7440 	add.w	r4, r4, #768	; 0x300
 80008d2:	d202      	bcs.n	80008da <__aeabi_ddiv+0x6e>
 80008d4:	085b      	lsrs	r3, r3, #1
 80008d6:	ea4f 0232 	mov.w	r2, r2, rrx
 80008da:	1ab6      	subs	r6, r6, r2
 80008dc:	eb65 0503 	sbc.w	r5, r5, r3
 80008e0:	085b      	lsrs	r3, r3, #1
 80008e2:	ea4f 0232 	mov.w	r2, r2, rrx
 80008e6:	f44f 1080 	mov.w	r0, #1048576	; 0x100000
 80008ea:	f44f 2c00 	mov.w	ip, #524288	; 0x80000
 80008ee:	ebb6 0e02 	subs.w	lr, r6, r2
 80008f2:	eb75 0e03 	sbcs.w	lr, r5, r3
 80008f6:	bf22      	ittt	cs
 80008f8:	1ab6      	subcs	r6, r6, r2
 80008fa:	4675      	movcs	r5, lr
 80008fc:	ea40 000c 	orrcs.w	r0, r0, ip
 8000900:	085b      	lsrs	r3, r3, #1
 8000902:	ea4f 0232 	mov.w	r2, r2, rrx
 8000906:	ebb6 0e02 	subs.w	lr, r6, r2
 800090a:	eb75 0e03 	sbcs.w	lr, r5, r3
 800090e:	bf22      	ittt	cs
 8000910:	1ab6      	subcs	r6, r6, r2
 8000912:	4675      	movcs	r5, lr
 8000914:	ea40 005c 	orrcs.w	r0, r0, ip, lsr #1
 8000918:	085b      	lsrs	r3, r3, #1
 800091a:	ea4f 0232 	mov.w	r2, r2, rrx
 800091e:	ebb6 0e02 	subs.w	lr, r6, r2
 8000922:	eb75 0e03 	sbcs.w	lr, r5, r3
 8000926:	bf22      	ittt	cs
 8000928:	1ab6      	subcs	r6, r6, r2
 800092a:	4675      	movcs	r5, lr
 800092c:	ea40 009c 	orrcs.w	r0, r0, ip, lsr #2
 8000930:	085b      	lsrs	r3, r3, #1
 8000932:	ea4f 0232 	mov.w	r2, r2, rrx
 8000936:	ebb6 0e02 	subs.w	lr, r6, r2
 800093a:	eb75 0e03 	sbcs.w	lr, r5, r3
 800093e:	bf22      	ittt	cs
 8000940:	1ab6      	subcs	r6, r6, r2
 8000942:	4675      	movcs	r5, lr
 8000944:	ea40 00dc 	orrcs.w	r0, r0, ip, lsr #3
 8000948:	ea55 0e06 	orrs.w	lr, r5, r6
 800094c:	d018      	beq.n	8000980 <__aeabi_ddiv+0x114>
 800094e:	ea4f 1505 	mov.w	r5, r5, lsl #4
 8000952:	ea45 7516 	orr.w	r5, r5, r6, lsr #28
 8000956:	ea4f 1606 	mov.w	r6, r6, lsl #4
 800095a:	ea4f 03c3 	mov.w	r3, r3, lsl #3
 800095e:	ea43 7352 	orr.w	r3, r3, r2, lsr #29
 8000962:	ea4f 02c2 	mov.w	r2, r2, lsl #3
 8000966:	ea5f 1c1c 	movs.w	ip, ip, lsr #4
 800096a:	d1c0      	bne.n	80008ee <__aeabi_ddiv+0x82>
 800096c:	f411 1f80 	tst.w	r1, #1048576	; 0x100000
 8000970:	d10b      	bne.n	800098a <__aeabi_ddiv+0x11e>
 8000972:	ea41 0100 	orr.w	r1, r1, r0
 8000976:	f04f 0000 	mov.w	r0, #0
 800097a:	f04f 4c00 	mov.w	ip, #2147483648	; 0x80000000
 800097e:	e7b6      	b.n	80008ee <__aeabi_ddiv+0x82>
 8000980:	f411 1f80 	tst.w	r1, #1048576	; 0x100000
 8000984:	bf04      	itt	eq
 8000986:	4301      	orreq	r1, r0
 8000988:	2000      	moveq	r0, #0
 800098a:	f1b4 0cfd 	subs.w	ip, r4, #253	; 0xfd
 800098e:	bf88      	it	hi
 8000990:	f5bc 6fe0 	cmphi.w	ip, #1792	; 0x700
 8000994:	f63f aeaf 	bhi.w	80006f6 <__aeabi_dmul+0xde>
 8000998:	ebb5 0c03 	subs.w	ip, r5, r3
 800099c:	bf04      	itt	eq
 800099e:	ebb6 0c02 	subseq.w	ip, r6, r2
 80009a2:	ea5f 0c50 	movseq.w	ip, r0, lsr #1
 80009a6:	f150 0000 	adcs.w	r0, r0, #0
 80009aa:	eb41 5104 	adc.w	r1, r1, r4, lsl #20
 80009ae:	bd70      	pop	{r4, r5, r6, pc}
 80009b0:	f00e 4e00 	and.w	lr, lr, #2147483648	; 0x80000000
 80009b4:	ea4e 3111 	orr.w	r1, lr, r1, lsr #12
 80009b8:	eb14 045c 	adds.w	r4, r4, ip, lsr #1
 80009bc:	bfc2      	ittt	gt
 80009be:	ebd4 050c 	rsbsgt	r5, r4, ip
 80009c2:	ea41 5104 	orrgt.w	r1, r1, r4, lsl #20
 80009c6:	bd70      	popgt	{r4, r5, r6, pc}
 80009c8:	f441 1180 	orr.w	r1, r1, #1048576	; 0x100000
 80009cc:	f04f 0e00 	mov.w	lr, #0
 80009d0:	3c01      	subs	r4, #1
 80009d2:	e690      	b.n	80006f6 <__aeabi_dmul+0xde>
 80009d4:	ea45 0e06 	orr.w	lr, r5, r6
 80009d8:	e68d      	b.n	80006f6 <__aeabi_dmul+0xde>
 80009da:	ea0c 5513 	and.w	r5, ip, r3, lsr #20
 80009de:	ea94 0f0c 	teq	r4, ip
 80009e2:	bf08      	it	eq
 80009e4:	ea95 0f0c 	teqeq	r5, ip
 80009e8:	f43f af3b 	beq.w	8000862 <__aeabi_dmul+0x24a>
 80009ec:	ea94 0f0c 	teq	r4, ip
 80009f0:	d10a      	bne.n	8000a08 <__aeabi_ddiv+0x19c>
 80009f2:	ea50 3401 	orrs.w	r4, r0, r1, lsl #12
 80009f6:	f47f af34 	bne.w	8000862 <__aeabi_dmul+0x24a>
 80009fa:	ea95 0f0c 	teq	r5, ip
 80009fe:	f47f af25 	bne.w	800084c <__aeabi_dmul+0x234>
 8000a02:	4610      	mov	r0, r2
 8000a04:	4619      	mov	r1, r3
 8000a06:	e72c      	b.n	8000862 <__aeabi_dmul+0x24a>
 8000a08:	ea95 0f0c 	teq	r5, ip
 8000a0c:	d106      	bne.n	8000a1c <__aeabi_ddiv+0x1b0>
 8000a0e:	ea52 3503 	orrs.w	r5, r2, r3, lsl #12
 8000a12:	f43f aefd 	beq.w	8000810 <__aeabi_dmul+0x1f8>
 8000a16:	4610      	mov	r0, r2
 8000a18:	4619      	mov	r1, r3
 8000a1a:	e722      	b.n	8000862 <__aeabi_dmul+0x24a>
 8000a1c:	ea50 0641 	orrs.w	r6, r0, r1, lsl #1
 8000a20:	bf18      	it	ne
 8000a22:	ea52 0643 	orrsne.w	r6, r2, r3, lsl #1
 8000a26:	f47f aec5 	bne.w	80007b4 <__aeabi_dmul+0x19c>
 8000a2a:	ea50 0441 	orrs.w	r4, r0, r1, lsl #1
 8000a2e:	f47f af0d 	bne.w	800084c <__aeabi_dmul+0x234>
 8000a32:	ea52 0543 	orrs.w	r5, r2, r3, lsl #1
 8000a36:	f47f aeeb 	bne.w	8000810 <__aeabi_dmul+0x1f8>
 8000a3a:	e712      	b.n	8000862 <__aeabi_dmul+0x24a>

08000a3c <__gedf2>:
 8000a3c:	f04f 3cff 	mov.w	ip, #4294967295
 8000a40:	e006      	b.n	8000a50 <__cmpdf2+0x4>
 8000a42:	bf00      	nop

08000a44 <__ledf2>:
 8000a44:	f04f 0c01 	mov.w	ip, #1
 8000a48:	e002      	b.n	8000a50 <__cmpdf2+0x4>
 8000a4a:	bf00      	nop

08000a4c <__cmpdf2>:
 8000a4c:	f04f 0c01 	mov.w	ip, #1
 8000a50:	f84d cd04 	str.w	ip, [sp, #-4]!
 8000a54:	ea4f 0c41 	mov.w	ip, r1, lsl #1
 8000a58:	ea7f 5c6c 	mvns.w	ip, ip, asr #21
 8000a5c:	ea4f 0c43 	mov.w	ip, r3, lsl #1
 8000a60:	bf18      	it	ne
 8000a62:	ea7f 5c6c 	mvnsne.w	ip, ip, asr #21
 8000a66:	d01b      	beq.n	8000aa0 <__cmpdf2+0x54>
 8000a68:	b001      	add	sp, #4
 8000a6a:	ea50 0c41 	orrs.w	ip, r0, r1, lsl #1
 8000a6e:	bf0c      	ite	eq
 8000a70:	ea52 0c43 	orrseq.w	ip, r2, r3, lsl #1
 8000a74:	ea91 0f03 	teqne	r1, r3
 8000a78:	bf02      	ittt	eq
 8000a7a:	ea90 0f02 	teqeq	r0, r2
 8000a7e:	2000      	moveq	r0, #0
 8000a80:	4770      	bxeq	lr
 8000a82:	f110 0f00 	cmn.w	r0, #0
 8000a86:	ea91 0f03 	teq	r1, r3
 8000a8a:	bf58      	it	pl
 8000a8c:	4299      	cmppl	r1, r3
 8000a8e:	bf08      	it	eq
 8000a90:	4290      	cmpeq	r0, r2
 8000a92:	bf2c      	ite	cs
 8000a94:	17d8      	asrcs	r0, r3, #31
 8000a96:	ea6f 70e3 	mvncc.w	r0, r3, asr #31
 8000a9a:	f040 0001 	orr.w	r0, r0, #1
 8000a9e:	4770      	bx	lr
 8000aa0:	ea4f 0c41 	mov.w	ip, r1, lsl #1
 8000aa4:	ea7f 5c6c 	mvns.w	ip, ip, asr #21
 8000aa8:	d102      	bne.n	8000ab0 <__cmpdf2+0x64>
 8000aaa:	ea50 3c01 	orrs.w	ip, r0, r1, lsl #12
 8000aae:	d107      	bne.n	8000ac0 <__cmpdf2+0x74>
 8000ab0:	ea4f 0c43 	mov.w	ip, r3, lsl #1
 8000ab4:	ea7f 5c6c 	mvns.w	ip, ip, asr #21
 8000ab8:	d1d6      	bne.n	8000a68 <__cmpdf2+0x1c>
 8000aba:	ea52 3c03 	orrs.w	ip, r2, r3, lsl #12
 8000abe:	d0d3      	beq.n	8000a68 <__cmpdf2+0x1c>
 8000ac0:	f85d 0b04 	ldr.w	r0, [sp], #4
 8000ac4:	4770      	bx	lr
 8000ac6:	bf00      	nop

08000ac8 <__aeabi_cdrcmple>:
 8000ac8:	4684      	mov	ip, r0
 8000aca:	4610      	mov	r0, r2
 8000acc:	4662      	mov	r2, ip
 8000ace:	468c      	mov	ip, r1
 8000ad0:	4619      	mov	r1, r3
 8000ad2:	4663      	mov	r3, ip
 8000ad4:	e000      	b.n	8000ad8 <__aeabi_cdcmpeq>
 8000ad6:	bf00      	nop

08000ad8 <__aeabi_cdcmpeq>:
 8000ad8:	b501      	push	{r0, lr}
 8000ada:	f7ff ffb7 	bl	8000a4c <__cmpdf2>
 8000ade:	2800      	cmp	r0, #0
 8000ae0:	bf48      	it	mi
 8000ae2:	f110 0f00 	cmnmi.w	r0, #0
 8000ae6:	bd01      	pop	{r0, pc}

08000ae8 <__aeabi_dcmpeq>:
 8000ae8:	f84d ed08 	str.w	lr, [sp, #-8]!
 8000aec:	f7ff fff4 	bl	8000ad8 <__aeabi_cdcmpeq>
 8000af0:	bf0c      	ite	eq
 8000af2:	2001      	moveq	r0, #1
 8000af4:	2000      	movne	r0, #0
 8000af6:	f85d fb08 	ldr.w	pc, [sp], #8
 8000afa:	bf00      	nop

08000afc <__aeabi_dcmplt>:
 8000afc:	f84d ed08 	str.w	lr, [sp, #-8]!
 8000b00:	f7ff ffea 	bl	8000ad8 <__aeabi_cdcmpeq>
 8000b04:	bf34      	ite	cc
 8000b06:	2001      	movcc	r0, #1
 8000b08:	2000      	movcs	r0, #0
 8000b0a:	f85d fb08 	ldr.w	pc, [sp], #8
 8000b0e:	bf00      	nop

08000b10 <__aeabi_dcmple>:
 8000b10:	f84d ed08 	str.w	lr, [sp, #-8]!
 8000b14:	f7ff ffe0 	bl	8000ad8 <__aeabi_cdcmpeq>
 8000b18:	bf94      	ite	ls
 8000b1a:	2001      	movls	r0, #1
 8000b1c:	2000      	movhi	r0, #0
 8000b1e:	f85d fb08 	ldr.w	pc, [sp], #8
 8000b22:	bf00      	nop

08000b24 <__aeabi_dcmpge>:
 8000b24:	f84d ed08 	str.w	lr, [sp, #-8]!
 8000b28:	f7ff ffce 	bl	8000ac8 <__aeabi_cdrcmple>
 8000b2c:	bf94      	ite	ls
 8000b2e:	2001      	movls	r0, #1
 8000b30:	2000      	movhi	r0, #0
 8000b32:	f85d fb08 	ldr.w	pc, [sp], #8
 8000b36:	bf00      	nop

08000b38 <__aeabi_dcmpgt>:
 8000b38:	f84d ed08 	str.w	lr, [sp, #-8]!
 8000b3c:	f7ff ffc4 	bl	8000ac8 <__aeabi_cdrcmple>
 8000b40:	bf34      	ite	cc
 8000b42:	2001      	movcc	r0, #1
 8000b44:	2000      	movcs	r0, #0
 8000b46:	f85d fb08 	ldr.w	pc, [sp], #8
 8000b4a:	bf00      	nop

08000b4c <__aeabi_dcmpun>:
 8000b4c:	ea4f 0c41 	mov.w	ip, r1, lsl #1
 8000b50:	ea7f 5c6c 	mvns.w	ip, ip, asr #21
 8000b54:	d102      	bne.n	8000b5c <__aeabi_dcmpun+0x10>
 8000b56:	ea50 3c01 	orrs.w	ip, r0, r1, lsl #12
 8000b5a:	d10a      	bne.n	8000b72 <__aeabi_dcmpun+0x26>
 8000b5c:	ea4f 0c43 	mov.w	ip, r3, lsl #1
 8000b60:	ea7f 5c6c 	mvns.w	ip, ip, asr #21
 8000b64:	d102      	bne.n	8000b6c <__aeabi_dcmpun+0x20>
 8000b66:	ea52 3c03 	orrs.w	ip, r2, r3, lsl #12
 8000b6a:	d102      	bne.n	8000b72 <__aeabi_dcmpun+0x26>
 8000b6c:	f04f 0000 	mov.w	r0, #0
 8000b70:	4770      	bx	lr
 8000b72:	f04f 0001 	mov.w	r0, #1
 8000b76:	4770      	bx	lr

08000b78 <__aeabi_d2iz>:
 8000b78:	ea4f 0241 	mov.w	r2, r1, lsl #1
 8000b7c:	f512 1200 	adds.w	r2, r2, #2097152	; 0x200000
 8000b80:	d215      	bcs.n	8000bae <__aeabi_d2iz+0x36>
 8000b82:	d511      	bpl.n	8000ba8 <__aeabi_d2iz+0x30>
 8000b84:	f46f 7378 	mvn.w	r3, #992	; 0x3e0
 8000b88:	ebb3 5262 	subs.w	r2, r3, r2, asr #21
 8000b8c:	d912      	bls.n	8000bb4 <__aeabi_d2iz+0x3c>
 8000b8e:	ea4f 23c1 	mov.w	r3, r1, lsl #11
 8000b92:	f043 4300 	orr.w	r3, r3, #2147483648	; 0x80000000
 8000b96:	ea43 5350 	orr.w	r3, r3, r0, lsr #21
 8000b9a:	f011 4f00 	tst.w	r1, #2147483648	; 0x80000000
 8000b9e:	fa23 f002 	lsr.w	r0, r3, r2
 8000ba2:	bf18      	it	ne
 8000ba4:	4240      	negne	r0, r0
 8000ba6:	4770      	bx	lr
 8000ba8:	f04f 0000 	mov.w	r0, #0
 8000bac:	4770      	bx	lr
 8000bae:	ea50 3001 	orrs.w	r0, r0, r1, lsl #12
 8000bb2:	d105      	bne.n	8000bc0 <__aeabi_d2iz+0x48>
 8000bb4:	f011 4000 	ands.w	r0, r1, #2147483648	; 0x80000000
 8000bb8:	bf08      	it	eq
 8000bba:	f06f 4000 	mvneq.w	r0, #2147483648	; 0x80000000
 8000bbe:	4770      	bx	lr
 8000bc0:	f04f 0000 	mov.w	r0, #0
 8000bc4:	4770      	bx	lr
 8000bc6:	bf00      	nop

08000bc8 <__aeabi_d2f>:
 8000bc8:	ea4f 0241 	mov.w	r2, r1, lsl #1
 8000bcc:	f1b2 43e0 	subs.w	r3, r2, #1879048192	; 0x70000000
 8000bd0:	bf24      	itt	cs
 8000bd2:	f5b3 1c00 	subscs.w	ip, r3, #2097152	; 0x200000
 8000bd6:	f1dc 5cfe 	rsbscs	ip, ip, #532676608	; 0x1fc00000
 8000bda:	d90d      	bls.n	8000bf8 <__aeabi_d2f+0x30>
 8000bdc:	f001 4c00 	and.w	ip, r1, #2147483648	; 0x80000000
 8000be0:	ea4f 02c0 	mov.w	r2, r0, lsl #3
 8000be4:	ea4c 7050 	orr.w	r0, ip, r0, lsr #29
 8000be8:	f1b2 4f00 	cmp.w	r2, #2147483648	; 0x80000000
 8000bec:	eb40 0083 	adc.w	r0, r0, r3, lsl #2
 8000bf0:	bf08      	it	eq
 8000bf2:	f020 0001 	biceq.w	r0, r0, #1
 8000bf6:	4770      	bx	lr
 8000bf8:	f011 4f80 	tst.w	r1, #1073741824	; 0x40000000
 8000bfc:	d121      	bne.n	8000c42 <__aeabi_d2f+0x7a>
 8000bfe:	f113 7238 	adds.w	r2, r3, #48234496	; 0x2e00000
 8000c02:	bfbc      	itt	lt
 8000c04:	f001 4000 	andlt.w	r0, r1, #2147483648	; 0x80000000
 8000c08:	4770      	bxlt	lr
 8000c0a:	f441 1180 	orr.w	r1, r1, #1048576	; 0x100000
 8000c0e:	ea4f 5252 	mov.w	r2, r2, lsr #21
 8000c12:	f1c2 0218 	rsb	r2, r2, #24
 8000c16:	f1c2 0c20 	rsb	ip, r2, #32
 8000c1a:	fa10 f30c 	lsls.w	r3, r0, ip
 8000c1e:	fa20 f002 	lsr.w	r0, r0, r2
 8000c22:	bf18      	it	ne
 8000c24:	f040 0001 	orrne.w	r0, r0, #1
 8000c28:	ea4f 23c1 	mov.w	r3, r1, lsl #11
 8000c2c:	ea4f 23d3 	mov.w	r3, r3, lsr #11
 8000c30:	fa03 fc0c 	lsl.w	ip, r3, ip
 8000c34:	ea40 000c 	orr.w	r0, r0, ip
 8000c38:	fa23 f302 	lsr.w	r3, r3, r2
 8000c3c:	ea4f 0343 	mov.w	r3, r3, lsl #1
 8000c40:	e7cc      	b.n	8000bdc <__aeabi_d2f+0x14>
 8000c42:	ea7f 5362 	mvns.w	r3, r2, asr #21
 8000c46:	d107      	bne.n	8000c58 <__aeabi_d2f+0x90>
 8000c48:	ea50 3301 	orrs.w	r3, r0, r1, lsl #12
 8000c4c:	bf1e      	ittt	ne
 8000c4e:	f04f 40fe 	movne.w	r0, #2130706432	; 0x7f000000
 8000c52:	f440 0040 	orrne.w	r0, r0, #12582912	; 0xc00000
 8000c56:	4770      	bxne	lr
 8000c58:	f001 4000 	and.w	r0, r1, #2147483648	; 0x80000000
 8000c5c:	f040 40fe 	orr.w	r0, r0, #2130706432	; 0x7f000000
 8000c60:	f440 0000 	orr.w	r0, r0, #8388608	; 0x800000
 8000c64:	4770      	bx	lr
 8000c66:	bf00      	nop

08000c68 <__aeabi_uldivmod>:
 8000c68:	b953      	cbnz	r3, 8000c80 <__aeabi_uldivmod+0x18>
 8000c6a:	b94a      	cbnz	r2, 8000c80 <__aeabi_uldivmod+0x18>
 8000c6c:	2900      	cmp	r1, #0
 8000c6e:	bf08      	it	eq
 8000c70:	2800      	cmpeq	r0, #0
 8000c72:	bf1c      	itt	ne
 8000c74:	f04f 31ff 	movne.w	r1, #4294967295
 8000c78:	f04f 30ff 	movne.w	r0, #4294967295
 8000c7c:	f000 b974 	b.w	8000f68 <__aeabi_idiv0>
 8000c80:	f1ad 0c08 	sub.w	ip, sp, #8
 8000c84:	e96d ce04 	strd	ip, lr, [sp, #-16]!
 8000c88:	f000 f806 	bl	8000c98 <__udivmoddi4>
 8000c8c:	f8dd e004 	ldr.w	lr, [sp, #4]
 8000c90:	e9dd 2302 	ldrd	r2, r3, [sp, #8]
 8000c94:	b004      	add	sp, #16
 8000c96:	4770      	bx	lr

08000c98 <__udivmoddi4>:
 8000c98:	e92d 47f0 	stmdb	sp!, {r4, r5, r6, r7, r8, r9, sl, lr}
 8000c9c:	9d08      	ldr	r5, [sp, #32]
 8000c9e:	4604      	mov	r4, r0
 8000ca0:	468e      	mov	lr, r1
 8000ca2:	2b00      	cmp	r3, #0
 8000ca4:	d14d      	bne.n	8000d42 <__udivmoddi4+0xaa>
 8000ca6:	428a      	cmp	r2, r1
 8000ca8:	4694      	mov	ip, r2
 8000caa:	d969      	bls.n	8000d80 <__udivmoddi4+0xe8>
 8000cac:	fab2 f282 	clz	r2, r2
 8000cb0:	b152      	cbz	r2, 8000cc8 <__udivmoddi4+0x30>
 8000cb2:	fa01 f302 	lsl.w	r3, r1, r2
 8000cb6:	f1c2 0120 	rsb	r1, r2, #32
 8000cba:	fa20 f101 	lsr.w	r1, r0, r1
 8000cbe:	fa0c fc02 	lsl.w	ip, ip, r2
 8000cc2:	ea41 0e03 	orr.w	lr, r1, r3
 8000cc6:	4094      	lsls	r4, r2
 8000cc8:	ea4f 481c 	mov.w	r8, ip, lsr #16
 8000ccc:	0c21      	lsrs	r1, r4, #16
 8000cce:	fbbe f6f8 	udiv	r6, lr, r8
 8000cd2:	fa1f f78c 	uxth.w	r7, ip
 8000cd6:	fb08 e316 	mls	r3, r8, r6, lr
 8000cda:	ea41 4303 	orr.w	r3, r1, r3, lsl #16
 8000cde:	fb06 f107 	mul.w	r1, r6, r7
 8000ce2:	4299      	cmp	r1, r3
 8000ce4:	d90a      	bls.n	8000cfc <__udivmoddi4+0x64>
 8000ce6:	eb1c 0303 	adds.w	r3, ip, r3
 8000cea:	f106 30ff 	add.w	r0, r6, #4294967295
 8000cee:	f080 811f 	bcs.w	8000f30 <__udivmoddi4+0x298>
 8000cf2:	4299      	cmp	r1, r3
 8000cf4:	f240 811c 	bls.w	8000f30 <__udivmoddi4+0x298>
 8000cf8:	3e02      	subs	r6, #2
 8000cfa:	4463      	add	r3, ip
 8000cfc:	1a5b      	subs	r3, r3, r1
 8000cfe:	b2a4      	uxth	r4, r4
 8000d00:	fbb3 f0f8 	udiv	r0, r3, r8
 8000d04:	fb08 3310 	mls	r3, r8, r0, r3
 8000d08:	ea44 4403 	orr.w	r4, r4, r3, lsl #16
 8000d0c:	fb00 f707 	mul.w	r7, r0, r7
 8000d10:	42a7      	cmp	r7, r4
 8000d12:	d90a      	bls.n	8000d2a <__udivmoddi4+0x92>
 8000d14:	eb1c 0404 	adds.w	r4, ip, r4
 8000d18:	f100 33ff 	add.w	r3, r0, #4294967295
 8000d1c:	f080 810a 	bcs.w	8000f34 <__udivmoddi4+0x29c>
 8000d20:	42a7      	cmp	r7, r4
 8000d22:	f240 8107 	bls.w	8000f34 <__udivmoddi4+0x29c>
 8000d26:	4464      	add	r4, ip
 8000d28:	3802      	subs	r0, #2
 8000d2a:	ea40 4006 	orr.w	r0, r0, r6, lsl #16
 8000d2e:	1be4      	subs	r4, r4, r7
 8000d30:	2600      	movs	r6, #0
 8000d32:	b11d      	cbz	r5, 8000d3c <__udivmoddi4+0xa4>
 8000d34:	40d4      	lsrs	r4, r2
 8000d36:	2300      	movs	r3, #0
 8000d38:	e9c5 4300 	strd	r4, r3, [r5]
 8000d3c:	4631      	mov	r1, r6
 8000d3e:	e8bd 87f0 	ldmia.w	sp!, {r4, r5, r6, r7, r8, r9, sl, pc}
 8000d42:	428b      	cmp	r3, r1
 8000d44:	d909      	bls.n	8000d5a <__udivmoddi4+0xc2>
 8000d46:	2d00      	cmp	r5, #0
 8000d48:	f000 80ef 	beq.w	8000f2a <__udivmoddi4+0x292>
 8000d4c:	2600      	movs	r6, #0
 8000d4e:	e9c5 0100 	strd	r0, r1, [r5]
 8000d52:	4630      	mov	r0, r6
 8000d54:	4631      	mov	r1, r6
 8000d56:	e8bd 87f0 	ldmia.w	sp!, {r4, r5, r6, r7, r8, r9, sl, pc}
 8000d5a:	fab3 f683 	clz	r6, r3
 8000d5e:	2e00      	cmp	r6, #0
 8000d60:	d14a      	bne.n	8000df8 <__udivmoddi4+0x160>
 8000d62:	428b      	cmp	r3, r1
 8000d64:	d302      	bcc.n	8000d6c <__udivmoddi4+0xd4>
 8000d66:	4282      	cmp	r2, r0
 8000d68:	f200 80f9 	bhi.w	8000f5e <__udivmoddi4+0x2c6>
 8000d6c:	1a84      	subs	r4, r0, r2
 8000d6e:	eb61 0303 	sbc.w	r3, r1, r3
 8000d72:	2001      	movs	r0, #1
 8000d74:	469e      	mov	lr, r3
 8000d76:	2d00      	cmp	r5, #0
 8000d78:	d0e0      	beq.n	8000d3c <__udivmoddi4+0xa4>
 8000d7a:	e9c5 4e00 	strd	r4, lr, [r5]
 8000d7e:	e7dd      	b.n	8000d3c <__udivmoddi4+0xa4>
 8000d80:	b902      	cbnz	r2, 8000d84 <__udivmoddi4+0xec>
 8000d82:	deff      	udf	#255	; 0xff
 8000d84:	fab2 f282 	clz	r2, r2
 8000d88:	2a00      	cmp	r2, #0
 8000d8a:	f040 8092 	bne.w	8000eb2 <__udivmoddi4+0x21a>
 8000d8e:	eba1 010c 	sub.w	r1, r1, ip
 8000d92:	ea4f 471c 	mov.w	r7, ip, lsr #16
 8000d96:	fa1f fe8c 	uxth.w	lr, ip
 8000d9a:	2601      	movs	r6, #1
 8000d9c:	0c20      	lsrs	r0, r4, #16
 8000d9e:	fbb1 f3f7 	udiv	r3, r1, r7
 8000da2:	fb07 1113 	mls	r1, r7, r3, r1
 8000da6:	ea40 4101 	orr.w	r1, r0, r1, lsl #16
 8000daa:	fb0e f003 	mul.w	r0, lr, r3
 8000dae:	4288      	cmp	r0, r1
 8000db0:	d908      	bls.n	8000dc4 <__udivmoddi4+0x12c>
 8000db2:	eb1c 0101 	adds.w	r1, ip, r1
 8000db6:	f103 38ff 	add.w	r8, r3, #4294967295
 8000dba:	d202      	bcs.n	8000dc2 <__udivmoddi4+0x12a>
 8000dbc:	4288      	cmp	r0, r1
 8000dbe:	f200 80cb 	bhi.w	8000f58 <__udivmoddi4+0x2c0>
 8000dc2:	4643      	mov	r3, r8
 8000dc4:	1a09      	subs	r1, r1, r0
 8000dc6:	b2a4      	uxth	r4, r4
 8000dc8:	fbb1 f0f7 	udiv	r0, r1, r7
 8000dcc:	fb07 1110 	mls	r1, r7, r0, r1
 8000dd0:	ea44 4401 	orr.w	r4, r4, r1, lsl #16
 8000dd4:	fb0e fe00 	mul.w	lr, lr, r0
 8000dd8:	45a6      	cmp	lr, r4
 8000dda:	d908      	bls.n	8000dee <__udivmoddi4+0x156>
 8000ddc:	eb1c 0404 	adds.w	r4, ip, r4
 8000de0:	f100 31ff 	add.w	r1, r0, #4294967295
 8000de4:	d202      	bcs.n	8000dec <__udivmoddi4+0x154>
 8000de6:	45a6      	cmp	lr, r4
 8000de8:	f200 80bb 	bhi.w	8000f62 <__udivmoddi4+0x2ca>
 8000dec:	4608      	mov	r0, r1
 8000dee:	eba4 040e 	sub.w	r4, r4, lr
 8000df2:	ea40 4003 	orr.w	r0, r0, r3, lsl #16
 8000df6:	e79c      	b.n	8000d32 <__udivmoddi4+0x9a>
 8000df8:	f1c6 0720 	rsb	r7, r6, #32
 8000dfc:	40b3      	lsls	r3, r6
 8000dfe:	fa22 fc07 	lsr.w	ip, r2, r7
 8000e02:	ea4c 0c03 	orr.w	ip, ip, r3
 8000e06:	fa20 f407 	lsr.w	r4, r0, r7
 8000e0a:	fa01 f306 	lsl.w	r3, r1, r6
 8000e0e:	431c      	orrs	r4, r3
 8000e10:	40f9      	lsrs	r1, r7
 8000e12:	ea4f 491c 	mov.w	r9, ip, lsr #16
 8000e16:	fa00 f306 	lsl.w	r3, r0, r6
 8000e1a:	fbb1 f8f9 	udiv	r8, r1, r9
 8000e1e:	0c20      	lsrs	r0, r4, #16
 8000e20:	fa1f fe8c 	uxth.w	lr, ip
 8000e24:	fb09 1118 	mls	r1, r9, r8, r1
 8000e28:	ea40 4101 	orr.w	r1, r0, r1, lsl #16
 8000e2c:	fb08 f00e 	mul.w	r0, r8, lr
 8000e30:	4288      	cmp	r0, r1
 8000e32:	fa02 f206 	lsl.w	r2, r2, r6
 8000e36:	d90b      	bls.n	8000e50 <__udivmoddi4+0x1b8>
 8000e38:	eb1c 0101 	adds.w	r1, ip, r1
 8000e3c:	f108 3aff 	add.w	sl, r8, #4294967295
 8000e40:	f080 8088 	bcs.w	8000f54 <__udivmoddi4+0x2bc>
 8000e44:	4288      	cmp	r0, r1
 8000e46:	f240 8085 	bls.w	8000f54 <__udivmoddi4+0x2bc>
 8000e4a:	f1a8 0802 	sub.w	r8, r8, #2
 8000e4e:	4461      	add	r1, ip
 8000e50:	1a09      	subs	r1, r1, r0
 8000e52:	b2a4      	uxth	r4, r4
 8000e54:	fbb1 f0f9 	udiv	r0, r1, r9
 8000e58:	fb09 1110 	mls	r1, r9, r0, r1
 8000e5c:	ea44 4101 	orr.w	r1, r4, r1, lsl #16
 8000e60:	fb00 fe0e 	mul.w	lr, r0, lr
 8000e64:	458e      	cmp	lr, r1
 8000e66:	d908      	bls.n	8000e7a <__udivmoddi4+0x1e2>
 8000e68:	eb1c 0101 	adds.w	r1, ip, r1
 8000e6c:	f100 34ff 	add.w	r4, r0, #4294967295
 8000e70:	d26c      	bcs.n	8000f4c <__udivmoddi4+0x2b4>
 8000e72:	458e      	cmp	lr, r1
 8000e74:	d96a      	bls.n	8000f4c <__udivmoddi4+0x2b4>
 8000e76:	3802      	subs	r0, #2
 8000e78:	4461      	add	r1, ip
 8000e7a:	ea40 4008 	orr.w	r0, r0, r8, lsl #16
 8000e7e:	fba0 9402 	umull	r9, r4, r0, r2
 8000e82:	eba1 010e 	sub.w	r1, r1, lr
 8000e86:	42a1      	cmp	r1, r4
 8000e88:	46c8      	mov	r8, r9
 8000e8a:	46a6      	mov	lr, r4
 8000e8c:	d356      	bcc.n	8000f3c <__udivmoddi4+0x2a4>
 8000e8e:	d053      	beq.n	8000f38 <__udivmoddi4+0x2a0>
 8000e90:	b15d      	cbz	r5, 8000eaa <__udivmoddi4+0x212>
 8000e92:	ebb3 0208 	subs.w	r2, r3, r8
 8000e96:	eb61 010e 	sbc.w	r1, r1, lr
 8000e9a:	fa01 f707 	lsl.w	r7, r1, r7
 8000e9e:	fa22 f306 	lsr.w	r3, r2, r6
 8000ea2:	40f1      	lsrs	r1, r6
 8000ea4:	431f      	orrs	r7, r3
 8000ea6:	e9c5 7100 	strd	r7, r1, [r5]
 8000eaa:	2600      	movs	r6, #0
 8000eac:	4631      	mov	r1, r6
 8000eae:	e8bd 87f0 	ldmia.w	sp!, {r4, r5, r6, r7, r8, r9, sl, pc}
 8000eb2:	f1c2 0320 	rsb	r3, r2, #32
 8000eb6:	40d8      	lsrs	r0, r3
 8000eb8:	fa0c fc02 	lsl.w	ip, ip, r2
 8000ebc:	fa21 f303 	lsr.w	r3, r1, r3
 8000ec0:	4091      	lsls	r1, r2
 8000ec2:	4301      	orrs	r1, r0
 8000ec4:	ea4f 471c 	mov.w	r7, ip, lsr #16
 8000ec8:	fa1f fe8c 	uxth.w	lr, ip
 8000ecc:	fbb3 f0f7 	udiv	r0, r3, r7
 8000ed0:	fb07 3610 	mls	r6, r7, r0, r3
 8000ed4:	0c0b      	lsrs	r3, r1, #16
 8000ed6:	ea43 4306 	orr.w	r3, r3, r6, lsl #16
 8000eda:	fb00 f60e 	mul.w	r6, r0, lr
 8000ede:	429e      	cmp	r6, r3
 8000ee0:	fa04 f402 	lsl.w	r4, r4, r2
 8000ee4:	d908      	bls.n	8000ef8 <__udivmoddi4+0x260>
 8000ee6:	eb1c 0303 	adds.w	r3, ip, r3
 8000eea:	f100 38ff 	add.w	r8, r0, #4294967295
 8000eee:	d22f      	bcs.n	8000f50 <__udivmoddi4+0x2b8>
 8000ef0:	429e      	cmp	r6, r3
 8000ef2:	d92d      	bls.n	8000f50 <__udivmoddi4+0x2b8>
 8000ef4:	3802      	subs	r0, #2
 8000ef6:	4463      	add	r3, ip
 8000ef8:	1b9b      	subs	r3, r3, r6
 8000efa:	b289      	uxth	r1, r1
 8000efc:	fbb3 f6f7 	udiv	r6, r3, r7
 8000f00:	fb07 3316 	mls	r3, r7, r6, r3
 8000f04:	ea41 4103 	orr.w	r1, r1, r3, lsl #16
 8000f08:	fb06 f30e 	mul.w	r3, r6, lr
 8000f0c:	428b      	cmp	r3, r1
 8000f0e:	d908      	bls.n	8000f22 <__udivmoddi4+0x28a>
 8000f10:	eb1c 0101 	adds.w	r1, ip, r1
 8000f14:	f106 38ff 	add.w	r8, r6, #4294967295
 8000f18:	d216      	bcs.n	8000f48 <__udivmoddi4+0x2b0>
 8000f1a:	428b      	cmp	r3, r1
 8000f1c:	d914      	bls.n	8000f48 <__udivmoddi4+0x2b0>
 8000f1e:	3e02      	subs	r6, #2
 8000f20:	4461      	add	r1, ip
 8000f22:	1ac9      	subs	r1, r1, r3
 8000f24:	ea46 4600 	orr.w	r6, r6, r0, lsl #16
 8000f28:	e738      	b.n	8000d9c <__udivmoddi4+0x104>
 8000f2a:	462e      	mov	r6, r5
 8000f2c:	4628      	mov	r0, r5
 8000f2e:	e705      	b.n	8000d3c <__udivmoddi4+0xa4>
 8000f30:	4606      	mov	r6, r0
 8000f32:	e6e3      	b.n	8000cfc <__udivmoddi4+0x64>
 8000f34:	4618      	mov	r0, r3
 8000f36:	e6f8      	b.n	8000d2a <__udivmoddi4+0x92>
 8000f38:	454b      	cmp	r3, r9
 8000f3a:	d2a9      	bcs.n	8000e90 <__udivmoddi4+0x1f8>
 8000f3c:	ebb9 0802 	subs.w	r8, r9, r2
 8000f40:	eb64 0e0c 	sbc.w	lr, r4, ip
 8000f44:	3801      	subs	r0, #1
 8000f46:	e7a3      	b.n	8000e90 <__udivmoddi4+0x1f8>
 8000f48:	4646      	mov	r6, r8
 8000f4a:	e7ea      	b.n	8000f22 <__udivmoddi4+0x28a>
 8000f4c:	4620      	mov	r0, r4
 8000f4e:	e794      	b.n	8000e7a <__udivmoddi4+0x1e2>
 8000f50:	4640      	mov	r0, r8
 8000f52:	e7d1      	b.n	8000ef8 <__udivmoddi4+0x260>
 8000f54:	46d0      	mov	r8, sl
 8000f56:	e77b      	b.n	8000e50 <__udivmoddi4+0x1b8>
 8000f58:	3b02      	subs	r3, #2
 8000f5a:	4461      	add	r1, ip
 8000f5c:	e732      	b.n	8000dc4 <__udivmoddi4+0x12c>
 8000f5e:	4630      	mov	r0, r6
 8000f60:	e709      	b.n	8000d76 <__udivmoddi4+0xde>
 8000f62:	4464      	add	r4, ip
 8000f64:	3802      	subs	r0, #2
 8000f66:	e742      	b.n	8000dee <__udivmoddi4+0x156>

08000f68 <__aeabi_idiv0>:
 8000f68:	4770      	bx	lr
 8000f6a:	bf00      	nop

08000f6c <Reset_Handler>:

    .section  .text.Reset_Handler
  .weak  Reset_Handler
  .type  Reset_Handler, %function
Reset_Handler: 
  ldr   sp, =_estack       /* set stack pointer */
 8000f6c:	f8df d034 	ldr.w	sp, [pc, #52]	; 8000fa4 <LoopFillZerobss+0x14>
 
/* Copy the data segment initializers from flash to SRAM */  
  movs  r1, #0
 8000f70:	2100      	movs	r1, #0
  b  LoopCopyDataInit
 8000f72:	e003      	b.n	8000f7c <LoopCopyDataInit>

08000f74 <CopyDataInit>:

CopyDataInit:
  ldr  r3, =_sidata
 8000f74:	4b0c      	ldr	r3, [pc, #48]	; (8000fa8 <LoopFillZerobss+0x18>)
  ldr  r3, [r3, r1]
 8000f76:	585b      	ldr	r3, [r3, r1]
  str  r3, [r0, r1]
 8000f78:	5043      	str	r3, [r0, r1]
  adds  r1, r1, #4
 8000f7a:	3104      	adds	r1, #4

08000f7c <LoopCopyDataInit>:
    
LoopCopyDataInit:
  ldr  r0, =_sdata
 8000f7c:	480b      	ldr	r0, [pc, #44]	; (8000fac <LoopFillZerobss+0x1c>)
  ldr  r3, =_edata
 8000f7e:	4b0c      	ldr	r3, [pc, #48]	; (8000fb0 <LoopFillZerobss+0x20>)
  adds  r2, r0, r1
 8000f80:	1842      	adds	r2, r0, r1
  cmp  r2, r3
 8000f82:	429a      	cmp	r2, r3
  bcc  CopyDataInit
 8000f84:	d3f6      	bcc.n	8000f74 <CopyDataInit>
  ldr  r2, =_sbss
 8000f86:	4a0b      	ldr	r2, [pc, #44]	; (8000fb4 <LoopFillZerobss+0x24>)
  b  LoopFillZerobss
 8000f88:	e002      	b.n	8000f90 <LoopFillZerobss>

08000f8a <FillZerobss>:
/* Zero fill the bss segment. */  
FillZerobss:
  movs  r3, #0
 8000f8a:	2300      	movs	r3, #0
  str  r3, [r2], #4
 8000f8c:	f842 3b04 	str.w	r3, [r2], #4

08000f90 <LoopFillZerobss>:
    
LoopFillZerobss:
  ldr  r3, = _ebss
 8000f90:	4b09      	ldr	r3, [pc, #36]	; (8000fb8 <LoopFillZerobss+0x28>)
  cmp  r2, r3
 8000f92:	429a      	cmp	r2, r3
  bcc  FillZerobss
 8000f94:	d3f9      	bcc.n	8000f8a <FillZerobss>

/* Call the clock system intitialization function.*/
  bl  SystemInit   
 8000f96:	f003 f9dd 	bl	8004354 <SystemInit>
/* Call static constructors */
    bl __libc_init_array
 8000f9a:	f01a fd8f 	bl	801babc <__libc_init_array>
/* Call the application's entry point.*/
  bl  main
 8000f9e:	f001 f89f 	bl	80020e0 <main>
  bx  lr    
 8000fa2:	4770      	bx	lr
  ldr   sp, =_estack       /* set stack pointer */
 8000fa4:	20030000 	.word	0x20030000
  ldr  r3, =_sidata
 8000fa8:	080ddc60 	.word	0x080ddc60
  ldr  r0, =_sdata
 8000fac:	20000000 	.word	0x20000000
  ldr  r3, =_edata
 8000fb0:	200002d0 	.word	0x200002d0
  ldr  r2, =_sbss
 8000fb4:	200002d0 	.word	0x200002d0
  ldr  r3, = _ebss
 8000fb8:	200128d4 	.word	0x200128d4

08000fbc <ADC_IRQHandler>:
 * @retval None       
*/
    .section  .text.Default_Handler,"ax",%progbits
Default_Handler:
Infinite_Loop:
  b  Infinite_Loop
 8000fbc:	e7fe      	b.n	8000fbc <ADC_IRQHandler>

08000fbe <MX_TouchGFX_Init>:
 * Initialize TouchGFX application
 */
void MX_TouchGFX_Init(void)
{
  // Calling farward to touchgfx_init in C++ domain
  touchgfx_init();
 8000fbe:	f000 bc23 	b.w	8001808 <touchgfx_init>

08000fc2 <TouchGFX_Task>:
 * TouchGFX application thread
 */
void TouchGFX_Task(void *argument)
{
  // Calling farward to touchgfx_taskEntry in C++ domain
  touchgfx_taskEntry();
 8000fc2:	f000 bc91 	b.w	80018e8 <touchgfx_taskEntry>

08000fc6 <_ZN20STM32TouchControllerD1Ev>:
 * @brief This class specializes TouchController Interface.
 *
 * @sa touchgfx::TouchController
 */

class STM32TouchController : public touchgfx::TouchController
 8000fc6:	4770      	bx	lr

08000fc8 <_ZN20STM32TouchControllerD0Ev>:
 8000fc8:	b510      	push	{r4, lr}
 8000fca:	2104      	movs	r1, #4
 8000fcc:	4604      	mov	r4, r0
 8000fce:	f01a fcfc 	bl	801b9ca <_ZdlPvj>
 8000fd2:	4620      	mov	r0, r4
 8000fd4:	bd10      	pop	{r4, pc}
	...

08000fd8 <_Z11BSP_TS_Inittt>:
  * @param  XSize: The maximum X size of the TS area on LCD
  * @param  YSize: The maximum Y size of the TS area on LCD
  * @retval TS_OK: if all initializations are OK. Other value if error.
  */
uint8_t BSP_TS_Init(uint16_t XSize, uint16_t YSize)
{
 8000fd8:	b538      	push	{r3, r4, r5, lr}
    uint8_t ret = TS_ERROR;

    /* Initialize x and y positions boundaries */
    TsXBoundary = XSize;
 8000fda:	4b0c      	ldr	r3, [pc, #48]	; (800100c <_Z11BSP_TS_Inittt+0x34>)
    TsYBoundary = YSize;

    /* Read ID and verify if the IO expander is ready */
    if (stmpe811_ts_drv.ReadID(TS_I2C_ADDRESS) == STMPE811_ID)
 8000fdc:	4c0c      	ldr	r4, [pc, #48]	; (8001010 <_Z11BSP_TS_Inittt+0x38>)
    TsXBoundary = XSize;
 8000fde:	8018      	strh	r0, [r3, #0]
    TsYBoundary = YSize;
 8000fe0:	4b0c      	ldr	r3, [pc, #48]	; (8001014 <_Z11BSP_TS_Inittt+0x3c>)
    if (stmpe811_ts_drv.ReadID(TS_I2C_ADDRESS) == STMPE811_ID)
 8000fe2:	2082      	movs	r0, #130	; 0x82
    TsYBoundary = YSize;
 8000fe4:	8019      	strh	r1, [r3, #0]
    if (stmpe811_ts_drv.ReadID(TS_I2C_ADDRESS) == STMPE811_ID)
 8000fe6:	6863      	ldr	r3, [r4, #4]
 8000fe8:	4798      	blx	r3
 8000fea:	f640 0311 	movw	r3, #2065	; 0x811
 8000fee:	4298      	cmp	r0, r3
 8000ff0:	d10a      	bne.n	8001008 <_Z11BSP_TS_Inittt+0x30>
    {
        /* Initialize the TS driver structure */
        TsDrv = &stmpe811_ts_drv;
 8000ff2:	4d09      	ldr	r5, [pc, #36]	; (8001018 <_Z11BSP_TS_Inittt+0x40>)
    }

    if (ret == TS_OK)
    {
        /* Initialize the LL TS Driver */
        TsDrv->Init(TS_I2C_ADDRESS);
 8000ff4:	6823      	ldr	r3, [r4, #0]
        TsDrv = &stmpe811_ts_drv;
 8000ff6:	602c      	str	r4, [r5, #0]
        TsDrv->Init(TS_I2C_ADDRESS);
 8000ff8:	2082      	movs	r0, #130	; 0x82
 8000ffa:	4798      	blx	r3
        TsDrv->Start(TS_I2C_ADDRESS);
 8000ffc:	682b      	ldr	r3, [r5, #0]
 8000ffe:	2082      	movs	r0, #130	; 0x82
 8001000:	68db      	ldr	r3, [r3, #12]
 8001002:	4798      	blx	r3
 8001004:	2000      	movs	r0, #0
    }

    return ret;
}
 8001006:	bd38      	pop	{r3, r4, r5, pc}
    uint8_t ret = TS_ERROR;
 8001008:	2001      	movs	r0, #1
 800100a:	e7fc      	b.n	8001006 <_Z11BSP_TS_Inittt+0x2e>
 800100c:	200002ec 	.word	0x200002ec
 8001010:	2000004c 	.word	0x2000004c
 8001014:	200002ee 	.word	0x200002ee
 8001018:	200002f0 	.word	0x200002f0

0800101c <_ZN20STM32TouchController4initEv>:
    BSP_TS_Init(240, 320);
 800101c:	f44f 71a0 	mov.w	r1, #320	; 0x140
 8001020:	20f0      	movs	r0, #240	; 0xf0
 8001022:	f7ff bfd9 	b.w	8000fd8 <_Z11BSP_TS_Inittt>
	...

08001028 <_Z15BSP_TS_GetStateP15TS_StateTypeDef>:
/**
  * @brief  Returns status and positions of the touch screen.
  * @param  TsState: Pointer to touch screen current state structure
  */
void BSP_TS_GetState(TS_StateTypeDef* TsState)
{
 8001028:	b5f7      	push	{r0, r1, r2, r4, r5, r6, r7, lr}
    static uint32_t _x = 0, _y = 0;
    uint16_t xDiff, yDiff, x, y, xr, yr;

    TsState->TouchDetected = TsDrv->DetectTouch(TS_I2C_ADDRESS);
 800102a:	4d34      	ldr	r5, [pc, #208]	; (80010fc <_Z15BSP_TS_GetStateP15TS_StateTypeDef+0xd4>)
 800102c:	682b      	ldr	r3, [r5, #0]
{
 800102e:	4604      	mov	r4, r0
    TsState->TouchDetected = TsDrv->DetectTouch(TS_I2C_ADDRESS);
 8001030:	691b      	ldr	r3, [r3, #16]
 8001032:	2082      	movs	r0, #130	; 0x82
 8001034:	4798      	blx	r3
 8001036:	b280      	uxth	r0, r0
 8001038:	8020      	strh	r0, [r4, #0]

    if (TsState->TouchDetected)
 800103a:	2800      	cmp	r0, #0
 800103c:	d04c      	beq.n	80010d8 <_Z15BSP_TS_GetStateP15TS_StateTypeDef+0xb0>
    {
        TsDrv->GetXY(TS_I2C_ADDRESS, &x, &y);
 800103e:	682b      	ldr	r3, [r5, #0]
 8001040:	f10d 0206 	add.w	r2, sp, #6
 8001044:	695b      	ldr	r3, [r3, #20]
 8001046:	a901      	add	r1, sp, #4
 8001048:	2082      	movs	r0, #130	; 0x82
 800104a:	4798      	blx	r3

        //Ensures the coordinates is within the screen
        if (y > 3700)
 800104c:	f8bd 3006 	ldrh.w	r3, [sp, #6]
 8001050:	f640 6274 	movw	r2, #3700	; 0xe74
 8001054:	4293      	cmp	r3, r2
 8001056:	d941      	bls.n	80010dc <_Z15BSP_TS_GetStateP15TS_StateTypeDef+0xb4>
        {
            y = 3700;
 8001058:	f8ad 2006 	strh.w	r2, [sp, #6]

        /* Y value first correction */
        y -= 180;

        /* Y value second correction */
        y = 3520 - y;
 800105c:	f8bd 2006 	ldrh.w	r2, [sp, #6]
 8001060:	f5c2 6267 	rsb	r2, r2, #3696	; 0xe70
 8001064:	3204      	adds	r2, #4
 8001066:	b292      	uxth	r2, r2

        /* Y value third correction */
        yr = y / 11;

        /* Return y position value */
        if (yr <= 0)
 8001068:	2a0a      	cmp	r2, #10
 800106a:	d93d      	bls.n	80010e8 <_Z15BSP_TS_GetStateP15TS_StateTypeDef+0xc0>
        yr = y / 11;
 800106c:	230b      	movs	r3, #11
 800106e:	fbb2 f2f3 	udiv	r2, r2, r3
        {
            yr = 0;
        }
        else if (yr > TsYBoundary)
 8001072:	4b23      	ldr	r3, [pc, #140]	; (8001100 <_Z15BSP_TS_GetStateP15TS_StateTypeDef+0xd8>)
 8001074:	881b      	ldrh	r3, [r3, #0]
 8001076:	429a      	cmp	r2, r3
 8001078:	d901      	bls.n	800107e <_Z15BSP_TS_GetStateP15TS_StateTypeDef+0x56>
        {
            yr = TsYBoundary - 1;
 800107a:	3b01      	subs	r3, #1
 800107c:	b29a      	uxth	r2, r3
        {
        }
        y = yr;

        /* X value first correction */
        if (x <= 3000)
 800107e:	f8bd 3004 	ldrh.w	r3, [sp, #4]
 8001082:	f640 31b8 	movw	r1, #3000	; 0xbb8
 8001086:	428b      	cmp	r3, r1
 8001088:	d830      	bhi.n	80010ec <_Z15BSP_TS_GetStateP15TS_StateTypeDef+0xc4>
        {
            x = 3870 - x;
 800108a:	f5c3 6371 	rsb	r3, r3, #3856	; 0xf10
 800108e:	330e      	adds	r3, #14
 8001090:	b29b      	uxth	r3, r3
        {
            x = 3800 - x;
        }

        /* X value second correction */
        xr = x / 15;
 8001092:	210f      	movs	r1, #15
 8001094:	fbb3 f3f1 	udiv	r3, r3, r1
        /* Return X position value */
        if (xr <= 0)
        {
            xr = 0;
        }
        else if (xr > TsXBoundary)
 8001098:	491a      	ldr	r1, [pc, #104]	; (8001104 <_Z15BSP_TS_GetStateP15TS_StateTypeDef+0xdc>)
 800109a:	8809      	ldrh	r1, [r1, #0]
 800109c:	428b      	cmp	r3, r1
 800109e:	d901      	bls.n	80010a4 <_Z15BSP_TS_GetStateP15TS_StateTypeDef+0x7c>
        {
            xr = TsXBoundary - 1;
 80010a0:	1e4b      	subs	r3, r1, #1
 80010a2:	b29b      	uxth	r3, r3
        else
        {
        }

        x = xr;
        xDiff = x > _x ? (x - _x) : (_x - x);
 80010a4:	4e18      	ldr	r6, [pc, #96]	; (8001108 <_Z15BSP_TS_GetStateP15TS_StateTypeDef+0xe0>)
        yDiff = y > _y ? (y - _y) : (_y - y);
 80010a6:	4d19      	ldr	r5, [pc, #100]	; (800110c <_Z15BSP_TS_GetStateP15TS_StateTypeDef+0xe4>)
        xDiff = x > _x ? (x - _x) : (_x - x);
 80010a8:	6830      	ldr	r0, [r6, #0]
        yDiff = y > _y ? (y - _y) : (_y - y);
 80010aa:	682f      	ldr	r7, [r5, #0]
        xDiff = x > _x ? (x - _x) : (_x - x);
 80010ac:	4283      	cmp	r3, r0
 80010ae:	b281      	uxth	r1, r0
 80010b0:	bf8c      	ite	hi
 80010b2:	1a59      	subhi	r1, r3, r1
 80010b4:	1ac9      	subls	r1, r1, r3
        yDiff = y > _y ? (y - _y) : (_y - y);
 80010b6:	b2b8      	uxth	r0, r7
 80010b8:	42ba      	cmp	r2, r7
 80010ba:	bf8c      	ite	hi
 80010bc:	1a10      	subhi	r0, r2, r0
 80010be:	1a80      	subls	r0, r0, r2
        xDiff = x > _x ? (x - _x) : (_x - x);
 80010c0:	b289      	uxth	r1, r1
        yDiff = y > _y ? (y - _y) : (_y - y);
 80010c2:	b280      	uxth	r0, r0

        if (xDiff + yDiff > 5)
 80010c4:	4401      	add	r1, r0
 80010c6:	2905      	cmp	r1, #5
        {
            _x = x;
 80010c8:	bfc8      	it	gt
 80010ca:	6033      	strgt	r3, [r6, #0]
            _y = y;
        }

        /* Update the X position */
        TsState->X = _x;
 80010cc:	6833      	ldr	r3, [r6, #0]
            _y = y;
 80010ce:	bfc8      	it	gt
 80010d0:	602a      	strgt	r2, [r5, #0]
        TsState->X = _x;
 80010d2:	8063      	strh	r3, [r4, #2]

        /* Update the Y position */
        TsState->Y = _y;
 80010d4:	682b      	ldr	r3, [r5, #0]
 80010d6:	80a3      	strh	r3, [r4, #4]
    }
}
 80010d8:	b003      	add	sp, #12
 80010da:	bdf0      	pop	{r4, r5, r6, r7, pc}
        else if (y < 180)
 80010dc:	2bb3      	cmp	r3, #179	; 0xb3
            y = 180;
 80010de:	bf9c      	itt	ls
 80010e0:	23b4      	movls	r3, #180	; 0xb4
 80010e2:	f8ad 3006 	strhls.w	r3, [sp, #6]
 80010e6:	e7b9      	b.n	800105c <_Z15BSP_TS_GetStateP15TS_StateTypeDef+0x34>
            yr = 0;
 80010e8:	2200      	movs	r2, #0
 80010ea:	e7c8      	b.n	800107e <_Z15BSP_TS_GetStateP15TS_StateTypeDef+0x56>
            x = 3800 - x;
 80010ec:	f5c3 636d 	rsb	r3, r3, #3792	; 0xed0
 80010f0:	3308      	adds	r3, #8
 80010f2:	b29b      	uxth	r3, r3
        if (xr <= 0)
 80010f4:	2b0e      	cmp	r3, #14
 80010f6:	d8cc      	bhi.n	8001092 <_Z15BSP_TS_GetStateP15TS_StateTypeDef+0x6a>
            xr = 0;
 80010f8:	2300      	movs	r3, #0
 80010fa:	e7d3      	b.n	80010a4 <_Z15BSP_TS_GetStateP15TS_StateTypeDef+0x7c>
 80010fc:	200002f0 	.word	0x200002f0
 8001100:	200002ee 	.word	0x200002ee
 8001104:	200002ec 	.word	0x200002ec
 8001108:	200002f4 	.word	0x200002f4
 800110c:	200002f8 	.word	0x200002f8

08001110 <_ZN20STM32TouchController11sampleTouchERlS0_>:
{
 8001110:	b537      	push	{r0, r1, r2, r4, r5, lr}
    BSP_TS_GetState(&state);
 8001112:	4668      	mov	r0, sp
{
 8001114:	460d      	mov	r5, r1
 8001116:	4614      	mov	r4, r2
    BSP_TS_GetState(&state);
 8001118:	f7ff ff86 	bl	8001028 <_Z15BSP_TS_GetStateP15TS_StateTypeDef>
    if (state.TouchDetected)
 800111c:	f8bd 0000 	ldrh.w	r0, [sp]
 8001120:	b130      	cbz	r0, 8001130 <_ZN20STM32TouchController11sampleTouchERlS0_+0x20>
        x = state.X;
 8001122:	f8bd 3002 	ldrh.w	r3, [sp, #2]
 8001126:	602b      	str	r3, [r5, #0]
        y = state.Y;
 8001128:	f8bd 3004 	ldrh.w	r3, [sp, #4]
 800112c:	6023      	str	r3, [r4, #0]
        return true;
 800112e:	2001      	movs	r0, #1
}
 8001130:	b003      	add	sp, #12
 8001132:	bd30      	pop	{r4, r5, pc}

08001134 <_ZN8touchgfx4GPIO3setENS0_7GPIO_IDE>:
 * Sets a pin high.
 */
void GPIO::set(GPIO_ID id)
{

}
 8001134:	4770      	bx	lr

08001136 <_ZN8touchgfx4GPIO5clearENS0_7GPIO_IDE>:
 8001136:	4770      	bx	lr

08001138 <_ZN8touchgfx4GPIO6toggleENS0_7GPIO_IDE>:
 8001138:	4770      	bx	lr

0800113a <_ZN8touchgfx3HAL21setDisplayOrientationENS_18DisplayOrientationE>:
     * @note A screen transition must occur before this takes effect!
     */
    virtual void setDisplayOrientation(DisplayOrientation orientation)
    {
        requestedOrientation = orientation;
        displayOrientationChangeRequested = true;
 800113a:	2301      	movs	r3, #1
        requestedOrientation = orientation;
 800113c:	f880 1074 	strb.w	r1, [r0, #116]	; 0x74
        displayOrientationChangeRequested = true;
 8001140:	f880 3075 	strb.w	r3, [r0, #117]	; 0x75
    }
 8001144:	4770      	bx	lr

08001146 <_ZN8touchgfx3HAL9sampleKeyERh>:
     * @return True if a keypress was detected and the "key" parameter is set to a value.
     */
    virtual bool sampleKey(uint8_t& key)
    {
        return false;
    }
 8001146:	2000      	movs	r0, #0
 8001148:	4770      	bx	lr

0800114a <_ZNK8touchgfx3HAL18getFlashDataReaderEv>:
     * @return the FlashDataReader.
     */
    virtual FlashDataReader* getFlashDataReader() const
    {
        return 0;
    }
 800114a:	2000      	movs	r0, #0
 800114c:	4770      	bx	lr

0800114e <_ZN8touchgfx3HAL9taskDelayEt>:
     *
     * @see registerTaskDelayFunction
     */
    virtual void taskDelay(uint16_t ms)
    {
        if (taskDelayFunc)
 800114e:	6b83      	ldr	r3, [r0, #56]	; 0x38
 8001150:	b10b      	cbz	r3, 8001156 <_ZN8touchgfx3HAL9taskDelayEt+0x8>
        {
            taskDelayFunc(ms);
 8001152:	4608      	mov	r0, r1
 8001154:	4718      	bx	r3
        }
    }
 8001156:	4770      	bx	lr

08001158 <_ZN8touchgfx3HAL17getTFTCurrentLineEv>:
     *         implemented".
     */
    virtual uint16_t getTFTCurrentLine()
    {
        return 0xFFFFu;
    }
 8001158:	f64f 70ff 	movw	r0, #65535	; 0xffff
 800115c:	4770      	bx	lr

0800115e <_ZN8touchgfx3HAL10getDMATypeEv>:
     *
     * @return a DMAType value of the concrete DMA implementation.
     */
    virtual DMAType getDMAType()
    {
        return dma.getDMAType();
 800115e:	6840      	ldr	r0, [r0, #4]
 8001160:	6803      	ldr	r3, [r0, #0]
 8001162:	699b      	ldr	r3, [r3, #24]
 8001164:	4718      	bx	r3

08001166 <_ZN8touchgfx3HAL15InvalidateCacheEv>:
     * Called by setRenderingMethod when changing rendering method
     * from Hardware to Software indicating the cache should be invalidated.
     */
    virtual void InvalidateCache()
    {
    }
 8001166:	4770      	bx	lr

08001168 <_ZN8touchgfx3HAL10FlushCacheEv>:
     * Called by setRenderingMethod when changing rendering method
     * from Software to Hardware indicating the cache should be invalidated.
     */
    virtual void FlushCache()
    {
    }
 8001168:	4770      	bx	lr

0800116a <_ZN11TouchGFXHALD1Ev>:
 *
 * @brief HAL implementation for TouchGFX.
 *
 * @sa HAL
 */
class TouchGFXHAL : public TouchGFXGeneratedHAL
 800116a:	4770      	bx	lr

0800116c <_ZN11TouchGFXHAL10initializeEv>:
using namespace touchgfx;

uint32_t animationStorage[(240 * 320 * 2 + 3) / 4] LOCATION_ATTRIBUTE("TouchGFX_Framebuffer");

void TouchGFXHAL::initialize()
{
 800116c:	b570      	push	{r4, r5, r6, lr}
 800116e:	4604      	mov	r4, r0
    //
    // To overwrite the generated implementation, omit call to parent function
    // and implemented needed functionality here.
    // Please note, HAL::initialize() must be called to initialize the framework.

    TouchGFXGeneratedHAL::initialize();
 8001170:	f000 fc5a 	bl	8001a28 <_ZN20TouchGFXGeneratedHAL10initializeEv>
    setFrameBufferStartAddresses((void*)frameBuffer0, (void*)frameBuffer1, (void*)animationStorage);
 8001174:	6823      	ldr	r3, [r4, #0]
 8001176:	f8d3 5080 	ldr.w	r5, [r3, #128]	; 0x80
 800117a:	4b04      	ldr	r3, [pc, #16]	; (800118c <_ZN11TouchGFXHAL10initializeEv+0x20>)
 800117c:	e9d4 120f 	ldrd	r1, r2, [r4, #60]	; 0x3c
 8001180:	4620      	mov	r0, r4
 8001182:	46ac      	mov	ip, r5
}
 8001184:	e8bd 4070 	ldmia.w	sp!, {r4, r5, r6, lr}
    setFrameBufferStartAddresses((void*)frameBuffer0, (void*)frameBuffer1, (void*)animationStorage);
 8001188:	4760      	bx	ip
 800118a:	bf00      	nop
 800118c:	d0000000 	.word	0xd0000000

08001190 <_ZN11TouchGFXHAL9taskEntryEv>:

void TouchGFXHAL::taskEntry()
{
 8001190:	b508      	push	{r3, lr}
    enableLCDControllerInterrupt();
 8001192:	6803      	ldr	r3, [r0, #0]
{
 8001194:	4604      	mov	r4, r0
    enableLCDControllerInterrupt();
 8001196:	6f9b      	ldr	r3, [r3, #120]	; 0x78
 8001198:	4798      	blx	r3
    enableInterrupts();
 800119a:	6823      	ldr	r3, [r4, #0]
 800119c:	4620      	mov	r0, r4
 800119e:	6f1b      	ldr	r3, [r3, #112]	; 0x70
 80011a0:	4798      	blx	r3

    OSWrappers::waitForVSync();
 80011a2:	f000 f8d7 	bl	8001354 <_ZN8touchgfx10OSWrappers12waitForVSyncEv>
    backPorchExited();
 80011a6:	6823      	ldr	r3, [r4, #0]
 80011a8:	4620      	mov	r0, r4
 80011aa:	6e9b      	ldr	r3, [r3, #104]	; 0x68
 80011ac:	4798      	blx	r3

    LCD_IO_WriteReg(0x29);
 80011ae:	2029      	movs	r0, #41	; 0x29
 80011b0:	f001 fa2c 	bl	800260c <LCD_IO_WriteReg>

    for (;;)
    {
        OSWrappers::waitForVSync();
 80011b4:	f000 f8ce 	bl	8001354 <_ZN8touchgfx10OSWrappers12waitForVSyncEv>
        backPorchExited();
 80011b8:	6823      	ldr	r3, [r4, #0]
 80011ba:	4620      	mov	r0, r4
 80011bc:	6e9b      	ldr	r3, [r3, #104]	; 0x68
 80011be:	4798      	blx	r3
    for (;;)
 80011c0:	e7f8      	b.n	80011b4 <_ZN11TouchGFXHAL9taskEntryEv+0x24>

080011c2 <_ZN8touchgfx3HAL15backPorchExitedEv>:
    virtual void backPorchExited()
 80011c2:	b510      	push	{r4, lr}
 80011c4:	4604      	mov	r4, r0
        swapFrameBuffers();
 80011c6:	f008 ffeb 	bl	800a1a0 <_ZN8touchgfx3HAL16swapFrameBuffersEv>
        tick();
 80011ca:	6823      	ldr	r3, [r4, #0]
 80011cc:	4620      	mov	r0, r4
 80011ce:	f8d3 30a0 	ldr.w	r3, [r3, #160]	; 0xa0
    }
 80011d2:	e8bd 4010 	ldmia.w	sp!, {r4, lr}
        tick();
 80011d6:	4718      	bx	r3

080011d8 <_ZNK11TouchGFXHAL17getTFTFrameBufferEv>:
    // Calling parent implementation of getTFTFrameBuffer().
    //
    // To overwrite the generated implementation, omit call to parent function
    // and implemented needed functionality here.

    return TouchGFXGeneratedHAL::getTFTFrameBuffer();
 80011d8:	f000 bc18 	b.w	8001a0c <_ZNK20TouchGFXGeneratedHAL17getTFTFrameBufferEv>

080011dc <_ZN11TouchGFXHAL17setTFTFrameBufferEPt>:
    // Calling parent implementation of setTFTFrameBuffer(uint16_t* address).
    //
    // To overwrite the generated implementation, omit call to parent function
    // and implemented needed functionality here.

    TouchGFXGeneratedHAL::setTFTFrameBuffer(address);
 80011dc:	f000 bc1c 	b.w	8001a18 <_ZN20TouchGFXGeneratedHAL17setTFTFrameBufferEPt>

080011e0 <_ZN11TouchGFXHAL16flushFrameBufferERKN8touchgfx4RectE>:
    // To overwrite the generated implementation, omit call to parent function
    // and implemented needed functionality here.
    // Please note, HAL::flushFrameBuffer(const touchgfx::Rect& rect) must
    // be called to notify the touchgfx framework that flush has been performed.

    TouchGFXGeneratedHAL::flushFrameBuffer(rect);
 80011e0:	f000 bc40 	b.w	8001a64 <_ZN20TouchGFXGeneratedHAL16flushFrameBufferERKN8touchgfx4RectE>

080011e4 <_ZN11TouchGFXHAL19configureInterruptsEv>:
    // Calling parent implementation of configureInterrupts().
    //
    // To overwrite the generated implementation, omit call to parent function
    // and implemented needed functionality here.

    TouchGFXGeneratedHAL::configureInterrupts();
 80011e4:	f000 bbee 	b.w	80019c4 <_ZN20TouchGFXGeneratedHAL19configureInterruptsEv>

080011e8 <_ZN11TouchGFXHAL16enableInterruptsEv>:
    // Calling parent implementation of enableInterrupts().
    //
    // To overwrite the generated implementation, omit call to parent function
    // and implemented needed functionality here.

    TouchGFXGeneratedHAL::enableInterrupts();
 80011e8:	f000 bc40 	b.w	8001a6c <_ZN20TouchGFXGeneratedHAL16enableInterruptsEv>

080011ec <_ZN11TouchGFXHAL17disableInterruptsEv>:
    // Calling parent implementation of disableInterrupts().
    //
    // To overwrite the generated implementation, omit call to parent function
    // and implemented needed functionality here.

    TouchGFXGeneratedHAL::disableInterrupts();
 80011ec:	f000 bc48 	b.w	8001a80 <_ZN20TouchGFXGeneratedHAL17disableInterruptsEv>

080011f0 <_ZN11TouchGFXHAL28enableLCDControllerInterruptEv>:
    // Calling parent implementation of enableLCDControllerInterrupt().
    //
    // To overwrite the generated implementation, omit call to parent function
    // and implemented needed functionality here.

    TouchGFXGeneratedHAL::enableLCDControllerInterrupt();
 80011f0:	f000 bbf2 	b.w	80019d8 <_ZN20TouchGFXGeneratedHAL28enableLCDControllerInterruptEv>

080011f4 <_ZN11TouchGFXHAL16flushFrameBufferEv>:
     * Rect version.
     * @see HAL::flushFrameBuffer
     */
    virtual void flushFrameBuffer()
    {
        HAL::flushFrameBuffer();
 80011f4:	f008 b98c 	b.w	8009510 <_ZN8touchgfx3HAL16flushFrameBufferEv>

080011f8 <_ZN11TouchGFXHALD0Ev>:
 80011f8:	b510      	push	{r4, lr}
 80011fa:	217c      	movs	r1, #124	; 0x7c
 80011fc:	4604      	mov	r4, r0
 80011fe:	f01a fbe4 	bl	801b9ca <_ZdlPvj>
 8001202:	4620      	mov	r0, r4
 8001204:	bd10      	pop	{r4, pc}

08001206 <_ZN8touchgfx3HAL11getBlitCapsEv>:
        if (useDMAAcceleration)
 8001206:	f890 3077 	ldrb.w	r3, [r0, #119]	; 0x77
 800120a:	b11b      	cbz	r3, 8001214 <_ZN8touchgfx3HAL11getBlitCapsEv+0xe>
            return dma.getBlitCaps();
 800120c:	6840      	ldr	r0, [r0, #4]
 800120e:	6803      	ldr	r3, [r0, #0]
 8001210:	681b      	ldr	r3, [r3, #0]
 8001212:	4718      	bx	r3
    }
 8001214:	4618      	mov	r0, r3
 8001216:	4770      	bx	lr

08001218 <_ZN8touchgfx3HAL31performDisplayOrientationChangeEv>:
    virtual void performDisplayOrientationChange()
 8001218:	b530      	push	{r4, r5, lr}
        if (requestedOrientation != nativeDisplayOrientation)
 800121a:	f890 1034 	ldrb.w	r1, [r0, #52]	; 0x34
 800121e:	f890 4074 	ldrb.w	r4, [r0, #116]	; 0x74
            if (DISPLAY_ROTATION == rotate0)
 8001222:	4b10      	ldr	r3, [pc, #64]	; (8001264 <_ZN8touchgfx3HAL31performDisplayOrientationChangeEv+0x4c>)
        if (requestedOrientation != nativeDisplayOrientation)
 8001224:	428c      	cmp	r4, r1
            if (DISPLAY_ROTATION == rotate0)
 8001226:	781a      	ldrb	r2, [r3, #0]
        if (requestedOrientation != nativeDisplayOrientation)
 8001228:	d00d      	beq.n	8001246 <_ZN8touchgfx3HAL31performDisplayOrientationChangeEv+0x2e>
            if (DISPLAY_ROTATION == rotate0)
 800122a:	b95a      	cbnz	r2, 8001244 <_ZN8touchgfx3HAL31performDisplayOrientationChangeEv+0x2c>
                FRAME_BUFFER_WIDTH = DISPLAY_WIDTH;
 800122c:	4a0e      	ldr	r2, [pc, #56]	; (8001268 <_ZN8touchgfx3HAL31performDisplayOrientationChangeEv+0x50>)
 800122e:	490f      	ldr	r1, [pc, #60]	; (800126c <_ZN8touchgfx3HAL31performDisplayOrientationChangeEv+0x54>)
                FRAME_BUFFER_HEIGHT = DISPLAY_HEIGHT;
 8001230:	480f      	ldr	r0, [pc, #60]	; (8001270 <_ZN8touchgfx3HAL31performDisplayOrientationChangeEv+0x58>)
                FRAME_BUFFER_WIDTH = DISPLAY_WIDTH;
 8001232:	8814      	ldrh	r4, [r2, #0]
                FRAME_BUFFER_HEIGHT = DISPLAY_HEIGHT;
 8001234:	4d0f      	ldr	r5, [pc, #60]	; (8001274 <_ZN8touchgfx3HAL31performDisplayOrientationChangeEv+0x5c>)
                FRAME_BUFFER_WIDTH = DISPLAY_WIDTH;
 8001236:	800c      	strh	r4, [r1, #0]
                FRAME_BUFFER_HEIGHT = DISPLAY_HEIGHT;
 8001238:	8801      	ldrh	r1, [r0, #0]
                DISPLAY_WIDTH = FRAME_BUFFER_HEIGHT;
 800123a:	8011      	strh	r1, [r2, #0]
                FRAME_BUFFER_HEIGHT = DISPLAY_HEIGHT;
 800123c:	8029      	strh	r1, [r5, #0]
                DISPLAY_HEIGHT = FRAME_BUFFER_WIDTH;
 800123e:	8004      	strh	r4, [r0, #0]
                DISPLAY_ROTATION = rotate90;
 8001240:	2201      	movs	r2, #1
            DISPLAY_ROTATION = rotate0;
 8001242:	701a      	strb	r2, [r3, #0]
    }
 8001244:	bd30      	pop	{r4, r5, pc}
        else if (DISPLAY_ROTATION != rotate0)
 8001246:	2a00      	cmp	r2, #0
 8001248:	d0fc      	beq.n	8001244 <_ZN8touchgfx3HAL31performDisplayOrientationChangeEv+0x2c>
            FRAME_BUFFER_WIDTH = DISPLAY_HEIGHT;
 800124a:	4809      	ldr	r0, [pc, #36]	; (8001270 <_ZN8touchgfx3HAL31performDisplayOrientationChangeEv+0x58>)
 800124c:	4a07      	ldr	r2, [pc, #28]	; (800126c <_ZN8touchgfx3HAL31performDisplayOrientationChangeEv+0x54>)
 800124e:	8801      	ldrh	r1, [r0, #0]
 8001250:	8011      	strh	r1, [r2, #0]
            FRAME_BUFFER_HEIGHT = DISPLAY_WIDTH;
 8001252:	4a05      	ldr	r2, [pc, #20]	; (8001268 <_ZN8touchgfx3HAL31performDisplayOrientationChangeEv+0x50>)
 8001254:	4d07      	ldr	r5, [pc, #28]	; (8001274 <_ZN8touchgfx3HAL31performDisplayOrientationChangeEv+0x5c>)
 8001256:	8814      	ldrh	r4, [r2, #0]
 8001258:	802c      	strh	r4, [r5, #0]
            DISPLAY_WIDTH = FRAME_BUFFER_WIDTH;
 800125a:	8011      	strh	r1, [r2, #0]
            DISPLAY_HEIGHT = FRAME_BUFFER_HEIGHT;
 800125c:	8004      	strh	r4, [r0, #0]
            DISPLAY_ROTATION = rotate0;
 800125e:	2200      	movs	r2, #0
 8001260:	e7ef      	b.n	8001242 <_ZN8touchgfx3HAL31performDisplayOrientationChangeEv+0x2a>
 8001262:	bf00      	nop
 8001264:	20012628 	.word	0x20012628
 8001268:	20012624 	.word	0x20012624
 800126c:	2001262a 	.word	0x2001262a
 8001270:	20012626 	.word	0x20012626
 8001274:	2001262c 	.word	0x2001262c

08001278 <_ZN8touchgfx3HAL28setFrameBufferStartAddressesEPvS1_S1_>:
    virtual void setFrameBufferStartAddresses(void* frameBuffer, void* doubleBuffer, void* animationStorage)
 8001278:	b508      	push	{r3, lr}
        assert(frameBuffer != 0 && "A framebuffer address must be set");
 800127a:	b931      	cbnz	r1, 800128a <_ZN8touchgfx3HAL28setFrameBufferStartAddressesEPvS1_S1_+0x12>
 800127c:	4b0a      	ldr	r3, [pc, #40]	; (80012a8 <_ZN8touchgfx3HAL28setFrameBufferStartAddressesEPvS1_S1_+0x30>)
 800127e:	4a0b      	ldr	r2, [pc, #44]	; (80012ac <_ZN8touchgfx3HAL28setFrameBufferStartAddressesEPvS1_S1_+0x34>)
 8001280:	480b      	ldr	r0, [pc, #44]	; (80012b0 <_ZN8touchgfx3HAL28setFrameBufferStartAddressesEPvS1_S1_+0x38>)
 8001282:	f44f 7125 	mov.w	r1, #660	; 0x294
 8001286:	f01a fbcf 	bl	801ba28 <__assert_func>
        frameBuffer1 = reinterpret_cast<uint16_t*>(doubleBuffer);
 800128a:	e9c0 120f 	strd	r1, r2, [r0, #60]	; 0x3c
        USE_DOUBLE_BUFFERING = doubleBuffer != 0;
 800128e:	3a00      	subs	r2, #0
 8001290:	4908      	ldr	r1, [pc, #32]	; (80012b4 <_ZN8touchgfx3HAL28setFrameBufferStartAddressesEPvS1_S1_+0x3c>)
        frameBuffer2 = reinterpret_cast<uint16_t*>(animationStorage);
 8001292:	6443      	str	r3, [r0, #68]	; 0x44
        USE_DOUBLE_BUFFERING = doubleBuffer != 0;
 8001294:	bf18      	it	ne
 8001296:	2201      	movne	r2, #1
 8001298:	700a      	strb	r2, [r1, #0]
        USE_ANIMATION_STORAGE = animationStorage != 0;
 800129a:	3b00      	subs	r3, #0
 800129c:	4a06      	ldr	r2, [pc, #24]	; (80012b8 <_ZN8touchgfx3HAL28setFrameBufferStartAddressesEPvS1_S1_+0x40>)
 800129e:	bf18      	it	ne
 80012a0:	2301      	movne	r3, #1
 80012a2:	7013      	strb	r3, [r2, #0]
    }
 80012a4:	bd08      	pop	{r3, pc}
 80012a6:	bf00      	nop
 80012a8:	0801e648 	.word	0x0801e648
 80012ac:	0801e680 	.word	0x0801e680
 80012b0:	0801e6ce 	.word	0x0801e6ce
 80012b4:	2001262e 	.word	0x2001262e
 80012b8:	2001262f 	.word	0x2001262f

080012bc <_ZN8touchgfx10OSWrappers10initializeEv>:
 * Initialize frame buffer semaphore and queue/mutex for VSYNC signal.
 */
void OSWrappers::initialize()
{
    // Create a queue of length 1
    frame_buffer_sem = osSemaphoreNew(1, 1, NULL); // Binary semaphore
 80012bc:	2101      	movs	r1, #1
{
 80012be:	b508      	push	{r3, lr}
    frame_buffer_sem = osSemaphoreNew(1, 1, NULL); // Binary semaphore
 80012c0:	2200      	movs	r2, #0
 80012c2:	4608      	mov	r0, r1
 80012c4:	f005 fe54 	bl	8006f70 <osSemaphoreNew>
 80012c8:	4b0a      	ldr	r3, [pc, #40]	; (80012f4 <_ZN8touchgfx10OSWrappers10initializeEv+0x38>)
 80012ca:	6018      	str	r0, [r3, #0]
    assert((frame_buffer_sem != NULL) && "Creation of framebuffer semaphore failed");
 80012cc:	b928      	cbnz	r0, 80012da <_ZN8touchgfx10OSWrappers10initializeEv+0x1e>
 80012ce:	4b0a      	ldr	r3, [pc, #40]	; (80012f8 <_ZN8touchgfx10OSWrappers10initializeEv+0x3c>)
 80012d0:	4a0a      	ldr	r2, [pc, #40]	; (80012fc <_ZN8touchgfx10OSWrappers10initializeEv+0x40>)
 80012d2:	2127      	movs	r1, #39	; 0x27

    // Create a queue of length 1
    vsync_queue = osMessageQueueNew(1, 4, NULL);
    assert((vsync_queue != NULL) && "Creation of vsync message queue failed");
 80012d4:	480a      	ldr	r0, [pc, #40]	; (8001300 <_ZN8touchgfx10OSWrappers10initializeEv+0x44>)
 80012d6:	f01a fba7 	bl	801ba28 <__assert_func>
    vsync_queue = osMessageQueueNew(1, 4, NULL);
 80012da:	2200      	movs	r2, #0
 80012dc:	2104      	movs	r1, #4
 80012de:	2001      	movs	r0, #1
 80012e0:	f005 fee3 	bl	80070aa <osMessageQueueNew>
 80012e4:	4b07      	ldr	r3, [pc, #28]	; (8001304 <_ZN8touchgfx10OSWrappers10initializeEv+0x48>)
 80012e6:	6018      	str	r0, [r3, #0]
    assert((vsync_queue != NULL) && "Creation of vsync message queue failed");
 80012e8:	b918      	cbnz	r0, 80012f2 <_ZN8touchgfx10OSWrappers10initializeEv+0x36>
 80012ea:	4b07      	ldr	r3, [pc, #28]	; (8001308 <_ZN8touchgfx10OSWrappers10initializeEv+0x4c>)
 80012ec:	4a03      	ldr	r2, [pc, #12]	; (80012fc <_ZN8touchgfx10OSWrappers10initializeEv+0x40>)
 80012ee:	212b      	movs	r1, #43	; 0x2b
 80012f0:	e7f0      	b.n	80012d4 <_ZN8touchgfx10OSWrappers10initializeEv+0x18>
}
 80012f2:	bd08      	pop	{r3, pc}
 80012f4:	20000300 	.word	0x20000300
 80012f8:	0801e7e0 	.word	0x0801e7e0
 80012fc:	0801e829 	.word	0x0801e829
 8001300:	0801e858 	.word	0x0801e858
 8001304:	200002fc 	.word	0x200002fc
 8001308:	0801e8a8 	.word	0x0801e8a8

0800130c <_ZN8touchgfx10OSWrappers24takeFrameBufferSemaphoreEv>:
/*
 * Take the frame buffer semaphore. Blocks until semaphore is available.
 */
void OSWrappers::takeFrameBufferSemaphore()
{
    osSemaphoreAcquire(frame_buffer_sem, osWaitForever);
 800130c:	4b02      	ldr	r3, [pc, #8]	; (8001318 <_ZN8touchgfx10OSWrappers24takeFrameBufferSemaphoreEv+0xc>)
 800130e:	f04f 31ff 	mov.w	r1, #4294967295
 8001312:	6818      	ldr	r0, [r3, #0]
 8001314:	f005 be76 	b.w	8007004 <osSemaphoreAcquire>
 8001318:	20000300 	.word	0x20000300

0800131c <_ZN8touchgfx10OSWrappers24giveFrameBufferSemaphoreEv>:
/*
 * Release the frame buffer semaphore.
 */
void OSWrappers::giveFrameBufferSemaphore()
{
    osSemaphoreRelease(frame_buffer_sem);
 800131c:	4b01      	ldr	r3, [pc, #4]	; (8001324 <_ZN8touchgfx10OSWrappers24giveFrameBufferSemaphoreEv+0x8>)
 800131e:	6818      	ldr	r0, [r3, #0]
 8001320:	f005 be9b 	b.w	800705a <osSemaphoreRelease>
 8001324:	20000300 	.word	0x20000300

08001328 <_ZN8touchgfx10OSWrappers27tryTakeFrameBufferSemaphoreEv>:
 * Note must return immediately! This function does not care who has the taken the semaphore,
 * it only serves to make sure that the semaphore is taken by someone.
 */
void OSWrappers::tryTakeFrameBufferSemaphore()
{
    osSemaphoreAcquire(frame_buffer_sem, 0);
 8001328:	4b02      	ldr	r3, [pc, #8]	; (8001334 <_ZN8touchgfx10OSWrappers27tryTakeFrameBufferSemaphoreEv+0xc>)
 800132a:	2100      	movs	r1, #0
 800132c:	6818      	ldr	r0, [r3, #0]
 800132e:	f005 be69 	b.w	8007004 <osSemaphoreAcquire>
 8001332:	bf00      	nop
 8001334:	20000300 	.word	0x20000300

08001338 <_ZN8touchgfx10OSWrappers31giveFrameBufferSemaphoreFromISREv>:
 8001338:	f7ff bff0 	b.w	800131c <_ZN8touchgfx10OSWrappers24giveFrameBufferSemaphoreEv>

0800133c <_ZN8touchgfx10OSWrappers11signalVSyncEv>:
 * Note This function is called from an ISR, and should (depending on OS) trigger a
 * scheduling.
 */
void OSWrappers::signalVSync()
{
    osMessageQueuePut(vsync_queue, &dummy, 0, 0);
 800133c:	4803      	ldr	r0, [pc, #12]	; (800134c <_ZN8touchgfx10OSWrappers11signalVSyncEv+0x10>)
 800133e:	4904      	ldr	r1, [pc, #16]	; (8001350 <_ZN8touchgfx10OSWrappers11signalVSyncEv+0x14>)
 8001340:	6800      	ldr	r0, [r0, #0]
 8001342:	2300      	movs	r3, #0
 8001344:	461a      	mov	r2, r3
 8001346:	f005 beeb 	b.w	8007120 <osMessageQueuePut>
 800134a:	bf00      	nop
 800134c:	200002fc 	.word	0x200002fc
 8001350:	20000004 	.word	0x20000004

08001354 <_ZN8touchgfx10OSWrappers12waitForVSyncEv>:
 *
 * Note This function must first clear the mutex/queue and then wait for the next one to
 * occur.
 */
void OSWrappers::waitForVSync()
{
 8001354:	b513      	push	{r0, r1, r4, lr}
    uint32_t dummyGet;
    // First make sure the queue is empty, by trying to remove an element with 0 timeout.
    osMessageQueueGet(vsync_queue, &dummyGet, 0, 0);
 8001356:	4c08      	ldr	r4, [pc, #32]	; (8001378 <_ZN8touchgfx10OSWrappers12waitForVSyncEv+0x24>)
 8001358:	2300      	movs	r3, #0
 800135a:	461a      	mov	r2, r3
 800135c:	a901      	add	r1, sp, #4
 800135e:	6820      	ldr	r0, [r4, #0]
 8001360:	f005 ff0e 	bl	8007180 <osMessageQueueGet>

    // Then, wait for next VSYNC to occur.
    osMessageQueueGet(vsync_queue, &dummyGet, 0, osWaitForever);
 8001364:	6820      	ldr	r0, [r4, #0]
 8001366:	f04f 33ff 	mov.w	r3, #4294967295
 800136a:	2200      	movs	r2, #0
 800136c:	a901      	add	r1, sp, #4
 800136e:	f005 ff07 	bl	8007180 <osMessageQueueGet>
}
 8001372:	b002      	add	sp, #8
 8001374:	bd10      	pop	{r4, pc}
 8001376:	bf00      	nop
 8001378:	200002fc 	.word	0x200002fc

0800137c <_ZN8touchgfx10OSWrappers9taskYieldEv>:
 * running without an operating system, the implementation can run
 * a very short task and return.
 */
void OSWrappers::taskYield()
{
    osThreadYield();
 800137c:	f005 bddb 	b.w	8006f36 <osThreadYield>

08001380 <_ZN8touchgfx13DMA_Interface5flushEv>:
    virtual void addToQueue(const BlitOp& op);

    /** This function blocks until all DMA transfers in the queue have been completed. */
    virtual void flush()
    {
        waitForFrameBufferSemaphore();
 8001380:	6803      	ldr	r3, [r0, #0]
 8001382:	6c5b      	ldr	r3, [r3, #68]	; 0x44
 8001384:	4718      	bx	r3

08001386 <_ZN10STM32F4DMA10getDMATypeEv>:
     * @return a DMAType value of the concrete DMA_Interface implementation.
     */
    virtual touchgfx::DMAType getDMAType(void)
    {
        return touchgfx::DMA_TYPE_CHROMART;
    }
 8001386:	2001      	movs	r0, #1
 8001388:	4770      	bx	lr

0800138a <_ZN10STM32F4DMA18signalDMAInterruptEv>:
     *
     *        Raises a DMA interrupt signal.
     */
    virtual void signalDMAInterrupt()
    {
        executeCompleted();
 800138a:	6803      	ldr	r3, [r0, #0]
 800138c:	6a9b      	ldr	r3, [r3, #40]	; 0x28
 800138e:	4718      	bx	r3

08001390 <_ZN10STM32F4DMA10initializeEv>:
    /* Disable DMA2D global Interrupt */
    NVIC_DisableIRQ(DMA2D_IRQn);
}

void STM32F4DMA::initialize()
{
 8001390:	b082      	sub	sp, #8
    /* Ensure DMA2D Clock is enabled */
    __HAL_RCC_DMA2D_CLK_ENABLE();
 8001392:	2300      	movs	r3, #0
 8001394:	9301      	str	r3, [sp, #4]
 8001396:	4b0d      	ldr	r3, [pc, #52]	; (80013cc <_ZN10STM32F4DMA10initializeEv+0x3c>)
 8001398:	6b1a      	ldr	r2, [r3, #48]	; 0x30
 800139a:	f442 0200 	orr.w	r2, r2, #8388608	; 0x800000
 800139e:	631a      	str	r2, [r3, #48]	; 0x30
 80013a0:	6b1a      	ldr	r2, [r3, #48]	; 0x30
 80013a2:	f402 0200 	and.w	r2, r2, #8388608	; 0x800000
 80013a6:	9201      	str	r2, [sp, #4]
 80013a8:	9a01      	ldr	r2, [sp, #4]
    __HAL_RCC_DMA2D_FORCE_RESET();
 80013aa:	691a      	ldr	r2, [r3, #16]
 80013ac:	f442 0200 	orr.w	r2, r2, #8388608	; 0x800000
 80013b0:	611a      	str	r2, [r3, #16]
    __HAL_RCC_DMA2D_RELEASE_RESET();
 80013b2:	691a      	ldr	r2, [r3, #16]
 80013b4:	f422 0200 	bic.w	r2, r2, #8388608	; 0x800000
 80013b8:	611a      	str	r2, [r3, #16]

    /* Add transfer complete callback function */
    hdma2d.XferCpltCallback = DMA2D_XferCpltCallback;
 80013ba:	4b05      	ldr	r3, [pc, #20]	; (80013d0 <_ZN10STM32F4DMA10initializeEv+0x40>)
 80013bc:	4a05      	ldr	r2, [pc, #20]	; (80013d4 <_ZN10STM32F4DMA10initializeEv+0x44>)
 80013be:	611a      	str	r2, [r3, #16]
 */
__STATIC_INLINE void __NVIC_EnableIRQ(IRQn_Type IRQn)
{
  if ((int32_t)(IRQn) >= 0)
  {
    NVIC->ISER[(((uint32_t)IRQn) >> 5UL)] = (uint32_t)(1UL << (((uint32_t)IRQn) & 0x1FUL));
 80013c0:	4b05      	ldr	r3, [pc, #20]	; (80013d8 <_ZN10STM32F4DMA10initializeEv+0x48>)
 80013c2:	f04f 6280 	mov.w	r2, #67108864	; 0x4000000
 80013c6:	609a      	str	r2, [r3, #8]

    /* Enable DMA2D global Interrupt */
    NVIC_EnableIRQ(DMA2D_IRQn);
}
 80013c8:	b002      	add	sp, #8
 80013ca:	4770      	bx	lr
 80013cc:	40023800 	.word	0x40023800
 80013d0:	200013c4 	.word	0x200013c4
 80013d4:	0800141d 	.word	0x0800141d
 80013d8:	e000e100 	.word	0xe000e100

080013dc <_ZN10STM32F4DMA11getBlitCapsEv>:
                                       | BLIT_OP_COPY_WITH_ALPHA
                                       | BLIT_OP_COPY_ARGB8888
                                       | BLIT_OP_COPY_ARGB8888_WITH_ALPHA
                                       | BLIT_OP_COPY_A4
                                       | BLIT_OP_COPY_A8);
}
 80013dc:	f240 30ef 	movw	r0, #1007	; 0x3ef
 80013e0:	4770      	bx	lr
	...

080013e4 <_ZN10STM32F4DMAD1Ev>:
STM32F4DMA::~STM32F4DMA()
 80013e4:	4b05      	ldr	r3, [pc, #20]	; (80013fc <_ZN10STM32F4DMAD1Ev+0x18>)
 80013e6:	6003      	str	r3, [r0, #0]
 */
__STATIC_INLINE void __NVIC_DisableIRQ(IRQn_Type IRQn)
{
  if ((int32_t)(IRQn) >= 0)
  {
    NVIC->ICER[(((uint32_t)IRQn) >> 5UL)] = (uint32_t)(1UL << (((uint32_t)IRQn) & 0x1FUL));
 80013e8:	4b05      	ldr	r3, [pc, #20]	; (8001400 <_ZN10STM32F4DMAD1Ev+0x1c>)
 80013ea:	f04f 6280 	mov.w	r2, #67108864	; 0x4000000
 80013ee:	f8c3 2088 	str.w	r2, [r3, #136]	; 0x88
  \details Acts as a special kind of Data Memory Barrier.
           It completes when all explicit memory accesses before this instruction complete.
 */
__STATIC_FORCEINLINE void __DSB(void)
{
  __ASM volatile ("dsb 0xF":::"memory");
 80013f2:	f3bf 8f4f 	dsb	sy
  __ASM volatile ("isb 0xF":::"memory");
 80013f6:	f3bf 8f6f 	isb	sy
}
 80013fa:	4770      	bx	lr
 80013fc:	0801ea50 	.word	0x0801ea50
 8001400:	e000e100 	.word	0xe000e100

08001404 <_ZN10STM32F4DMAD0Ev>:
STM32F4DMA::~STM32F4DMA()
 8001404:	b510      	push	{r4, lr}
 8001406:	4604      	mov	r4, r0
}
 8001408:	f44f 6142 	mov.w	r1, #3104	; 0xc20
 800140c:	f7ff ffea 	bl	80013e4 <_ZN10STM32F4DMAD1Ev>
 8001410:	4620      	mov	r0, r4
 8001412:	f01a fada 	bl	801b9ca <_ZdlPvj>
 8001416:	4620      	mov	r0, r4
 8001418:	bd10      	pop	{r4, pc}
	...

0800141c <DMA2D_XferCpltCallback>:
        return instance;
 800141c:	4b02      	ldr	r3, [pc, #8]	; (8001428 <DMA2D_XferCpltCallback+0xc>)
 800141e:	681b      	ldr	r3, [r3, #0]
 8001420:	6858      	ldr	r0, [r3, #4]
        dma.signalDMAInterrupt();
 8001422:	6803      	ldr	r3, [r0, #0]
 8001424:	695b      	ldr	r3, [r3, #20]
 8001426:	4718      	bx	r3
 8001428:	20012630 	.word	0x20012630

0800142c <_ZN10STM32F4DMAC1Ev>:
STM32F4DMA::STM32F4DMA()
 800142c:	b570      	push	{r4, r5, r6, lr}
 800142e:	4604      	mov	r4, r0
    : DMA_Interface(dma_queue), dma_queue(queue_storage, sizeof(queue_storage) / sizeof(queue_storage[0]))
 8001430:	4625      	mov	r5, r4
 8001432:	4b0a      	ldr	r3, [pc, #40]	; (800145c <_ZN10STM32F4DMAC1Ev+0x30>)
 8001434:	300c      	adds	r0, #12
     * Constructs a DMA Interface object.
     *
     * @param [in] dmaQueue Reference to the queue of DMA operations.
     */
    DMA_Interface(DMA_Queue& dmaQueue)
        : queue(dmaQueue), isRunning(false), isAllowed(false)
 8001436:	2600      	movs	r6, #0
 8001438:	6060      	str	r0, [r4, #4]
 800143a:	7226      	strb	r6, [r4, #8]
 800143c:	7266      	strb	r6, [r4, #9]
 800143e:	f845 3b20 	str.w	r3, [r5], #32
 8001442:	2260      	movs	r2, #96	; 0x60
 8001444:	4629      	mov	r1, r5
 8001446:	f008 ffe5 	bl	800a414 <_ZN8touchgfx17LockFreeDMA_QueueC1EPNS_6BlitOpEi>
 800144a:	f504 6342 	add.w	r3, r4, #3104	; 0xc20
 */
struct colortype
{
    /** Default constructor. Creates a black (0) color. */
    colortype()
        : color(0)
 800144e:	60ee      	str	r6, [r5, #12]
 8001450:	3520      	adds	r5, #32
 8001452:	42ab      	cmp	r3, r5
 8001454:	d1fb      	bne.n	800144e <_ZN10STM32F4DMAC1Ev+0x22>
}
 8001456:	4620      	mov	r0, r4
 8001458:	bd70      	pop	{r4, r5, r6, pc}
 800145a:	bf00      	nop
 800145c:	0801ea50 	.word	0x0801ea50

08001460 <_ZN10STM32F4DMA22getChromARTInputFormatEN8touchgfx6Bitmap12BitmapFormatE>:
{
 8001460:	b508      	push	{r3, lr}
    switch (format)
 8001462:	290b      	cmp	r1, #11
 8001464:	d80b      	bhi.n	800147e <_ZN10STM32F4DMA22getChromARTInputFormatEN8touchgfx6Bitmap12BitmapFormatE+0x1e>
 8001466:	e8df f001 	tbb	[pc, r1]
 800146a:	0612      	.short	0x0612
 800146c:	0a0a0a10 	.word	0x0a0a0a10
 8001470:	0808080a 	.word	0x0808080a
 8001474:	0808      	.short	0x0808
 8001476:	2001      	movs	r0, #1
}
 8001478:	bd08      	pop	{r3, pc}
        dma2dColorMode = DMA2D_INPUT_L8;
 800147a:	2005      	movs	r0, #5
        break;
 800147c:	e7fc      	b.n	8001478 <_ZN10STM32F4DMA22getChromARTInputFormatEN8touchgfx6Bitmap12BitmapFormatE+0x18>
        assert(0 && "Unsupported Format!");
 800147e:	4b05      	ldr	r3, [pc, #20]	; (8001494 <_ZN10STM32F4DMA22getChromARTInputFormatEN8touchgfx6Bitmap12BitmapFormatE+0x34>)
 8001480:	4a05      	ldr	r2, [pc, #20]	; (8001498 <_ZN10STM32F4DMA22getChromARTInputFormatEN8touchgfx6Bitmap12BitmapFormatE+0x38>)
 8001482:	4806      	ldr	r0, [pc, #24]	; (800149c <_ZN10STM32F4DMA22getChromARTInputFormatEN8touchgfx6Bitmap12BitmapFormatE+0x3c>)
 8001484:	2165      	movs	r1, #101	; 0x65
 8001486:	f01a facf 	bl	801ba28 <__assert_func>
        dma2dColorMode = DMA2D_INPUT_ARGB8888;
 800148a:	2000      	movs	r0, #0
 800148c:	e7f4      	b.n	8001478 <_ZN10STM32F4DMA22getChromARTInputFormatEN8touchgfx6Bitmap12BitmapFormatE+0x18>
        dma2dColorMode = DMA2D_INPUT_RGB565;
 800148e:	2002      	movs	r0, #2
    return dma2dColorMode;
 8001490:	e7f2      	b.n	8001478 <_ZN10STM32F4DMA22getChromARTInputFormatEN8touchgfx6Bitmap12BitmapFormatE+0x18>
 8001492:	bf00      	nop
 8001494:	0801e8ea 	.word	0x0801e8ea
 8001498:	0801e905 	.word	0x0801e905
 800149c:	0801e951 	.word	0x0801e951

080014a0 <_ZN10STM32F4DMA23getChromARTOutputFormatEN8touchgfx6Bitmap12BitmapFormatE>:
{
 80014a0:	b508      	push	{r3, lr}
    switch (format)
 80014a2:	290a      	cmp	r1, #10
 80014a4:	d809      	bhi.n	80014ba <_ZN10STM32F4DMA23getChromARTOutputFormatEN8touchgfx6Bitmap12BitmapFormatE+0x1a>
 80014a6:	e8df f001 	tbb	[pc, r1]
 80014aa:	0610      	.short	0x0610
 80014ac:	0808080e 	.word	0x0808080e
 80014b0:	06060608 	.word	0x06060608
 80014b4:	06          	.byte	0x06
 80014b5:	00          	.byte	0x00
 80014b6:	2001      	movs	r0, #1
}
 80014b8:	bd08      	pop	{r3, pc}
        assert(0 && "Unsupported Format!");
 80014ba:	4b05      	ldr	r3, [pc, #20]	; (80014d0 <_ZN10STM32F4DMA23getChromARTOutputFormatEN8touchgfx6Bitmap12BitmapFormatE+0x30>)
 80014bc:	4a05      	ldr	r2, [pc, #20]	; (80014d4 <_ZN10STM32F4DMA23getChromARTOutputFormatEN8touchgfx6Bitmap12BitmapFormatE+0x34>)
 80014be:	4806      	ldr	r0, [pc, #24]	; (80014d8 <_ZN10STM32F4DMA23getChromARTOutputFormatEN8touchgfx6Bitmap12BitmapFormatE+0x38>)
 80014c0:	2186      	movs	r1, #134	; 0x86
 80014c2:	f01a fab1 	bl	801ba28 <__assert_func>
        dma2dColorMode = DMA2D_OUTPUT_ARGB8888;
 80014c6:	2000      	movs	r0, #0
 80014c8:	e7f6      	b.n	80014b8 <_ZN10STM32F4DMA23getChromARTOutputFormatEN8touchgfx6Bitmap12BitmapFormatE+0x18>
        dma2dColorMode = DMA2D_OUTPUT_RGB565;
 80014ca:	2002      	movs	r0, #2
    return dma2dColorMode;
 80014cc:	e7f4      	b.n	80014b8 <_ZN10STM32F4DMA23getChromARTOutputFormatEN8touchgfx6Bitmap12BitmapFormatE+0x18>
 80014ce:	bf00      	nop
 80014d0:	0801e8ea 	.word	0x0801e8ea
 80014d4:	0801e99f 	.word	0x0801e99f
 80014d8:	0801e951 	.word	0x0801e951

080014dc <_ZN10STM32F4DMA13setupDataCopyERKN8touchgfx6BlitOpE>:
 * BLIT_OP_COPY_ARGB8888_WITH_ALPHA
 * BLIT_OP_COPY_A4
 * BLIT_OP_COPY_A8
 */
void STM32F4DMA::setupDataCopy(const BlitOp& blitOp)
{
 80014dc:	e92d 43f8 	stmdb	sp!, {r3, r4, r5, r6, r7, r8, r9, lr}
    uint32_t dma2dForegroundColorMode = getChromARTInputFormat(static_cast<Bitmap::BitmapFormat>(blitOp.srcFormat));
 80014e0:	7f4f      	ldrb	r7, [r1, #29]
{
 80014e2:	460c      	mov	r4, r1
    uint32_t dma2dForegroundColorMode = getChromARTInputFormat(static_cast<Bitmap::BitmapFormat>(blitOp.srcFormat));
 80014e4:	4639      	mov	r1, r7
{
 80014e6:	4681      	mov	r9, r0
    uint32_t dma2dForegroundColorMode = getChromARTInputFormat(static_cast<Bitmap::BitmapFormat>(blitOp.srcFormat));
 80014e8:	f7ff ffba 	bl	8001460 <_ZN10STM32F4DMA22getChromARTInputFormatEN8touchgfx6Bitmap12BitmapFormatE>
    uint32_t dma2dBackgroundColorMode = getChromARTInputFormat(static_cast<Bitmap::BitmapFormat>(blitOp.dstFormat));
 80014ec:	f894 801e 	ldrb.w	r8, [r4, #30]
    uint32_t dma2dForegroundColorMode = getChromARTInputFormat(static_cast<Bitmap::BitmapFormat>(blitOp.srcFormat));
 80014f0:	4605      	mov	r5, r0
    uint32_t dma2dBackgroundColorMode = getChromARTInputFormat(static_cast<Bitmap::BitmapFormat>(blitOp.dstFormat));
 80014f2:	4641      	mov	r1, r8
 80014f4:	4648      	mov	r0, r9
 80014f6:	f7ff ffb3 	bl	8001460 <_ZN10STM32F4DMA22getChromARTInputFormatEN8touchgfx6Bitmap12BitmapFormatE>
    uint32_t dma2dOutputColorMode = getChromARTOutputFormat(static_cast<Bitmap::BitmapFormat>(blitOp.dstFormat));
 80014fa:	4641      	mov	r1, r8
    uint32_t dma2dBackgroundColorMode = getChromARTInputFormat(static_cast<Bitmap::BitmapFormat>(blitOp.dstFormat));
 80014fc:	4606      	mov	r6, r0
    uint32_t dma2dOutputColorMode = getChromARTOutputFormat(static_cast<Bitmap::BitmapFormat>(blitOp.dstFormat));
 80014fe:	4648      	mov	r0, r9
 8001500:	f7ff ffce 	bl	80014a0 <_ZN10STM32F4DMA23getChromARTOutputFormatEN8touchgfx6Bitmap12BitmapFormatE>

    /* DMA2D OOR register configuration ------------------------------------------*/
    WRITE_REG(DMA2D->OOR, blitOp.dstLoopStride - blitOp.nSteps);
 8001504:	8aa1      	ldrh	r1, [r4, #20]
 8001506:	8b62      	ldrh	r2, [r4, #26]
 8001508:	4b49      	ldr	r3, [pc, #292]	; (8001630 <_ZN10STM32F4DMA13setupDataCopyERKN8touchgfx6BlitOpE+0x154>)
 800150a:	1a52      	subs	r2, r2, r1
 800150c:	641a      	str	r2, [r3, #64]	; 0x40

    /* DMA2D BGOR register configuration -------------------------------------*/
    WRITE_REG(DMA2D->BGOR, blitOp.dstLoopStride - blitOp.nSteps);
 800150e:	619a      	str	r2, [r3, #24]

    /* DMA2D FGOR register configuration -------------------------------------*/
    WRITE_REG(DMA2D->FGOR, blitOp.srcLoopStride - blitOp.nSteps);
 8001510:	8b22      	ldrh	r2, [r4, #24]
 8001512:	1a52      	subs	r2, r2, r1
 8001514:	611a      	str	r2, [r3, #16]

    /* DMA2D OPFCCR register configuration ---------------------------------------*/
    WRITE_REG(DMA2D->OPFCCR, dma2dOutputColorMode);

    /* Configure DMA2D data size */
    WRITE_REG(DMA2D->NLR, (blitOp.nLoops | (blitOp.nSteps << DMA2D_NLR_PL_Pos)));
 8001516:	8ae2      	ldrh	r2, [r4, #22]
    WRITE_REG(DMA2D->OPFCCR, dma2dOutputColorMode);
 8001518:	6358      	str	r0, [r3, #52]	; 0x34
    WRITE_REG(DMA2D->NLR, (blitOp.nLoops | (blitOp.nSteps << DMA2D_NLR_PL_Pos)));
 800151a:	ea42 4201 	orr.w	r2, r2, r1, lsl #16
 800151e:	645a      	str	r2, [r3, #68]	; 0x44

    /* Configure DMA2D destination address */
    WRITE_REG(DMA2D->OMAR, reinterpret_cast<uint32_t>(blitOp.pDst));
 8001520:	6920      	ldr	r0, [r4, #16]

    /* Configure DMA2D source address */
    WRITE_REG(DMA2D->FGMAR, reinterpret_cast<uint32_t>(blitOp.pSrc));
 8001522:	6862      	ldr	r2, [r4, #4]
    WRITE_REG(DMA2D->OMAR, reinterpret_cast<uint32_t>(blitOp.pDst));
 8001524:	63d8      	str	r0, [r3, #60]	; 0x3c
    WRITE_REG(DMA2D->FGMAR, reinterpret_cast<uint32_t>(blitOp.pSrc));
 8001526:	60da      	str	r2, [r3, #12]

    switch (blitOp.operation)
 8001528:	6821      	ldr	r1, [r4, #0]
    {
    case BLIT_OP_COPY_A4:
        /* Set DMA2D color mode and alpha mode */
        WRITE_REG(DMA2D->FGPFCCR, DMA2D_INPUT_A4 | (DMA2D_COMBINE_ALPHA << DMA2D_BGPFCCR_AM_Pos) | (blitOp.alpha << 24));
 800152a:	f894 c01c 	ldrb.w	ip, [r4, #28]
    switch (blitOp.operation)
 800152e:	2980      	cmp	r1, #128	; 0x80
        WRITE_REG(DMA2D->FGPFCCR, DMA2D_INPUT_A4 | (DMA2D_COMBINE_ALPHA << DMA2D_BGPFCCR_AM_Pos) | (blitOp.alpha << 24));
 8001530:	ea4f 620c 	mov.w	r2, ip, lsl #24
    switch (blitOp.operation)
 8001534:	d034      	beq.n	80015a0 <_ZN10STM32F4DMA13setupDataCopyERKN8touchgfx6BlitOpE+0xc4>
 8001536:	d812      	bhi.n	800155e <_ZN10STM32F4DMA13setupDataCopyERKN8touchgfx6BlitOpE+0x82>
 8001538:	2920      	cmp	r1, #32
 800153a:	ea45 0402 	orr.w	r4, r5, r2
 800153e:	d073      	beq.n	8001628 <_ZN10STM32F4DMA13setupDataCopyERKN8touchgfx6BlitOpE+0x14c>
 8001540:	2940      	cmp	r1, #64	; 0x40
 8001542:	d071      	beq.n	8001628 <_ZN10STM32F4DMA13setupDataCopyERKN8touchgfx6BlitOpE+0x14c>
 8001544:	2904      	cmp	r1, #4
 8001546:	d06f      	beq.n	8001628 <_ZN10STM32F4DMA13setupDataCopyERKN8touchgfx6BlitOpE+0x14c>
        /* Set DMA2D mode */
        WRITE_REG(DMA2D->CR, DMA2D_M2M_BLEND | DMA2D_IT_TC | DMA2D_CR_START);
        break;
    default: /* BLIT_OP_COPY */
        /* Set DMA2D color mode and alpha mode */
        WRITE_REG(DMA2D->FGPFCCR, dma2dForegroundColorMode | (DMA2D_COMBINE_ALPHA << DMA2D_BGPFCCR_AM_Pos) | (blitOp.alpha << 24));
 8001548:	4b39      	ldr	r3, [pc, #228]	; (8001630 <_ZN10STM32F4DMA13setupDataCopyERKN8touchgfx6BlitOpE+0x154>)
 800154a:	432a      	orrs	r2, r5
 800154c:	f442 3200 	orr.w	r2, r2, #131072	; 0x20000

        /* Perform pixel-format-conversion (PFC) If Bitmap format is not same format as framebuffer format */
        if (blitOp.srcFormat != blitOp.dstFormat)
 8001550:	4547      	cmp	r7, r8
        WRITE_REG(DMA2D->FGPFCCR, dma2dForegroundColorMode | (DMA2D_COMBINE_ALPHA << DMA2D_BGPFCCR_AM_Pos) | (blitOp.alpha << 24));
 8001552:	61da      	str	r2, [r3, #28]
        {
            /* Start DMA2D : PFC Mode */
            WRITE_REG(DMA2D->CR, DMA2D_M2M_PFC | DMA2D_IT_TC | DMA2D_CR_START);
 8001554:	bf14      	ite	ne
 8001556:	4a37      	ldrne	r2, [pc, #220]	; (8001634 <_ZN10STM32F4DMA13setupDataCopyERKN8touchgfx6BlitOpE+0x158>)
        }
        else
        {
            /* Start DMA2D : M2M Mode */
            WRITE_REG(DMA2D->CR, DMA2D_M2M | DMA2D_IT_TC | DMA2D_CR_START);
 8001558:	f240 2201 	movweq	r2, #513	; 0x201
 800155c:	e01e      	b.n	800159c <_ZN10STM32F4DMA13setupDataCopyERKN8touchgfx6BlitOpE+0xc0>
    switch (blitOp.operation)
 800155e:	f5b1 7f80 	cmp.w	r1, #256	; 0x100
 8001562:	d007      	beq.n	8001574 <_ZN10STM32F4DMA13setupDataCopyERKN8touchgfx6BlitOpE+0x98>
 8001564:	f5b1 7f00 	cmp.w	r1, #512	; 0x200
 8001568:	d1ee      	bne.n	8001548 <_ZN10STM32F4DMA13setupDataCopyERKN8touchgfx6BlitOpE+0x6c>
        WRITE_REG(DMA2D->FGPFCCR, DMA2D_INPUT_A8 | (DMA2D_COMBINE_ALPHA << DMA2D_BGPFCCR_AM_Pos) | (blitOp.alpha << 24));
 800156a:	f442 3200 	orr.w	r2, r2, #131072	; 0x20000
 800156e:	f042 0209 	orr.w	r2, r2, #9
 8001572:	e003      	b.n	800157c <_ZN10STM32F4DMA13setupDataCopyERKN8touchgfx6BlitOpE+0xa0>
        WRITE_REG(DMA2D->FGPFCCR, DMA2D_INPUT_A4 | (DMA2D_COMBINE_ALPHA << DMA2D_BGPFCCR_AM_Pos) | (blitOp.alpha << 24));
 8001574:	f442 3200 	orr.w	r2, r2, #131072	; 0x20000
 8001578:	f042 020a 	orr.w	r2, r2, #10
        WRITE_REG(DMA2D->FGPFCCR, DMA2D_INPUT_A8 | (DMA2D_COMBINE_ALPHA << DMA2D_BGPFCCR_AM_Pos) | (blitOp.alpha << 24));
 800157c:	61da      	str	r2, [r3, #28]
     *
     * @return The result of the operation.
     */
    operator uint32_t() const
    {
        return color;
 800157e:	68e1      	ldr	r1, [r4, #12]
        WRITE_REG(DMA2D->FGCOLR, ((blitOp.color & 0xF800) << 8) | ((blitOp.color & 0x07E0) << 5) | ((blitOp.color & 0x001F) << 3));
 8001580:	020a      	lsls	r2, r1, #8
 8001582:	014c      	lsls	r4, r1, #5
 8001584:	f402 0278 	and.w	r2, r2, #16252928	; 0xf80000
 8001588:	f404 447c 	and.w	r4, r4, #64512	; 0xfc00
 800158c:	00c9      	lsls	r1, r1, #3
 800158e:	4322      	orrs	r2, r4
 8001590:	b2c9      	uxtb	r1, r1
 8001592:	430a      	orrs	r2, r1
 8001594:	621a      	str	r2, [r3, #32]
        WRITE_REG(DMA2D->CR, DMA2D_M2M_BLEND | DMA2D_IT_TC | DMA2D_CR_START);
 8001596:	4a28      	ldr	r2, [pc, #160]	; (8001638 <_ZN10STM32F4DMA13setupDataCopyERKN8touchgfx6BlitOpE+0x15c>)
        WRITE_REG(DMA2D->BGPFCCR, dma2dBackgroundColorMode | (DMA2D_NO_MODIF_ALPHA << DMA2D_BGPFCCR_AM_Pos));
 8001598:	625e      	str	r6, [r3, #36]	; 0x24
        WRITE_REG(DMA2D->BGMAR, reinterpret_cast<uint32_t>(blitOp.pDst));
 800159a:	6158      	str	r0, [r3, #20]
            WRITE_REG(DMA2D->CR, DMA2D_M2M | DMA2D_IT_TC | DMA2D_CR_START);
 800159c:	601a      	str	r2, [r3, #0]
        }
        break;
    }
}
 800159e:	e03f      	b.n	8001620 <_ZN10STM32F4DMA13setupDataCopyERKN8touchgfx6BlitOpE+0x144>
            const clutData_t* const palette = reinterpret_cast<const clutData_t*>(blitOp.pClut);
 80015a0:	68a4      	ldr	r4, [r4, #8]
            WRITE_REG(DMA2D->FGPFCCR, dma2dForegroundColorMode | (DMA2D_COMBINE_ALPHA << DMA2D_BGPFCCR_AM_Pos) | (blitOp.alpha << 24));
 80015a2:	432a      	orrs	r2, r5
 80015a4:	f442 3200 	orr.w	r2, r2, #131072	; 0x20000
            WRITE_REG(DMA2D->FGCMAR, reinterpret_cast<uint32_t>(&palette->data));
 80015a8:	1d21      	adds	r1, r4, #4
 80015aa:	62d9      	str	r1, [r3, #44]	; 0x2c
            WRITE_REG(DMA2D->FGPFCCR, dma2dForegroundColorMode | (DMA2D_COMBINE_ALPHA << DMA2D_BGPFCCR_AM_Pos) | (blitOp.alpha << 24));
 80015ac:	61da      	str	r2, [r3, #28]
            switch ((Bitmap::ClutFormat)palette->format)
 80015ae:	7822      	ldrb	r2, [r4, #0]
            WRITE_REG(DMA2D->BGPFCCR, dma2dBackgroundColorMode | (DMA2D_NO_MODIF_ALPHA << DMA2D_BGPFCCR_AM_Pos));
 80015b0:	625e      	str	r6, [r3, #36]	; 0x24
            WRITE_REG(DMA2D->BGMAR, reinterpret_cast<uint32_t>(blitOp.pDst));
 80015b2:	6158      	str	r0, [r3, #20]
            switch ((Bitmap::ClutFormat)palette->format)
 80015b4:	b142      	cbz	r2, 80015c8 <_ZN10STM32F4DMA13setupDataCopyERKN8touchgfx6BlitOpE+0xec>
 80015b6:	2a01      	cmp	r2, #1
 80015b8:	d01c      	beq.n	80015f4 <_ZN10STM32F4DMA13setupDataCopyERKN8touchgfx6BlitOpE+0x118>
                assert(0 && "Unsupported format");
 80015ba:	4b20      	ldr	r3, [pc, #128]	; (800163c <_ZN10STM32F4DMA13setupDataCopyERKN8touchgfx6BlitOpE+0x160>)
 80015bc:	4a20      	ldr	r2, [pc, #128]	; (8001640 <_ZN10STM32F4DMA13setupDataCopyERKN8touchgfx6BlitOpE+0x164>)
 80015be:	4821      	ldr	r0, [pc, #132]	; (8001644 <_ZN10STM32F4DMA13setupDataCopyERKN8touchgfx6BlitOpE+0x168>)
 80015c0:	f44f 7188 	mov.w	r1, #272	; 0x110
 80015c4:	f01a fa30 	bl	801ba28 <__assert_func>
                MODIFY_REG(DMA2D->FGPFCCR, (DMA2D_FGPFCCR_CS | DMA2D_FGPFCCR_CCM), (((palette->size - 1) << DMA2D_FGPFCCR_CS_Pos) | (DMA2D_CCM_ARGB8888 << DMA2D_FGPFCCR_CCM_Pos)));
 80015c8:	69da      	ldr	r2, [r3, #28]
 80015ca:	8861      	ldrh	r1, [r4, #2]
 80015cc:	f422 427f 	bic.w	r2, r2, #65280	; 0xff00
 80015d0:	3901      	subs	r1, #1
 80015d2:	f022 0210 	bic.w	r2, r2, #16
 80015d6:	ea42 2201 	orr.w	r2, r2, r1, lsl #8
 80015da:	61da      	str	r2, [r3, #28]
            bool blend = true;
 80015dc:	2501      	movs	r5, #1
            SET_BIT(DMA2D->FGPFCCR, DMA2D_FGPFCCR_START);
 80015de:	4c14      	ldr	r4, [pc, #80]	; (8001630 <_ZN10STM32F4DMA13setupDataCopyERKN8touchgfx6BlitOpE+0x154>)
 80015e0:	69e3      	ldr	r3, [r4, #28]
 80015e2:	f043 0320 	orr.w	r3, r3, #32
 80015e6:	61e3      	str	r3, [r4, #28]
            while ((READ_REG(DMA2D->FGPFCCR) & DMA2D_FGPFCCR_START) != 0U)
 80015e8:	69e3      	ldr	r3, [r4, #28]
 80015ea:	069b      	lsls	r3, r3, #26
 80015ec:	d513      	bpl.n	8001616 <_ZN10STM32F4DMA13setupDataCopyERKN8touchgfx6BlitOpE+0x13a>
                OSWrappers::taskYield();
 80015ee:	f7ff fec5 	bl	800137c <_ZN8touchgfx10OSWrappers9taskYieldEv>
            while ((READ_REG(DMA2D->FGPFCCR) & DMA2D_FGPFCCR_START) != 0U)
 80015f2:	e7f9      	b.n	80015e8 <_ZN10STM32F4DMA13setupDataCopyERKN8touchgfx6BlitOpE+0x10c>
                MODIFY_REG(DMA2D->FGPFCCR, (DMA2D_FGPFCCR_CS | DMA2D_FGPFCCR_CCM), (((palette->size - 1) << DMA2D_FGPFCCR_CS_Pos) | (DMA2D_CCM_RGB888 << DMA2D_FGPFCCR_CCM_Pos)));
 80015f4:	8862      	ldrh	r2, [r4, #2]
 80015f6:	69d9      	ldr	r1, [r3, #28]
 80015f8:	1e50      	subs	r0, r2, #1
 80015fa:	f421 427f 	bic.w	r2, r1, #65280	; 0xff00
 80015fe:	f022 0210 	bic.w	r2, r2, #16
 8001602:	ea42 2200 	orr.w	r2, r2, r0, lsl #8
                if(blitOp.alpha == 255)
 8001606:	f1bc 05ff 	subs.w	r5, ip, #255	; 0xff
                MODIFY_REG(DMA2D->FGPFCCR, (DMA2D_FGPFCCR_CS | DMA2D_FGPFCCR_CCM), (((palette->size - 1) << DMA2D_FGPFCCR_CS_Pos) | (DMA2D_CCM_RGB888 << DMA2D_FGPFCCR_CCM_Pos)));
 800160a:	f042 0210 	orr.w	r2, r2, #16
                if(blitOp.alpha == 255)
 800160e:	bf18      	it	ne
 8001610:	2501      	movne	r5, #1
                MODIFY_REG(DMA2D->FGPFCCR, (DMA2D_FGPFCCR_CS | DMA2D_FGPFCCR_CCM), (((palette->size - 1) << DMA2D_FGPFCCR_CS_Pos) | (DMA2D_CCM_RGB888 << DMA2D_FGPFCCR_CCM_Pos)));
 8001612:	61da      	str	r2, [r3, #28]
                break;
 8001614:	e7e3      	b.n	80015de <_ZN10STM32F4DMA13setupDataCopyERKN8touchgfx6BlitOpE+0x102>
            DMA2D->IFCR = (DMA2D_FLAG_CTC);
 8001616:	2310      	movs	r3, #16
 8001618:	60a3      	str	r3, [r4, #8]
            if(blend)
 800161a:	b11d      	cbz	r5, 8001624 <_ZN10STM32F4DMA13setupDataCopyERKN8touchgfx6BlitOpE+0x148>
                WRITE_REG(DMA2D->CR, DMA2D_M2M_BLEND | DMA2D_IT_TC | DMA2D_CR_START);
 800161c:	4b06      	ldr	r3, [pc, #24]	; (8001638 <_ZN10STM32F4DMA13setupDataCopyERKN8touchgfx6BlitOpE+0x15c>)
                WRITE_REG(DMA2D->CR, DMA2D_M2M_PFC | DMA2D_IT_TC | DMA2D_CR_START);
 800161e:	6023      	str	r3, [r4, #0]
}
 8001620:	e8bd 83f8 	ldmia.w	sp!, {r3, r4, r5, r6, r7, r8, r9, pc}
                WRITE_REG(DMA2D->CR, DMA2D_M2M_PFC | DMA2D_IT_TC | DMA2D_CR_START);
 8001624:	4b03      	ldr	r3, [pc, #12]	; (8001634 <_ZN10STM32F4DMA13setupDataCopyERKN8touchgfx6BlitOpE+0x158>)
 8001626:	e7fa      	b.n	800161e <_ZN10STM32F4DMA13setupDataCopyERKN8touchgfx6BlitOpE+0x142>
        WRITE_REG(DMA2D->FGPFCCR, dma2dForegroundColorMode | (DMA2D_COMBINE_ALPHA << DMA2D_BGPFCCR_AM_Pos) | (blitOp.alpha << 24));
 8001628:	f444 3400 	orr.w	r4, r4, #131072	; 0x20000
 800162c:	61dc      	str	r4, [r3, #28]
 800162e:	e7b2      	b.n	8001596 <_ZN10STM32F4DMA13setupDataCopyERKN8touchgfx6BlitOpE+0xba>
 8001630:	4002b000 	.word	0x4002b000
 8001634:	00010201 	.word	0x00010201
 8001638:	00020201 	.word	0x00020201
 800163c:	0801e9ec 	.word	0x0801e9ec
 8001640:	0801ea06 	.word	0x0801ea06
 8001644:	0801e951 	.word	0x0801e951

08001648 <_ZN10STM32F4DMA13setupDataFillERKN8touchgfx6BlitOpE>:
 * void STM32F4DMA::setupDataFill(const BlitOp& blitOp) handles blit operation of
 * BLIT_OP_FILL
 * BLIT_OP_FILL_WITH_ALPHA
 */
void STM32F4DMA::setupDataFill(const BlitOp& blitOp)
{
 8001648:	b5f8      	push	{r3, r4, r5, r6, r7, lr}
    uint32_t dma2dOutputColorMode = getChromARTOutputFormat(static_cast<Bitmap::BitmapFormat>(blitOp.dstFormat));
 800164a:	7f8f      	ldrb	r7, [r1, #30]
{
 800164c:	460c      	mov	r4, r1
    uint32_t dma2dOutputColorMode = getChromARTOutputFormat(static_cast<Bitmap::BitmapFormat>(blitOp.dstFormat));
 800164e:	4639      	mov	r1, r7
 8001650:	f7ff ff26 	bl	80014a0 <_ZN10STM32F4DMA23getChromARTOutputFormatEN8touchgfx6Bitmap12BitmapFormatE>

    /* DMA2D OPFCCR register configuration ---------------------------------------*/
    WRITE_REG(DMA2D->OPFCCR, dma2dOutputColorMode);

    /* Configure DMA2D data size */
    WRITE_REG(DMA2D->NLR, (blitOp.nLoops | (blitOp.nSteps << DMA2D_NLR_PL_Pos)));
 8001654:	8aa1      	ldrh	r1, [r4, #20]
 8001656:	8ae2      	ldrh	r2, [r4, #22]

    /* Configure DMA2D destination address */
    WRITE_REG(DMA2D->OMAR, reinterpret_cast<uint32_t>(blitOp.pDst));

    /* DMA2D OOR register configuration ------------------------------------------*/
    WRITE_REG(DMA2D->OOR, blitOp.dstLoopStride - blitOp.nSteps);
 8001658:	8b65      	ldrh	r5, [r4, #26]
    WRITE_REG(DMA2D->OPFCCR, dma2dOutputColorMode);
 800165a:	4b1e      	ldr	r3, [pc, #120]	; (80016d4 <_ZN10STM32F4DMA13setupDataFillERKN8touchgfx6BlitOpE+0x8c>)
    WRITE_REG(DMA2D->OMAR, reinterpret_cast<uint32_t>(blitOp.pDst));
 800165c:	6926      	ldr	r6, [r4, #16]
    WRITE_REG(DMA2D->OPFCCR, dma2dOutputColorMode);
 800165e:	6358      	str	r0, [r3, #52]	; 0x34
    WRITE_REG(DMA2D->NLR, (blitOp.nLoops | (blitOp.nSteps << DMA2D_NLR_PL_Pos)));
 8001660:	ea42 4201 	orr.w	r2, r2, r1, lsl #16
    WRITE_REG(DMA2D->OOR, blitOp.dstLoopStride - blitOp.nSteps);
 8001664:	1a6d      	subs	r5, r5, r1
    WRITE_REG(DMA2D->NLR, (blitOp.nLoops | (blitOp.nSteps << DMA2D_NLR_PL_Pos)));
 8001666:	645a      	str	r2, [r3, #68]	; 0x44
    WRITE_REG(DMA2D->OMAR, reinterpret_cast<uint32_t>(blitOp.pDst));
 8001668:	63de      	str	r6, [r3, #60]	; 0x3c
    WRITE_REG(DMA2D->OOR, blitOp.dstLoopStride - blitOp.nSteps);
 800166a:	641d      	str	r5, [r3, #64]	; 0x40

    if (blitOp.operation == BLIT_OP_FILL_WITH_ALPHA)
 800166c:	6821      	ldr	r1, [r4, #0]
 800166e:	68e2      	ldr	r2, [r4, #12]
 8001670:	2908      	cmp	r1, #8
 8001672:	d118      	bne.n	80016a6 <_ZN10STM32F4DMA13setupDataFillERKN8touchgfx6BlitOpE+0x5e>
    {
        /* DMA2D BGOR register configuration -------------------------------------*/
        WRITE_REG(DMA2D->BGOR, blitOp.dstLoopStride - blitOp.nSteps);
 8001674:	619d      	str	r5, [r3, #24]

        /* DMA2D FGOR register configuration -------------------------------------*/
        WRITE_REG(DMA2D->FGOR, blitOp.dstLoopStride - blitOp.nSteps);
 8001676:	611d      	str	r5, [r3, #16]

        /* Write DMA2D BGPFCCR register */
        WRITE_REG(DMA2D->BGPFCCR, dma2dOutputColorMode | (DMA2D_NO_MODIF_ALPHA << DMA2D_BGPFCCR_AM_Pos));
 8001678:	6258      	str	r0, [r3, #36]	; 0x24

        /* Write DMA2D FGPFCCR register */
        WRITE_REG(DMA2D->FGPFCCR, CM_A8 | (DMA2D_REPLACE_ALPHA << DMA2D_BGPFCCR_AM_Pos) | ((blitOp.alpha << 24) & DMA2D_BGPFCCR_ALPHA));
 800167a:	7f20      	ldrb	r0, [r4, #28]
 800167c:	f101 1101 	add.w	r1, r1, #65537	; 0x10001
 8001680:	ea41 6100 	orr.w	r1, r1, r0, lsl #24
 8001684:	61d9      	str	r1, [r3, #28]

        /* DMA2D FGCOLR register configuration -------------------------------------*/
        WRITE_REG(DMA2D->FGCOLR, (((blitOp.color & 0xF800) << 8) | ((blitOp.color & 0x07E0) << 5) | ((blitOp.color & 0x001F) << 3)) & (DMA2D_FGCOLR_BLUE | DMA2D_FGCOLR_GREEN | DMA2D_FGCOLR_RED));
 8001686:	0150      	lsls	r0, r2, #5
 8001688:	0211      	lsls	r1, r2, #8
 800168a:	f401 0178 	and.w	r1, r1, #16252928	; 0xf80000
 800168e:	f400 407c 	and.w	r0, r0, #64512	; 0xfc00
 8001692:	00d2      	lsls	r2, r2, #3
 8001694:	4301      	orrs	r1, r0
 8001696:	b2d2      	uxtb	r2, r2
 8001698:	430a      	orrs	r2, r1
 800169a:	621a      	str	r2, [r3, #32]

        /* Configure DMA2D source address */
        WRITE_REG(DMA2D->FGMAR, reinterpret_cast<uint32_t>(blitOp.pDst));

        /* Enable the Peripheral and Enable the transfer complete interrupt */
        WRITE_REG(DMA2D->CR, (DMA2D_IT_TC | DMA2D_CR_START | DMA2D_M2M_BLEND));
 800169c:	4a0e      	ldr	r2, [pc, #56]	; (80016d8 <_ZN10STM32F4DMA13setupDataFillERKN8touchgfx6BlitOpE+0x90>)
        WRITE_REG(DMA2D->BGMAR, reinterpret_cast<uint32_t>(blitOp.pDst));
 800169e:	615e      	str	r6, [r3, #20]
        WRITE_REG(DMA2D->FGMAR, reinterpret_cast<uint32_t>(blitOp.pDst));
 80016a0:	60de      	str	r6, [r3, #12]
            // set color
            WRITE_REG(DMA2D->OCOLR, (blitOp.alpha << 24) | ((blitOp.color & 0xF800) << 8) | ((blitOp.color & 0x07E0) << 5) | ((blitOp.color & 0x001F) << 3));
        }

        /* Enable the Peripheral and Enable the transfer complete interrupt */
        WRITE_REG(DMA2D->CR, (DMA2D_IT_TC | DMA2D_CR_START | DMA2D_R2M));
 80016a2:	601a      	str	r2, [r3, #0]
    }
}
 80016a4:	bdf8      	pop	{r3, r4, r5, r6, r7, pc}
        WRITE_REG(DMA2D->FGOR, 0);
 80016a6:	2100      	movs	r1, #0
        WRITE_REG(DMA2D->FGPFCCR, dma2dOutputColorMode | (DMA2D_NO_MODIF_ALPHA << DMA2D_BGPFCCR_AM_Pos));
 80016a8:	61d8      	str	r0, [r3, #28]
        WRITE_REG(DMA2D->FGOR, 0);
 80016aa:	6119      	str	r1, [r3, #16]
        if (blitOp.dstFormat == Bitmap::RGB565)
 80016ac:	b91f      	cbnz	r7, 80016b6 <_ZN10STM32F4DMA13setupDataFillERKN8touchgfx6BlitOpE+0x6e>
            WRITE_REG(DMA2D->OCOLR, (blitOp.alpha << 24) | ((blitOp.color & 0xF800) << 8) | ((blitOp.color & 0x07E0) << 5) | ((blitOp.color & 0x001F) << 3));
 80016ae:	639a      	str	r2, [r3, #56]	; 0x38
        WRITE_REG(DMA2D->CR, (DMA2D_IT_TC | DMA2D_CR_START | DMA2D_R2M));
 80016b0:	4b08      	ldr	r3, [pc, #32]	; (80016d4 <_ZN10STM32F4DMA13setupDataFillERKN8touchgfx6BlitOpE+0x8c>)
 80016b2:	4a0a      	ldr	r2, [pc, #40]	; (80016dc <_ZN10STM32F4DMA13setupDataFillERKN8touchgfx6BlitOpE+0x94>)
 80016b4:	e7f5      	b.n	80016a2 <_ZN10STM32F4DMA13setupDataFillERKN8touchgfx6BlitOpE+0x5a>
            WRITE_REG(DMA2D->OCOLR, (blitOp.alpha << 24) | ((blitOp.color & 0xF800) << 8) | ((blitOp.color & 0x07E0) << 5) | ((blitOp.color & 0x001F) << 3));
 80016b6:	0211      	lsls	r1, r2, #8
 80016b8:	0150      	lsls	r0, r2, #5
 80016ba:	f401 0178 	and.w	r1, r1, #16252928	; 0xf80000
 80016be:	f400 407c 	and.w	r0, r0, #64512	; 0xfc00
 80016c2:	00d2      	lsls	r2, r2, #3
 80016c4:	4301      	orrs	r1, r0
 80016c6:	b2d2      	uxtb	r2, r2
 80016c8:	430a      	orrs	r2, r1
 80016ca:	7f21      	ldrb	r1, [r4, #28]
 80016cc:	ea42 6201 	orr.w	r2, r2, r1, lsl #24
 80016d0:	e7ed      	b.n	80016ae <_ZN10STM32F4DMA13setupDataFillERKN8touchgfx6BlitOpE+0x66>
 80016d2:	bf00      	nop
 80016d4:	4002b000 	.word	0x4002b000
 80016d8:	00020201 	.word	0x00020201
 80016dc:	00030201 	.word	0x00030201

080016e0 <_ZNK8touchgfx9PartitionINS_4meta8TypeListINS_12NoTransitionENS2_INS1_3NilES4_EEEELt1EE8capacityEv>:
    };

    virtual uint16_t capacity() const
    {
        return NUMBER_OF_ELEMENTS;
    }
 80016e0:	2001      	movs	r0, #1
 80016e2:	4770      	bx	lr

080016e4 <_ZN8touchgfx9PartitionINS_4meta8TypeListINS_12NoTransitionENS2_INS1_3NilES4_EEEELt1EE12element_sizeEv>:

    virtual uint32_t element_size()
    {
        return sizeof(stBlocks[0]);
    }
 80016e4:	200c      	movs	r0, #12
 80016e6:	4770      	bx	lr

080016e8 <_ZN8touchgfx9PartitionINS_4meta8TypeListINS_12NoTransitionENS2_INS1_3NilES4_EEEELt1EE7elementEt>:

protected:
    virtual void* element(uint16_t index)
    {
        return &stBlocks[index];
 80016e8:	230c      	movs	r3, #12
 80016ea:	fb03 0001 	mla	r0, r3, r1, r0
    }
 80016ee:	3008      	adds	r0, #8
 80016f0:	4770      	bx	lr

080016f2 <_ZNK8touchgfx9PartitionINS_4meta8TypeListINS_12NoTransitionENS2_INS1_3NilES4_EEEELt1EE7elementEt>:

    virtual const void* element(uint16_t index) const
    {
        return &stBlocks[index];
 80016f2:	230c      	movs	r3, #12
 80016f4:	fb03 0001 	mla	r0, r3, r1, r0
    }
 80016f8:	3008      	adds	r0, #8
 80016fa:	4770      	bx	lr

080016fc <_ZNK8touchgfx9PartitionINS_4meta8TypeListI11Screen1ViewNS2_INS1_3NilES4_EEEELt1EE8capacityEv>:
    }
 80016fc:	2001      	movs	r0, #1
 80016fe:	4770      	bx	lr

08001700 <_ZN8touchgfx9PartitionINS_4meta8TypeListI11Screen1ViewNS2_INS1_3NilES4_EEEELt1EE12element_sizeEv>:
    }
 8001700:	f44f 70ba 	mov.w	r0, #372	; 0x174
 8001704:	4770      	bx	lr

08001706 <_ZN8touchgfx9PartitionINS_4meta8TypeListI11Screen1ViewNS2_INS1_3NilES4_EEEELt1EE7elementEt>:
        return &stBlocks[index];
 8001706:	f44f 73ba 	mov.w	r3, #372	; 0x174
 800170a:	fb03 0001 	mla	r0, r3, r1, r0
    }
 800170e:	3008      	adds	r0, #8
 8001710:	4770      	bx	lr

08001712 <_ZNK8touchgfx9PartitionINS_4meta8TypeListI11Screen1ViewNS2_INS1_3NilES4_EEEELt1EE7elementEt>:
        return &stBlocks[index];
 8001712:	f44f 73ba 	mov.w	r3, #372	; 0x174
 8001716:	fb03 0001 	mla	r0, r3, r1, r0
    }
 800171a:	3008      	adds	r0, #8
 800171c:	4770      	bx	lr

0800171e <_ZNK8touchgfx9PartitionINS_4meta8TypeListI16Screen1PresenterNS2_INS1_3NilES4_EEEELt1EE8capacityEv>:
    }
 800171e:	2001      	movs	r0, #1
 8001720:	4770      	bx	lr

08001722 <_ZN8touchgfx9PartitionINS_4meta8TypeListI16Screen1PresenterNS2_INS1_3NilES4_EEEELt1EE12element_sizeEv>:
    }
 8001722:	2010      	movs	r0, #16
 8001724:	4770      	bx	lr

08001726 <_ZN8touchgfx9PartitionINS_4meta8TypeListI16Screen1PresenterNS2_INS1_3NilES4_EEEELt1EE7elementEt>:
        return &stBlocks[index];
 8001726:	eb00 1001 	add.w	r0, r0, r1, lsl #4
    }
 800172a:	3008      	adds	r0, #8
 800172c:	4770      	bx	lr

0800172e <_ZNK8touchgfx9PartitionINS_4meta8TypeListI16Screen1PresenterNS2_INS1_3NilES4_EEEELt1EE7elementEt>:
        return &stBlocks[index];
 800172e:	eb00 1001 	add.w	r0, r0, r1, lsl #4
    }
 8001732:	3008      	adds	r0, #8
 8001734:	4770      	bx	lr

08001736 <_ZN16FrontendHeapBase15gotoStartScreenER19FrontendApplication>:
     */
    typedef touchgfx::meta::select_type_maxsize< GeneratedTransitionTypes >::type MaxGeneratedTransitionType;

    virtual void gotoStartScreen(FrontendApplication& app)
    {
        app.gotoScreen1ScreenNoTransition();
 8001736:	4608      	mov	r0, r1
 8001738:	f001 be82 	b.w	8003440 <_ZN23FrontendApplicationBase29gotoScreen1ScreenNoTransitionEv>

0800173c <_ZN8touchgfx9PartitionINS_4meta8TypeListINS_12NoTransitionENS2_INS1_3NilES4_EEEELt1EED1Ev>:
class Partition : public AbstractPartition
 800173c:	b510      	push	{r4, lr}
 800173e:	4b03      	ldr	r3, [pc, #12]	; (800174c <_ZN8touchgfx9PartitionINS_4meta8TypeListINS_12NoTransitionENS2_INS1_3NilES4_EEEELt1EED1Ev+0x10>)
 8001740:	6003      	str	r3, [r0, #0]
 8001742:	4604      	mov	r4, r0
 8001744:	f007 fcfa 	bl	800913c <_ZN8touchgfx17AbstractPartitionD1Ev>
 8001748:	4620      	mov	r0, r4
 800174a:	bd10      	pop	{r4, pc}
 800174c:	0801eb08 	.word	0x0801eb08

08001750 <_ZN8touchgfx9PartitionINS_4meta8TypeListINS_12NoTransitionENS2_INS1_3NilES4_EEEELt1EED0Ev>:
 8001750:	b510      	push	{r4, lr}
 8001752:	4604      	mov	r4, r0
 8001754:	f7ff fff2 	bl	800173c <_ZN8touchgfx9PartitionINS_4meta8TypeListINS_12NoTransitionENS2_INS1_3NilES4_EEEELt1EED1Ev>
 8001758:	4620      	mov	r0, r4
 800175a:	2114      	movs	r1, #20
 800175c:	f01a f935 	bl	801b9ca <_ZdlPvj>
 8001760:	4620      	mov	r0, r4
 8001762:	bd10      	pop	{r4, pc}

08001764 <_ZN8touchgfx9PartitionINS_4meta8TypeListI11Screen1ViewNS2_INS1_3NilES4_EEEELt1EED1Ev>:
 8001764:	b510      	push	{r4, lr}
 8001766:	4b03      	ldr	r3, [pc, #12]	; (8001774 <_ZN8touchgfx9PartitionINS_4meta8TypeListI11Screen1ViewNS2_INS1_3NilES4_EEEELt1EED1Ev+0x10>)
 8001768:	6003      	str	r3, [r0, #0]
 800176a:	4604      	mov	r4, r0
 800176c:	f007 fce6 	bl	800913c <_ZN8touchgfx17AbstractPartitionD1Ev>
 8001770:	4620      	mov	r0, r4
 8001772:	bd10      	pop	{r4, pc}
 8001774:	0801ead4 	.word	0x0801ead4

08001778 <_ZN8touchgfx9PartitionINS_4meta8TypeListI11Screen1ViewNS2_INS1_3NilES4_EEEELt1EED0Ev>:
 8001778:	b510      	push	{r4, lr}
 800177a:	4604      	mov	r4, r0
 800177c:	f7ff fff2 	bl	8001764 <_ZN8touchgfx9PartitionINS_4meta8TypeListI11Screen1ViewNS2_INS1_3NilES4_EEEELt1EED1Ev>
 8001780:	4620      	mov	r0, r4
 8001782:	f44f 71be 	mov.w	r1, #380	; 0x17c
 8001786:	f01a f920 	bl	801b9ca <_ZdlPvj>
 800178a:	4620      	mov	r0, r4
 800178c:	bd10      	pop	{r4, pc}
	...

08001790 <_ZN8touchgfx9PartitionINS_4meta8TypeListI16Screen1PresenterNS2_INS1_3NilES4_EEEELt1EED1Ev>:
 8001790:	b510      	push	{r4, lr}
 8001792:	4b03      	ldr	r3, [pc, #12]	; (80017a0 <_ZN8touchgfx9PartitionINS_4meta8TypeListI16Screen1PresenterNS2_INS1_3NilES4_EEEELt1EED1Ev+0x10>)
 8001794:	6003      	str	r3, [r0, #0]
 8001796:	4604      	mov	r4, r0
 8001798:	f007 fcd0 	bl	800913c <_ZN8touchgfx17AbstractPartitionD1Ev>
 800179c:	4620      	mov	r0, r4
 800179e:	bd10      	pop	{r4, pc}
 80017a0:	0801eaa0 	.word	0x0801eaa0

080017a4 <_ZN8touchgfx9PartitionINS_4meta8TypeListI16Screen1PresenterNS2_INS1_3NilES4_EEEELt1EED0Ev>:
 80017a4:	b510      	push	{r4, lr}
 80017a6:	4604      	mov	r4, r0
 80017a8:	f7ff fff2 	bl	8001790 <_ZN8touchgfx9PartitionINS_4meta8TypeListI16Screen1PresenterNS2_INS1_3NilES4_EEEELt1EED1Ev>
 80017ac:	4620      	mov	r0, r4
 80017ae:	2118      	movs	r1, #24
 80017b0:	f01a f90b 	bl	801b9ca <_ZdlPvj>
 80017b4:	4620      	mov	r0, r4
 80017b6:	bd10      	pop	{r4, pc}

080017b8 <_ZN12FrontendHeapD1Ev>:
#ifndef FRONTENDHEAP_HPP
#define FRONTENDHEAP_HPP

#include <gui_generated/common/FrontendHeapBase.hpp>

class FrontendHeap : public FrontendHeapBase
 80017b8:	b510      	push	{r4, lr}
 80017ba:	4b08      	ldr	r3, [pc, #32]	; (80017dc <_ZN12FrontendHeapD1Ev+0x24>)
 80017bc:	6003      	str	r3, [r0, #0]
 80017be:	4604      	mov	r4, r0
 80017c0:	f500 70d4 	add.w	r0, r0, #424	; 0x1a8
 80017c4:	f7ff ffba 	bl	800173c <_ZN8touchgfx9PartitionINS_4meta8TypeListINS_12NoTransitionENS2_INS1_3NilES4_EEEELt1EED1Ev>
 80017c8:	f104 002c 	add.w	r0, r4, #44	; 0x2c
 80017cc:	f7ff ffca 	bl	8001764 <_ZN8touchgfx9PartitionINS_4meta8TypeListI11Screen1ViewNS2_INS1_3NilES4_EEEELt1EED1Ev>
 80017d0:	f104 0014 	add.w	r0, r4, #20
 80017d4:	f7ff ffdc 	bl	8001790 <_ZN8touchgfx9PartitionINS_4meta8TypeListI16Screen1PresenterNS2_INS1_3NilES4_EEEELt1EED1Ev>
 80017d8:	4620      	mov	r0, r4
 80017da:	bd10      	pop	{r4, pc}
 80017dc:	0801eb3c 	.word	0x0801eb3c

080017e0 <__tcf_0>:
                            > > CombinedTransitionTypes;
    typedef touchgfx::meta::select_type_maxsize< CombinedTransitionTypes >::type MaxTransitionType;

    static FrontendHeap& getInstance()
    {
        static FrontendHeap instance;
 80017e0:	b508      	push	{r3, lr}
 80017e2:	4802      	ldr	r0, [pc, #8]	; (80017ec <__tcf_0+0xc>)
 80017e4:	f7ff ffe8 	bl	80017b8 <_ZN12FrontendHeapD1Ev>
 80017e8:	bd08      	pop	{r3, pc}
 80017ea:	bf00      	nop
 80017ec:	20000308 	.word	0x20000308

080017f0 <_ZN12FrontendHeapD0Ev>:
class FrontendHeap : public FrontendHeapBase
 80017f0:	b510      	push	{r4, lr}
 80017f2:	4604      	mov	r4, r0
 80017f4:	f7ff ffe0 	bl	80017b8 <_ZN12FrontendHeapD1Ev>
 80017f8:	4620      	mov	r0, r4
 80017fa:	f44f 7146 	mov.w	r1, #792	; 0x318
 80017fe:	f01a f8e4 	bl	801b9ca <_ZdlPvj>
 8001802:	4620      	mov	r0, r4
 8001804:	bd10      	pop	{r4, pc}
	...

08001808 <touchgfx_init>:
static ApplicationFontProvider fontProvider;
static Texts texts;
static TouchGFXHAL hal(dma, display, tc, 240, 320);

void touchgfx_init()
{
 8001808:	e92d 41f3 	stmdb	sp!, {r0, r1, r4, r5, r6, r7, r8, lr}
    Bitmap::registerBitmapDatabase(BitmapDatabase::getInstance(), BitmapDatabase::getInstanceSize());
 800180c:	f001 fcb2 	bl	8003174 <_ZN14BitmapDatabase11getInstanceEv>
 8001810:	4605      	mov	r5, r0
 8001812:	f001 fcb3 	bl	800317c <_ZN14BitmapDatabase15getInstanceSizeEv>
 8001816:	2400      	movs	r4, #0
 8001818:	4601      	mov	r1, r0
 800181a:	4623      	mov	r3, r4
 800181c:	4628      	mov	r0, r5
 800181e:	4622      	mov	r2, r4
 8001820:	9400      	str	r4, [sp, #0]
 8001822:	f00e fa1f 	bl	800fc64 <_ZN8touchgfx6Bitmap22registerBitmapDatabaseEPKNS0_10BitmapDataEtPtmm>
     *
     * @param  t The array of texts.
     */
    static void registerTexts(const Texts* t)
    {
        texts = t;
 8001826:	4b25      	ldr	r3, [pc, #148]	; (80018bc <touchgfx_init+0xb4>)
 8001828:	4a25      	ldr	r2, [pc, #148]	; (80018c0 <touchgfx_init+0xb8>)
        static FrontendHeap instance;
 800182a:	4d26      	ldr	r5, [pc, #152]	; (80018c4 <touchgfx_init+0xbc>)
 800182c:	601a      	str	r2, [r3, #0]
    TypedText::registerTexts(&texts);
    Texts::setLanguage(0);
 800182e:	4620      	mov	r0, r4
 8001830:	f002 f9be 	bl	8003bb0 <_ZN8touchgfx5Texts11setLanguageEt>

    FontManager::setFontProvider(&fontProvider);
 8001834:	4824      	ldr	r0, [pc, #144]	; (80018c8 <touchgfx_init+0xc0>)
 8001836:	f00e f957 	bl	800fae8 <_ZN8touchgfx11FontManager15setFontProviderEPNS_12FontProviderE>
 800183a:	782b      	ldrb	r3, [r5, #0]
 800183c:	f3bf 8f5b 	dmb	ish
 8001840:	07db      	lsls	r3, r3, #31
 8001842:	d435      	bmi.n	80018b0 <touchgfx_init+0xa8>
 8001844:	4628      	mov	r0, r5
 8001846:	f01a f8c2 	bl	801b9ce <__cxa_guard_acquire>
 800184a:	b388      	cbz	r0, 80018b0 <touchgfx_init+0xa8>
            AbstractPartition& tra,
            MVPApplication& app)
        : presenterStorage(pres),
          screenStorage(scr),
          transitionStorage(tra),
          frontendApplication(app)
 800184c:	4c1f      	ldr	r4, [pc, #124]	; (80018cc <touchgfx_init+0xc4>)
    Model model;
    FrontendApplication app;

private:
    FrontendHeap() : FrontendHeapBase(presenters, views, transitions, app),
                     app(model, *this)
 800184e:	4b20      	ldr	r3, [pc, #128]	; (80018d0 <touchgfx_init+0xc8>)
 8001850:	6023      	str	r3, [r4, #0]
 8001852:	f504 76e0 	add.w	r6, r4, #448	; 0x1c0
 8001856:	f104 0014 	add.w	r0, r4, #20
 800185a:	f104 082c 	add.w	r8, r4, #44	; 0x2c
 800185e:	f504 77d4 	add.w	r7, r4, #424	; 0x1a8
 8001862:	6060      	str	r0, [r4, #4]
 8001864:	f8c4 8008 	str.w	r8, [r4, #8]
 8001868:	60e7      	str	r7, [r4, #12]
 800186a:	6126      	str	r6, [r4, #16]
 800186c:	f007 fc68 	bl	8009140 <_ZN8touchgfx17AbstractPartitionC1Ev>
 8001870:	4b18      	ldr	r3, [pc, #96]	; (80018d4 <touchgfx_init+0xcc>)
 8001872:	6163      	str	r3, [r4, #20]
 8001874:	4640      	mov	r0, r8
 8001876:	f007 fc63 	bl	8009140 <_ZN8touchgfx17AbstractPartitionC1Ev>
 800187a:	4b17      	ldr	r3, [pc, #92]	; (80018d8 <touchgfx_init+0xd0>)
 800187c:	62e3      	str	r3, [r4, #44]	; 0x2c
 800187e:	4638      	mov	r0, r7
 8001880:	f007 fc5e 	bl	8009140 <_ZN8touchgfx17AbstractPartitionC1Ev>
 8001884:	4b15      	ldr	r3, [pc, #84]	; (80018dc <touchgfx_init+0xd4>)
 8001886:	f8c4 31a8 	str.w	r3, [r4, #424]	; 0x1a8
 800188a:	f504 70de 	add.w	r0, r4, #444	; 0x1bc
 800188e:	f002 fa0b 	bl	8003ca8 <_ZN5ModelC1Ev>
 8001892:	4622      	mov	r2, r4
 8001894:	f504 71de 	add.w	r1, r4, #444	; 0x1bc
 8001898:	4630      	mov	r0, r6
 800189a:	f002 f9fb 	bl	8003c94 <_ZN19FrontendApplicationC1ER5ModelR12FrontendHeap>
 800189e:	4630      	mov	r0, r6
 80018a0:	f001 fdce 	bl	8003440 <_ZN23FrontendApplicationBase29gotoScreen1ScreenNoTransitionEv>
        static FrontendHeap instance;
 80018a4:	480e      	ldr	r0, [pc, #56]	; (80018e0 <touchgfx_init+0xd8>)
 80018a6:	f01a f8dd 	bl	801ba64 <atexit>
 80018aa:	4628      	mov	r0, r5
 80018ac:	f01a f89b 	bl	801b9e6 <__cxa_guard_release>
    (void)heap;

    /*
     * Initialize TouchGFX
     */
    hal.initialize();
 80018b0:	480c      	ldr	r0, [pc, #48]	; (80018e4 <touchgfx_init+0xdc>)
}
 80018b2:	b002      	add	sp, #8
 80018b4:	e8bd 41f0 	ldmia.w	sp!, {r4, r5, r6, r7, r8, lr}
    hal.initialize();
 80018b8:	f7ff bc58 	b.w	800116c <_ZN11TouchGFXHAL10initializeEv>
 80018bc:	2001268c 	.word	0x2001268c
 80018c0:	200012c0 	.word	0x200012c0
 80018c4:	20000304 	.word	0x20000304
 80018c8:	20000008 	.word	0x20000008
 80018cc:	20000308 	.word	0x20000308
 80018d0:	0801eb3c 	.word	0x0801eb3c
 80018d4:	0801eaa0 	.word	0x0801eaa0
 80018d8:	0801ead4 	.word	0x0801ead4
 80018dc:	0801eb08 	.word	0x0801eb08
 80018e0:	080017e1 	.word	0x080017e1
 80018e4:	20001244 	.word	0x20001244

080018e8 <touchgfx_taskEntry>:
     * Main event loop. Will wait for VSYNC signal, and then process next frame. Call
     * this function from your GUI task.
     *
     * Note This function never returns
     */
    hal.taskEntry();
 80018e8:	4801      	ldr	r0, [pc, #4]	; (80018f0 <touchgfx_taskEntry+0x8>)
 80018ea:	f7ff bc51 	b.w	8001190 <_ZN11TouchGFXHAL9taskEntryEv>
 80018ee:	bf00      	nop
 80018f0:	20001244 	.word	0x20001244

080018f4 <_GLOBAL__sub_I_touchgfx_init>:
}
 80018f4:	b570      	push	{r4, r5, r6, lr}
{
public:

    STM32TouchController() {}
 80018f6:	4c23      	ldr	r4, [pc, #140]	; (8001984 <_GLOBAL__sub_I_touchgfx_init+0x90>)
static STM32F4DMA dma;
 80018f8:	4e23      	ldr	r6, [pc, #140]	; (8001988 <_GLOBAL__sub_I_touchgfx_init+0x94>)
 80018fa:	4b24      	ldr	r3, [pc, #144]	; (800198c <_GLOBAL__sub_I_touchgfx_init+0x98>)
static LCD16bpp display;
 80018fc:	4d24      	ldr	r5, [pc, #144]	; (8001990 <_GLOBAL__sub_I_touchgfx_init+0x9c>)
 80018fe:	6023      	str	r3, [r4, #0]
static STM32F4DMA dma;
 8001900:	4630      	mov	r0, r6
 8001902:	f7ff fd93 	bl	800142c <_ZN10STM32F4DMAC1Ev>
static LCD16bpp display;
 8001906:	4628      	mov	r0, r5
 8001908:	f011 fa30 	bl	8012d6c <_ZN8touchgfx8LCD16bppC1Ev>
        instance = this;
 800190c:	4821      	ldr	r0, [pc, #132]	; (8001994 <_GLOBAL__sub_I_touchgfx_init+0xa0>)
          lastRenderMethod(HARDWARE)
 800190e:	4b22      	ldr	r3, [pc, #136]	; (8001998 <_GLOBAL__sub_I_touchgfx_init+0xa4>)
        instance = this;
 8001910:	6003      	str	r3, [r0, #0]
          lastRenderMethod(HARDWARE)
 8001912:	2200      	movs	r2, #0
        DISPLAY_WIDTH = width;
 8001914:	4821      	ldr	r0, [pc, #132]	; (800199c <_GLOBAL__sub_I_touchgfx_init+0xa8>)
          lastRenderMethod(HARDWARE)
 8001916:	60dc      	str	r4, [r3, #12]
 8001918:	f44f 7180 	mov.w	r1, #256	; 0x100
 800191c:	e9c3 1212 	strd	r1, r2, [r3, #72]	; 0x48
 8001920:	e9c3 6501 	strd	r6, r5, [r3, #4]
 8001924:	491e      	ldr	r1, [pc, #120]	; (80019a0 <_GLOBAL__sub_I_touchgfx_init+0xac>)
        DISPLAY_HEIGHT = height;
 8001926:	4d1f      	ldr	r5, [pc, #124]	; (80019a4 <_GLOBAL__sub_I_touchgfx_init+0xb0>)
    };

public:
    /** Default constructor. Does nothing. */
    Gestures()
        : drag(), listener(0), dragThresholdValue(0)
 8001928:	861a      	strh	r2, [r3, #48]	; 0x30
        DISPLAY_WIDTH = width;
 800192a:	24f0      	movs	r4, #240	; 0xf0
 800192c:	8004      	strh	r4, [r0, #0]
        DISPLAY_HEIGHT = height;
 800192e:	f44f 70a0 	mov.w	r0, #320	; 0x140
          lastRenderMethod(HARDWARE)
 8001932:	e9c3 1219 	strd	r1, r2, [r3, #100]	; 0x64
        DISPLAY_HEIGHT = height;
 8001936:	8028      	strh	r0, [r5, #0]
          lastRenderMethod(HARDWARE)
 8001938:	f04f 7180 	mov.w	r1, #16777216	; 0x1000000
        DISPLAY_ROTATION = rotate0;
 800193c:	4d1a      	ldr	r5, [pc, #104]	; (80019a8 <_GLOBAL__sub_I_touchgfx_init+0xb4>)
          lastRenderMethod(HARDWARE)
 800193e:	6759      	str	r1, [r3, #116]	; 0x74
 8001940:	2101      	movs	r1, #1
 8001942:	e9c3 2204 	strd	r2, r2, [r3, #16]
 8001946:	e9c3 2206 	strd	r2, r2, [r3, #24]
 800194a:	e9c3 2208 	strd	r2, r2, [r3, #32]
 800194e:	e9c3 220a 	strd	r2, r2, [r3, #40]	; 0x28
 8001952:	e9c3 220e 	strd	r2, r2, [r3, #56]	; 0x38
 8001956:	e9c3 2210 	strd	r2, r2, [r3, #64]	; 0x40
class Rect
{
public:
    /** Default constructor. Resulting in an empty Rect with coordinates 0,0. */
    Rect()
        : x(0), y(0), width(0), height(0)
 800195a:	e9c3 2214 	strd	r2, r2, [r3, #80]	; 0x50
 800195e:	e9c3 2216 	strd	r2, r2, [r3, #88]	; 0x58
 8001962:	661a      	str	r2, [r3, #96]	; 0x60
 8001964:	f883 206c 	strb.w	r2, [r3, #108]	; 0x6c
 8001968:	671a      	str	r2, [r3, #112]	; 0x70
 800196a:	f883 1078 	strb.w	r1, [r3, #120]	; 0x78
        DISPLAY_ROTATION = rotate0;
 800196e:	702a      	strb	r2, [r5, #0]
        FRAME_BUFFER_WIDTH = DISPLAY_WIDTH;
 8001970:	4a0e      	ldr	r2, [pc, #56]	; (80019ac <_GLOBAL__sub_I_touchgfx_init+0xb8>)
        nativeDisplayOrientation = ((width >= height) ? ORIENTATION_LANDSCAPE : ORIENTATION_PORTRAIT);
 8001972:	f883 1034 	strb.w	r1, [r3, #52]	; 0x34
        FRAME_BUFFER_WIDTH = DISPLAY_WIDTH;
 8001976:	8014      	strh	r4, [r2, #0]
        FRAME_BUFFER_HEIGHT = DISPLAY_HEIGHT;
 8001978:	4a0d      	ldr	r2, [pc, #52]	; (80019b0 <_GLOBAL__sub_I_touchgfx_init+0xbc>)
 800197a:	8010      	strh	r0, [r2, #0]
     * @param [in,out] display Reference to LCD interface.
     * @param [in,out] tc      Reference to Touch Controller driver.
     * @param width            Width of the display.
     * @param height           Height of the display.
     */
    TouchGFXHAL(touchgfx::DMA_Interface& dma, touchgfx::LCD& display, touchgfx::TouchController& tc, uint16_t width, uint16_t height) : TouchGFXGeneratedHAL(dma, display, tc, width, height)
 800197c:	4a0d      	ldr	r2, [pc, #52]	; (80019b4 <_GLOBAL__sub_I_touchgfx_init+0xc0>)
 800197e:	601a      	str	r2, [r3, #0]
}
 8001980:	bd70      	pop	{r4, r5, r6, pc}
 8001982:	bf00      	nop
 8001984:	20000620 	.word	0x20000620
 8001988:	20000624 	.word	0x20000624
 800198c:	0801e638 	.word	0x0801e638
 8001990:	200012c4 	.word	0x200012c4
 8001994:	20012630 	.word	0x20012630
 8001998:	20001244 	.word	0x20001244
 800199c:	20012624 	.word	0x20012624
 80019a0:	01000001 	.word	0x01000001
 80019a4:	20012626 	.word	0x20012626
 80019a8:	20012628 	.word	0x20012628
 80019ac:	2001262a 	.word	0x2001262a
 80019b0:	2001262c 	.word	0x2001262c
 80019b4:	0801e71c 	.word	0x0801e71c

080019b8 <_GLOBAL__sub_D_touchgfx_init>:
static STM32F4DMA dma;
 80019b8:	4801      	ldr	r0, [pc, #4]	; (80019c0 <_GLOBAL__sub_D_touchgfx_init+0x8>)
 80019ba:	f7ff bd13 	b.w	80013e4 <_ZN10STM32F4DMAD1Ev>
 80019be:	bf00      	nop
 80019c0:	20000624 	.word	0x20000624

080019c4 <_ZN20TouchGFXGeneratedHAL19configureInterruptsEv>:
 */
__STATIC_INLINE void __NVIC_SetPriority(IRQn_Type IRQn, uint32_t priority)
{
  if ((int32_t)(IRQn) >= 0)
  {
    NVIC->IP[((uint32_t)IRQn)]               = (uint8_t)((priority << (8U - __NVIC_PRIO_BITS)) & (uint32_t)0xFFUL);
 80019c4:	4b03      	ldr	r3, [pc, #12]	; (80019d4 <_ZN20TouchGFXGeneratedHAL19configureInterruptsEv+0x10>)
 80019c6:	2290      	movs	r2, #144	; 0x90
 80019c8:	f883 235a 	strb.w	r2, [r3, #858]	; 0x35a
 80019cc:	f883 2358 	strb.w	r2, [r3, #856]	; 0x358

void TouchGFXGeneratedHAL::configureInterrupts()
{
    NVIC_SetPriority(DMA2D_IRQn, 9);
    NVIC_SetPriority(LTDC_IRQn, 9);
}
 80019d0:	4770      	bx	lr
 80019d2:	bf00      	nop
 80019d4:	e000e100 	.word	0xe000e100

080019d8 <_ZN20TouchGFXGeneratedHAL28enableLCDControllerInterruptEv>:
    NVIC_DisableIRQ(LTDC_IRQn);
}

void TouchGFXGeneratedHAL::enableLCDControllerInterrupt()
{
    lcd_int_active_line = (LTDC->BPCR & 0x7FF) - 1;
 80019d8:	4a09      	ldr	r2, [pc, #36]	; (8001a00 <_ZN20TouchGFXGeneratedHAL28enableLCDControllerInterruptEv+0x28>)
 80019da:	490a      	ldr	r1, [pc, #40]	; (8001a04 <_ZN20TouchGFXGeneratedHAL28enableLCDControllerInterruptEv+0x2c>)
 80019dc:	68d3      	ldr	r3, [r2, #12]
    lcd_int_porch_line = (LTDC->AWCR & 0x7FF) - 1;
 80019de:	480a      	ldr	r0, [pc, #40]	; (8001a08 <_ZN20TouchGFXGeneratedHAL28enableLCDControllerInterruptEv+0x30>)
    lcd_int_active_line = (LTDC->BPCR & 0x7FF) - 1;
 80019e0:	f3c3 030a 	ubfx	r3, r3, #0, #11
 80019e4:	3b01      	subs	r3, #1
 80019e6:	b29b      	uxth	r3, r3
 80019e8:	800b      	strh	r3, [r1, #0]
    lcd_int_porch_line = (LTDC->AWCR & 0x7FF) - 1;
 80019ea:	6911      	ldr	r1, [r2, #16]
 80019ec:	f3c1 010a 	ubfx	r1, r1, #0, #11
 80019f0:	3901      	subs	r1, #1
 80019f2:	8001      	strh	r1, [r0, #0]

    /* Sets the Line Interrupt position */
    LTDC->LIPCR = lcd_int_active_line;
 80019f4:	6413      	str	r3, [r2, #64]	; 0x40
    /* Line Interrupt Enable            */
    LTDC->IER |= LTDC_IER_LIE;
 80019f6:	6b53      	ldr	r3, [r2, #52]	; 0x34
 80019f8:	f043 0301 	orr.w	r3, r3, #1
 80019fc:	6353      	str	r3, [r2, #52]	; 0x34
}
 80019fe:	4770      	bx	lr
 8001a00:	40016800 	.word	0x40016800
 8001a04:	2000133e 	.word	0x2000133e
 8001a08:	2000133c 	.word	0x2000133c

08001a0c <_ZNK20TouchGFXGeneratedHAL17getTFTFrameBufferEv>:
    HAL::endFrame();
}

uint16_t* TouchGFXGeneratedHAL::getTFTFrameBuffer() const
{
    return (uint16_t*)LTDC_Layer1->CFBAR;
 8001a0c:	4b01      	ldr	r3, [pc, #4]	; (8001a14 <_ZNK20TouchGFXGeneratedHAL17getTFTFrameBufferEv+0x8>)
 8001a0e:	f8d3 00ac 	ldr.w	r0, [r3, #172]	; 0xac
}
 8001a12:	4770      	bx	lr
 8001a14:	40016800 	.word	0x40016800

08001a18 <_ZN20TouchGFXGeneratedHAL17setTFTFrameBufferEPt>:

void TouchGFXGeneratedHAL::setTFTFrameBuffer(uint16_t* adr)
{
    LTDC_Layer1->CFBAR = (uint32_t)adr;
 8001a18:	4b02      	ldr	r3, [pc, #8]	; (8001a24 <_ZN20TouchGFXGeneratedHAL17setTFTFrameBufferEPt+0xc>)

    /* Reload immediate */
    LTDC->SRCR = (uint32_t)LTDC_SRCR_IMR;
 8001a1a:	2201      	movs	r2, #1
    LTDC_Layer1->CFBAR = (uint32_t)adr;
 8001a1c:	f8c3 10ac 	str.w	r1, [r3, #172]	; 0xac
    LTDC->SRCR = (uint32_t)LTDC_SRCR_IMR;
 8001a20:	625a      	str	r2, [r3, #36]	; 0x24
}
 8001a22:	4770      	bx	lr
 8001a24:	40016800 	.word	0x40016800

08001a28 <_ZN20TouchGFXGeneratedHAL10initializeEv>:
{
 8001a28:	b570      	push	{r4, r5, r6, lr}
 8001a2a:	4604      	mov	r4, r0
    HAL::initialize();
 8001a2c:	f007 fdc3 	bl	80095b6 <_ZN8touchgfx3HAL10initializeEv>
    registerEventListener(*(Application::getInstance()));
 8001a30:	6823      	ldr	r3, [r4, #0]
 8001a32:	6ddd      	ldr	r5, [r3, #92]	; 0x5c
 8001a34:	f00a ff1a 	bl	800c86c <_ZN8touchgfx11Application11getInstanceEv>
 8001a38:	4601      	mov	r1, r0
 8001a3a:	4620      	mov	r0, r4
 8001a3c:	47a8      	blx	r5
    setFrameBufferStartAddresses((void*)frameBuf, (void*)(frameBuf + sizeof(frameBuf) / (sizeof(uint32_t) * 2)), (void*)0);
 8001a3e:	6823      	ldr	r3, [r4, #0]
 8001a40:	4a05      	ldr	r2, [pc, #20]	; (8001a58 <_ZN20TouchGFXGeneratedHAL10initializeEv+0x30>)
 8001a42:	f8d3 5080 	ldr.w	r5, [r3, #128]	; 0x80
 8001a46:	4620      	mov	r0, r4
 8001a48:	46ac      	mov	ip, r5
 8001a4a:	2300      	movs	r3, #0
}
 8001a4c:	e8bd 4070 	ldmia.w	sp!, {r4, r5, r6, lr}
    setFrameBufferStartAddresses((void*)frameBuf, (void*)(frameBuf + sizeof(frameBuf) / (sizeof(uint32_t) * 2)), (void*)0);
 8001a50:	f5a2 3116 	sub.w	r1, r2, #153600	; 0x25800
 8001a54:	4760      	bx	ip
 8001a56:	bf00      	nop
 8001a58:	d004b000 	.word	0xd004b000

08001a5c <_ZN20TouchGFXGeneratedHAL10beginFrameEv>:
    return HAL::beginFrame();
 8001a5c:	f007 bd92 	b.w	8009584 <_ZN8touchgfx3HAL10beginFrameEv>

08001a60 <_ZN20TouchGFXGeneratedHAL8endFrameEv>:
    HAL::endFrame();
 8001a60:	f007 bd9c 	b.w	800959c <_ZN8touchgfx3HAL8endFrameEv>

08001a64 <_ZN20TouchGFXGeneratedHAL16flushFrameBufferERKN8touchgfx4RectE>:

void TouchGFXGeneratedHAL::flushFrameBuffer(const touchgfx::Rect& rect)
{
    HAL::flushFrameBuffer(rect);
 8001a64:	f007 bd5a 	b.w	800951c <_ZN8touchgfx3HAL16flushFrameBufferERKNS_4RectE>

08001a68 <_ZN20TouchGFXGeneratedHAL9blockCopyEPvPKvm>:
}

bool TouchGFXGeneratedHAL::blockCopy(void* RESTRICT dest, const void* RESTRICT src, uint32_t numBytes)
{
    return HAL::blockCopy(dest, src, numBytes);
 8001a68:	f007 beb3 	b.w	80097d2 <_ZN8touchgfx3HAL9blockCopyEPvPKvm>

08001a6c <_ZN20TouchGFXGeneratedHAL16enableInterruptsEv>:
    NVIC->ISER[(((uint32_t)IRQn) >> 5UL)] = (uint32_t)(1UL << (((uint32_t)IRQn) & 0x1FUL));
 8001a6c:	4b03      	ldr	r3, [pc, #12]	; (8001a7c <_ZN20TouchGFXGeneratedHAL16enableInterruptsEv+0x10>)
 8001a6e:	f04f 6280 	mov.w	r2, #67108864	; 0x4000000
 8001a72:	609a      	str	r2, [r3, #8]
 8001a74:	f04f 7280 	mov.w	r2, #16777216	; 0x1000000
 8001a78:	609a      	str	r2, [r3, #8]
}
 8001a7a:	4770      	bx	lr
 8001a7c:	e000e100 	.word	0xe000e100

08001a80 <_ZN20TouchGFXGeneratedHAL17disableInterruptsEv>:
    NVIC->ICER[(((uint32_t)IRQn) >> 5UL)] = (uint32_t)(1UL << (((uint32_t)IRQn) & 0x1FUL));
 8001a80:	4b08      	ldr	r3, [pc, #32]	; (8001aa4 <_ZN20TouchGFXGeneratedHAL17disableInterruptsEv+0x24>)
 8001a82:	f04f 6280 	mov.w	r2, #67108864	; 0x4000000
 8001a86:	f8c3 2088 	str.w	r2, [r3, #136]	; 0x88
  __ASM volatile ("dsb 0xF":::"memory");
 8001a8a:	f3bf 8f4f 	dsb	sy
  __ASM volatile ("isb 0xF":::"memory");
 8001a8e:	f3bf 8f6f 	isb	sy
 8001a92:	f04f 7280 	mov.w	r2, #16777216	; 0x1000000
 8001a96:	f8c3 2088 	str.w	r2, [r3, #136]	; 0x88
  __ASM volatile ("dsb 0xF":::"memory");
 8001a9a:	f3bf 8f4f 	dsb	sy
  __ASM volatile ("isb 0xF":::"memory");
 8001a9e:	f3bf 8f6f 	isb	sy
}
 8001aa2:	4770      	bx	lr
 8001aa4:	e000e100 	.word	0xe000e100

08001aa8 <HAL_LTDC_LineEventCallback>:

extern "C"
{
    void HAL_LTDC_LineEventCallback(LTDC_HandleTypeDef* hltdc)
    {
        if (LTDC->LIPCR == lcd_int_active_line)
 8001aa8:	4b13      	ldr	r3, [pc, #76]	; (8001af8 <HAL_LTDC_LineEventCallback+0x50>)
 8001aaa:	4a14      	ldr	r2, [pc, #80]	; (8001afc <HAL_LTDC_LineEventCallback+0x54>)
 8001aac:	6c1b      	ldr	r3, [r3, #64]	; 0x40
 8001aae:	8811      	ldrh	r1, [r2, #0]
 8001ab0:	428b      	cmp	r3, r1
    {
 8001ab2:	b510      	push	{r4, lr}
 8001ab4:	4c12      	ldr	r4, [pc, #72]	; (8001b00 <HAL_LTDC_LineEventCallback+0x58>)
        if (LTDC->LIPCR == lcd_int_active_line)
 8001ab6:	d113      	bne.n	8001ae0 <HAL_LTDC_LineEventCallback+0x38>
        {
            //entering active area
            HAL_LTDC_ProgramLineEvent(hltdc, lcd_int_porch_line);
 8001ab8:	4b12      	ldr	r3, [pc, #72]	; (8001b04 <HAL_LTDC_LineEventCallback+0x5c>)
 8001aba:	8819      	ldrh	r1, [r3, #0]
 8001abc:	f003 fd16 	bl	80054ec <HAL_LTDC_ProgramLineEvent>
        return instance;
 8001ac0:	6822      	ldr	r2, [r4, #0]
        vSyncCnt++;
 8001ac2:	f892 3066 	ldrb.w	r3, [r2, #102]	; 0x66
 8001ac6:	3301      	adds	r3, #1
 8001ac8:	f882 3066 	strb.w	r3, [r2, #102]	; 0x66
            HAL::getInstance()->vSync();
            OSWrappers::signalVSync();
 8001acc:	f7ff fc36 	bl	800133c <_ZN8touchgfx10OSWrappers11signalVSyncEv>
            // Swap frame buffers immediately instead of waiting for the task to be scheduled in.
            // Note: task will also swap when it wakes up, but that operation is guarded and will not have
            // any effect if already swapped.
            HAL::getInstance()->swapFrameBuffers();
 8001ad0:	6820      	ldr	r0, [r4, #0]
 8001ad2:	f008 fb65 	bl	800a1a0 <_ZN8touchgfx3HAL16swapFrameBuffersEv>
            //exiting active area
            HAL_LTDC_ProgramLineEvent(hltdc, lcd_int_active_line);
            GPIO::clear(GPIO::VSYNC_FREQ);
            HAL::getInstance()->frontPorchEntered();
        }
    }
 8001ad6:	e8bd 4010 	ldmia.w	sp!, {r4, lr}
            GPIO::set(GPIO::VSYNC_FREQ);
 8001ada:	2000      	movs	r0, #0
 8001adc:	f7ff bb2a 	b.w	8001134 <_ZN8touchgfx4GPIO3setENS0_7GPIO_IDE>
            HAL_LTDC_ProgramLineEvent(hltdc, lcd_int_active_line);
 8001ae0:	f003 fd04 	bl	80054ec <HAL_LTDC_ProgramLineEvent>
            GPIO::clear(GPIO::VSYNC_FREQ);
 8001ae4:	2000      	movs	r0, #0
 8001ae6:	f7ff fb26 	bl	8001136 <_ZN8touchgfx4GPIO5clearENS0_7GPIO_IDE>
        return instance;
 8001aea:	6820      	ldr	r0, [r4, #0]
        allowDMATransfers();
 8001aec:	6803      	ldr	r3, [r0, #0]
    }
 8001aee:	e8bd 4010 	ldmia.w	sp!, {r4, lr}
 8001af2:	69db      	ldr	r3, [r3, #28]
 8001af4:	4718      	bx	r3
 8001af6:	bf00      	nop
 8001af8:	40016800 	.word	0x40016800
 8001afc:	2000133e 	.word	0x2000133e
 8001b00:	20012630 	.word	0x20012630
 8001b04:	2000133c 	.word	0x2000133c

08001b08 <bmp_write_register>:
{
	bmp_280_get_temperature();
	bmp_280_get_pressure();
}

HAL_StatusTypeDef bmp_write_register(uint8_t sensor_register, uint8_t value){
 8001b08:	b537      	push	{r0, r1, r2, r4, r5, lr}
	HAL_StatusTypeDef ret_val;
	uint8_t data_to_write[2] = {sensor_register&0b01111111, value};
	HAL_GPIO_WritePin(bmp280_driver.SS_port, bmp280_driver.SS_pin, GPIO_PIN_RESET);
 8001b0a:	4c0e      	ldr	r4, [pc, #56]	; (8001b44 <bmp_write_register+0x3c>)
	uint8_t data_to_write[2] = {sensor_register&0b01111111, value};
 8001b0c:	f88d 1005 	strb.w	r1, [sp, #5]
 8001b10:	f000 007f 	and.w	r0, r0, #127	; 0x7f
	HAL_GPIO_WritePin(bmp280_driver.SS_port, bmp280_driver.SS_pin, GPIO_PIN_RESET);
 8001b14:	f8b4 105c 	ldrh.w	r1, [r4, #92]	; 0x5c
	uint8_t data_to_write[2] = {sensor_register&0b01111111, value};
 8001b18:	f88d 0004 	strb.w	r0, [sp, #4]
	HAL_GPIO_WritePin(bmp280_driver.SS_port, bmp280_driver.SS_pin, GPIO_PIN_RESET);
 8001b1c:	2200      	movs	r2, #0
 8001b1e:	6da0      	ldr	r0, [r4, #88]	; 0x58
 8001b20:	f002 ff06 	bl	8004930 <HAL_GPIO_WritePin>
	ret_val=HAL_SPI_Transmit(&bmp280_driver.bmp_280_SPI, data_to_write, 2, 1);
 8001b24:	2301      	movs	r3, #1
 8001b26:	a901      	add	r1, sp, #4
 8001b28:	2202      	movs	r2, #2
 8001b2a:	4620      	mov	r0, r4
 8001b2c:	f004 fa2e 	bl	8005f8c <HAL_SPI_Transmit>
	HAL_GPIO_WritePin(bmp280_driver.SS_port, bmp280_driver.SS_pin, GPIO_PIN_SET);
 8001b30:	f8b4 105c 	ldrh.w	r1, [r4, #92]	; 0x5c
	ret_val=HAL_SPI_Transmit(&bmp280_driver.bmp_280_SPI, data_to_write, 2, 1);
 8001b34:	4605      	mov	r5, r0
	HAL_GPIO_WritePin(bmp280_driver.SS_port, bmp280_driver.SS_pin, GPIO_PIN_SET);
 8001b36:	2201      	movs	r2, #1
 8001b38:	6da0      	ldr	r0, [r4, #88]	; 0x58
 8001b3a:	f002 fef9 	bl	8004930 <HAL_GPIO_WritePin>
	return(ret_val);
}
 8001b3e:	4628      	mov	r0, r5
 8001b40:	b003      	add	sp, #12
 8001b42:	bd30      	pop	{r4, r5, pc}
 8001b44:	20001340 	.word	0x20001340

08001b48 <bmp_280_driver_init>:
{
 8001b48:	b084      	sub	sp, #16
 8001b4a:	b538      	push	{r3, r4, r5, lr}
 8001b4c:	ac04      	add	r4, sp, #16
 8001b4e:	e884 000f 	stmia.w	r4, {r0, r1, r2, r3}
	bmp280_driver.bmp_280_SPI=bmp280_SPI_com;
 8001b52:	4b0b      	ldr	r3, [pc, #44]	; (8001b80 <bmp_280_driver_init+0x38>)
{
 8001b54:	9d1a      	ldr	r5, [sp, #104]	; 0x68
 8001b56:	f8bd 406c 	ldrh.w	r4, [sp, #108]	; 0x6c
	bmp280_driver.bmp_280_SPI=bmp280_SPI_com;
 8001b5a:	a904      	add	r1, sp, #16
 8001b5c:	4618      	mov	r0, r3
 8001b5e:	2258      	movs	r2, #88	; 0x58
 8001b60:	f019 ffe0 	bl	801bb24 <memcpy>
	bmp_write_register(BMP280_REG_ADDR_CTRL_MEAS, 0b00100111); 	//001 min oversampling in T and P for more variation, 11 in LSB is normal mode
 8001b64:	2127      	movs	r1, #39	; 0x27
	bmp280_driver.SS_port=bmp280_SS_port;
 8001b66:	6585      	str	r5, [r0, #88]	; 0x58
	bmp280_driver.SS_pin=bmp280_SS_pin;
 8001b68:	f8a0 405c 	strh.w	r4, [r0, #92]	; 0x5c
	bmp_write_register(BMP280_REG_ADDR_CTRL_MEAS, 0b00100111); 	//001 min oversampling in T and P for more variation, 11 in LSB is normal mode
 8001b6c:	20f4      	movs	r0, #244	; 0xf4
 8001b6e:	f7ff ffcb 	bl	8001b08 <bmp_write_register>
}
 8001b72:	e8bd 4038 	ldmia.w	sp!, {r3, r4, r5, lr}
	bmp_write_register(BMP280_REG_ADDR_CONFIG, 0b10000000);		//100 in MSB is 500ms standby for least 1 sampling per second, 000 IIR for more variation
 8001b76:	2180      	movs	r1, #128	; 0x80
 8001b78:	20f5      	movs	r0, #245	; 0xf5
}
 8001b7a:	b004      	add	sp, #16
	bmp_write_register(BMP280_REG_ADDR_CONFIG, 0b10000000);		//100 in MSB is 500ms standby for least 1 sampling per second, 000 IIR for more variation
 8001b7c:	f7ff bfc4 	b.w	8001b08 <bmp_write_register>
 8001b80:	20001340 	.word	0x20001340

08001b84 <bmp280_read_register>:

HAL_StatusTypeDef bmp280_read_register(uint8_t sensor_register, uint8_t *value){
 8001b84:	b537      	push	{r0, r1, r2, r4, r5, lr}
	HAL_StatusTypeDef ret_val=HAL_ERROR;
	//uint8_t data_to_write[2] = {sensor_register, value};
	HAL_GPIO_WritePin(bmp280_driver.SS_port, bmp280_driver.SS_pin, GPIO_PIN_RESET);
 8001b86:	4c12      	ldr	r4, [pc, #72]	; (8001bd0 <bmp280_read_register+0x4c>)
HAL_StatusTypeDef bmp280_read_register(uint8_t sensor_register, uint8_t *value){
 8001b88:	f88d 0007 	strb.w	r0, [sp, #7]
	HAL_GPIO_WritePin(bmp280_driver.SS_port, bmp280_driver.SS_pin, GPIO_PIN_RESET);
 8001b8c:	2200      	movs	r2, #0
 8001b8e:	6da0      	ldr	r0, [r4, #88]	; 0x58
HAL_StatusTypeDef bmp280_read_register(uint8_t sensor_register, uint8_t *value){
 8001b90:	460d      	mov	r5, r1
	HAL_GPIO_WritePin(bmp280_driver.SS_port, bmp280_driver.SS_pin, GPIO_PIN_RESET);
 8001b92:	f8b4 105c 	ldrh.w	r1, [r4, #92]	; 0x5c
 8001b96:	f002 fecb 	bl	8004930 <HAL_GPIO_WritePin>
	if(HAL_SPI_Transmit(&bmp280_driver.bmp_280_SPI, &sensor_register, 1, 1)==HAL_OK){
 8001b9a:	2301      	movs	r3, #1
 8001b9c:	461a      	mov	r2, r3
 8001b9e:	f10d 0107 	add.w	r1, sp, #7
 8001ba2:	4620      	mov	r0, r4
 8001ba4:	f004 f9f2 	bl	8005f8c <HAL_SPI_Transmit>
 8001ba8:	b978      	cbnz	r0, 8001bca <bmp280_read_register+0x46>
		ret_val=HAL_SPI_Receive(&bmp280_driver.bmp_280_SPI, value, 1, 1);
 8001baa:	2301      	movs	r3, #1
 8001bac:	4629      	mov	r1, r5
 8001bae:	461a      	mov	r2, r3
 8001bb0:	4620      	mov	r0, r4
 8001bb2:	f004 fb8d 	bl	80062d0 <HAL_SPI_Receive>
 8001bb6:	4605      	mov	r5, r0
	}
	HAL_GPIO_WritePin(bmp280_driver.SS_port, bmp280_driver.SS_pin, GPIO_PIN_SET);
 8001bb8:	6da0      	ldr	r0, [r4, #88]	; 0x58
 8001bba:	f8b4 105c 	ldrh.w	r1, [r4, #92]	; 0x5c
 8001bbe:	2201      	movs	r2, #1
 8001bc0:	f002 feb6 	bl	8004930 <HAL_GPIO_WritePin>
	return(ret_val);
}
 8001bc4:	4628      	mov	r0, r5
 8001bc6:	b003      	add	sp, #12
 8001bc8:	bd30      	pop	{r4, r5, pc}
	HAL_StatusTypeDef ret_val=HAL_ERROR;
 8001bca:	2501      	movs	r5, #1
 8001bcc:	e7f4      	b.n	8001bb8 <bmp280_read_register+0x34>
 8001bce:	bf00      	nop
 8001bd0:	20001340 	.word	0x20001340

08001bd4 <bmp280_get_raw_TorP>:

int32_t bmp280_get_raw_TorP(uint8_t *BMPregisters){
	return((int32_t)((BMPregisters[0]<<12)|(BMPregisters[1]<<4)|(BMPregisters[2]>>4)));
 8001bd4:	7843      	ldrb	r3, [r0, #1]
 8001bd6:	7802      	ldrb	r2, [r0, #0]
 8001bd8:	7880      	ldrb	r0, [r0, #2]
 8001bda:	011b      	lsls	r3, r3, #4
 8001bdc:	ea43 3302 	orr.w	r3, r3, r2, lsl #12
}
 8001be0:	ea43 1010 	orr.w	r0, r3, r0, lsr #4
 8001be4:	4770      	bx	lr
	...

08001be8 <bmp280_convert_temperature_to_degrees>:

float bmp280_convert_temperature_to_degrees(int32_t raw_temp){
 8001be8:	b538      	push	{r3, r4, r5, lr}
 8001bea:	ed2d 8b02 	vpush	{d8}
	float var1=0;
	float var2=0;

	var1=(float)((raw_temp)/16384.0-(27504)/1024.0)*(26435);
 8001bee:	f7fe fca9 	bl	8000544 <__aeabi_i2d>
	var2=(float)(raw_temp/131072.0-27504/8192.0);
 8001bf2:	4b1b      	ldr	r3, [pc, #108]	; (8001c60 <bmp280_convert_temperature_to_degrees+0x78>)
 8001bf4:	2200      	movs	r2, #0
	var1=(float)((raw_temp)/16384.0-(27504)/1024.0)*(26435);
 8001bf6:	4604      	mov	r4, r0
 8001bf8:	460d      	mov	r5, r1
	var2=(float)(raw_temp/131072.0-27504/8192.0);
 8001bfa:	f7fe fd0d 	bl	8000618 <__aeabi_dmul>
 8001bfe:	a314      	add	r3, pc, #80	; (adr r3, 8001c50 <bmp280_convert_temperature_to_degrees+0x68>)
 8001c00:	e9d3 2300 	ldrd	r2, r3, [r3]
 8001c04:	f7fe fb50 	bl	80002a8 <__aeabi_dsub>
 8001c08:	f7fe ffde 	bl	8000bc8 <__aeabi_d2f>
 8001c0c:	ee00 0a10 	vmov	s0, r0
	var1=(float)((raw_temp)/16384.0-(27504)/1024.0)*(26435);
 8001c10:	4b14      	ldr	r3, [pc, #80]	; (8001c64 <bmp280_convert_temperature_to_degrees+0x7c>)
 8001c12:	2200      	movs	r2, #0
 8001c14:	4620      	mov	r0, r4
 8001c16:	4629      	mov	r1, r5
	var2=var2*var2;
 8001c18:	ee20 8a00 	vmul.f32	s16, s0, s0
	var1=(float)((raw_temp)/16384.0-(27504)/1024.0)*(26435);
 8001c1c:	f7fe fcfc 	bl	8000618 <__aeabi_dmul>
 8001c20:	a30d      	add	r3, pc, #52	; (adr r3, 8001c58 <bmp280_convert_temperature_to_degrees+0x70>)
 8001c22:	e9d3 2300 	ldrd	r2, r3, [r3]
 8001c26:	f7fe fb3f 	bl	80002a8 <__aeabi_dsub>
 8001c2a:	f7fe ffcd 	bl	8000bc8 <__aeabi_d2f>
	var2=var2*(-1000);
 8001c2e:	ed9f 0a0e 	vldr	s0, [pc, #56]	; 8001c68 <bmp280_convert_temperature_to_degrees+0x80>
	return((float)(var1+var2)/5120.0);
 8001c32:	eddf 7a0e 	vldr	s15, [pc, #56]	; 8001c6c <bmp280_convert_temperature_to_degrees+0x84>
	var2=var2*(-1000);
 8001c36:	ee28 0a00 	vmul.f32	s0, s16, s0
	return((float)(var1+var2)/5120.0);
 8001c3a:	ee07 0a10 	vmov	s14, r0
}
 8001c3e:	ecbd 8b02 	vpop	{d8}
	return((float)(var1+var2)/5120.0);
 8001c42:	eea7 0a27 	vfma.f32	s0, s14, s15
}
 8001c46:	eddf 7a0a 	vldr	s15, [pc, #40]	; 8001c70 <bmp280_convert_temperature_to_degrees+0x88>
 8001c4a:	ee80 0a27 	vdiv.f32	s0, s0, s15
 8001c4e:	bd38      	pop	{r3, r4, r5, pc}
 8001c50:	00000000 	.word	0x00000000
 8001c54:	400adc00 	.word	0x400adc00
 8001c58:	00000000 	.word	0x00000000
 8001c5c:	403adc00 	.word	0x403adc00
 8001c60:	3ee00000 	.word	0x3ee00000
 8001c64:	3f100000 	.word	0x3f100000
 8001c68:	c47a0000 	.word	0xc47a0000
 8001c6c:	46ce8600 	.word	0x46ce8600
 8001c70:	45a00000 	.word	0x45a00000

08001c74 <bmp_280_get_temperature>:
{
 8001c74:	b507      	push	{r0, r1, r2, lr}
	bmp280_read_register(BMP280_REG_ADDR_TEMP_MSB, &dataT[0]);
 8001c76:	20fa      	movs	r0, #250	; 0xfa
 8001c78:	a901      	add	r1, sp, #4
 8001c7a:	f7ff ff83 	bl	8001b84 <bmp280_read_register>
	int32_t rawTemp=bmp280_get_raw_TorP(&dataT[0]);
 8001c7e:	a801      	add	r0, sp, #4
 8001c80:	f7ff ffa8 	bl	8001bd4 <bmp280_get_raw_TorP>
	bmp280_driver.current_temp=bmp280_convert_temperature_to_degrees(rawTemp);
 8001c84:	f7ff ffb0 	bl	8001be8 <bmp280_convert_temperature_to_degrees>
 8001c88:	4b02      	ldr	r3, [pc, #8]	; (8001c94 <bmp_280_get_temperature+0x20>)
 8001c8a:	ed83 0a18 	vstr	s0, [r3, #96]	; 0x60
}
 8001c8e:	b003      	add	sp, #12
 8001c90:	f85d fb04 	ldr.w	pc, [sp], #4
 8001c94:	20001340 	.word	0x20001340

08001c98 <set_float2char>:
uint64_t runtime=0;

/** Function definition ---------------------------------------------------------------------------------------*/

void set_float2char(uint8_t *str, float number)
{
 8001c98:	b513      	push	{r0, r1, r4, lr}
	str[0]=((uint8_t)number/10)+48;
 8001c9a:	eefc 7ac0 	vcvt.u32.f32	s15, s0
 8001c9e:	210a      	movs	r1, #10
 8001ca0:	edcd 7a01 	vstr	s15, [sp, #4]
	str[1]=((uint8_t)number%10)+48;
	str[2]='.';
	str[3]=((uint8_t)(number*10)%10)+48;
 8001ca4:	eef2 7a04 	vmov.f32	s15, #36	; 0x41200000  10.0
 8001ca8:	ee60 7a27 	vmul.f32	s15, s0, s15
	str[0]=((uint8_t)number/10)+48;
 8001cac:	f89d 2004 	ldrb.w	r2, [sp, #4]
 8001cb0:	fbb2 f3f1 	udiv	r3, r2, r1
	str[3]=((uint8_t)(number*10)%10)+48;
 8001cb4:	eefc 7ae7 	vcvt.u32.f32	s15, s15
	str[1]=((uint8_t)number%10)+48;
 8001cb8:	fb01 2213 	mls	r2, r1, r3, r2
	str[3]=((uint8_t)(number*10)%10)+48;
 8001cbc:	edcd 7a01 	vstr	s15, [sp, #4]
	str[4]=((uint8_t)(number*100)%10)+48;
 8001cc0:	eddf 7a10 	vldr	s15, [pc, #64]	; 8001d04 <set_float2char+0x6c>
 8001cc4:	ee20 0a27 	vmul.f32	s0, s0, s15
	str[1]=((uint8_t)number%10)+48;
 8001cc8:	3230      	adds	r2, #48	; 0x30
	str[4]=((uint8_t)(number*100)%10)+48;
 8001cca:	eefc 7ac0 	vcvt.u32.f32	s15, s0
	str[1]=((uint8_t)number%10)+48;
 8001cce:	7042      	strb	r2, [r0, #1]
	str[3]=((uint8_t)(number*10)%10)+48;
 8001cd0:	f89d 2004 	ldrb.w	r2, [sp, #4]
	str[4]=((uint8_t)(number*100)%10)+48;
 8001cd4:	edcd 7a01 	vstr	s15, [sp, #4]
	str[0]=((uint8_t)number/10)+48;
 8001cd8:	f103 0430 	add.w	r4, r3, #48	; 0x30
	str[2]='.';
 8001cdc:	232e      	movs	r3, #46	; 0x2e
 8001cde:	7083      	strb	r3, [r0, #2]
	str[3]=((uint8_t)(number*10)%10)+48;
 8001ce0:	fbb2 f3f1 	udiv	r3, r2, r1
 8001ce4:	fb01 2213 	mls	r2, r1, r3, r2
	str[4]=((uint8_t)(number*100)%10)+48;
 8001ce8:	f89d 3004 	ldrb.w	r3, [sp, #4]
	str[0]=((uint8_t)number/10)+48;
 8001cec:	7004      	strb	r4, [r0, #0]
	str[3]=((uint8_t)(number*10)%10)+48;
 8001cee:	3230      	adds	r2, #48	; 0x30
 8001cf0:	70c2      	strb	r2, [r0, #3]
	str[4]=((uint8_t)(number*100)%10)+48;
 8001cf2:	fbb3 f2f1 	udiv	r2, r3, r1
 8001cf6:	fb01 3312 	mls	r3, r1, r2, r3
 8001cfa:	3330      	adds	r3, #48	; 0x30
 8001cfc:	7103      	strb	r3, [r0, #4]
}
 8001cfe:	b002      	add	sp, #8
 8001d00:	bd10      	pop	{r4, pc}
 8001d02:	bf00      	nop
 8001d04:	42c80000 	.word	0x42c80000

08001d08 <response_temperature>:

void response_temperature(void)
{
 8001d08:	b57f      	push	{r0, r1, r2, r3, r4, r5, r6, lr}
	char response_message[20];
	response_message[0]=PROTOCOL_PREAMBLE;
 8001d0a:	232a      	movs	r3, #42	; 0x2a
 8001d0c:	f88d 3004 	strb.w	r3, [sp, #4]
	response_message[1]=(char)ELEMENT_TEMPERATURE;
 8001d10:	2354      	movs	r3, #84	; 0x54
 8001d12:	f88d 3005 	strb.w	r3, [sp, #5]
	set_float2char(&response_message[2], bmp_280_get_temperature());
 8001d16:	f7ff ffad 	bl	8001c74 <bmp_280_get_temperature>
 8001d1a:	f10d 0006 	add.w	r0, sp, #6
 8001d1e:	f7ff ffbb 	bl	8001c98 <set_float2char>
	response_message[7]=PROTOCOL_POSAMBLE;
 8001d22:	2323      	movs	r3, #35	; 0x23
	uart_driver_send(&uart_driver, (uint8_t *)response_message, 8);
 8001d24:	4804      	ldr	r0, [pc, #16]	; (8001d38 <response_temperature+0x30>)
	response_message[7]=PROTOCOL_POSAMBLE;
 8001d26:	f88d 300b 	strb.w	r3, [sp, #11]
	uart_driver_send(&uart_driver, (uint8_t *)response_message, 8);
 8001d2a:	2208      	movs	r2, #8
 8001d2c:	a901      	add	r1, sp, #4
 8001d2e:	f001 f927 	bl	8002f80 <uart_driver_send>
}
 8001d32:	b007      	add	sp, #28
 8001d34:	f85d fb04 	ldr.w	pc, [sp], #4
 8001d38:	20001768 	.word	0x20001768

08001d3c <get_runtime_seconds>:

uint64_t get_runtime_seconds(void)
{
 8001d3c:	b508      	push	{r3, lr}
	return ((uint64_t)__HAL_TIM_GET_COUNTER(&htim7)+runtime)/10000;
 8001d3e:	4b08      	ldr	r3, [pc, #32]	; (8001d60 <get_runtime_seconds+0x24>)
 8001d40:	4a08      	ldr	r2, [pc, #32]	; (8001d64 <get_runtime_seconds+0x28>)
 8001d42:	681b      	ldr	r3, [r3, #0]
 8001d44:	6a58      	ldr	r0, [r3, #36]	; 0x24
 8001d46:	e9d2 3100 	ldrd	r3, r1, [r2]
 8001d4a:	18c0      	adds	r0, r0, r3
 8001d4c:	f242 7210 	movw	r2, #10000	; 0x2710
 8001d50:	f04f 0300 	mov.w	r3, #0
 8001d54:	f141 0100 	adc.w	r1, r1, #0
 8001d58:	f7fe ff86 	bl	8000c68 <__aeabi_uldivmod>
}
 8001d5c:	bd08      	pop	{r3, pc}
 8001d5e:	bf00      	nop
 8001d60:	200015e8 	.word	0x200015e8
 8001d64:	200013a8 	.word	0x200013a8

08001d68 <get_runtime_DHMS>:

void get_runtime_DHMS(uint8_t *pTime)
{
 8001d68:	b570      	push	{r4, r5, r6, lr}
 8001d6a:	4604      	mov	r4, r0
	uint64_t time_buffer=get_runtime_seconds();
 8001d6c:	f7ff ffe6 	bl	8001d3c <get_runtime_seconds>
	pTime[3]=(uint8_t)(time_buffer%60);
 8001d70:	223c      	movs	r2, #60	; 0x3c
 8001d72:	2300      	movs	r3, #0
	uint64_t time_buffer=get_runtime_seconds();
 8001d74:	4606      	mov	r6, r0
 8001d76:	460d      	mov	r5, r1
	pTime[3]=(uint8_t)(time_buffer%60);
 8001d78:	f7fe ff76 	bl	8000c68 <__aeabi_uldivmod>
	time_buffer=time_buffer/60;
 8001d7c:	2300      	movs	r3, #0
	pTime[3]=(uint8_t)(time_buffer%60);
 8001d7e:	70e2      	strb	r2, [r4, #3]
	time_buffer=time_buffer/60;
 8001d80:	4630      	mov	r0, r6
 8001d82:	223c      	movs	r2, #60	; 0x3c
 8001d84:	4629      	mov	r1, r5
 8001d86:	f7fe ff6f 	bl	8000c68 <__aeabi_uldivmod>
	pTime[2]=(uint8_t)(time_buffer%60);
 8001d8a:	223c      	movs	r2, #60	; 0x3c
 8001d8c:	2300      	movs	r3, #0
	time_buffer=time_buffer/60;
 8001d8e:	4606      	mov	r6, r0
 8001d90:	460d      	mov	r5, r1
	pTime[2]=(uint8_t)(time_buffer%60);
 8001d92:	f7fe ff69 	bl	8000c68 <__aeabi_uldivmod>
	time_buffer=time_buffer/60;
 8001d96:	2300      	movs	r3, #0
	pTime[2]=(uint8_t)(time_buffer%60);
 8001d98:	70a2      	strb	r2, [r4, #2]
	time_buffer=time_buffer/60;
 8001d9a:	4630      	mov	r0, r6
 8001d9c:	223c      	movs	r2, #60	; 0x3c
 8001d9e:	4629      	mov	r1, r5
 8001da0:	f7fe ff62 	bl	8000c68 <__aeabi_uldivmod>
	pTime[1]=(uint8_t)(time_buffer%24);
 8001da4:	2218      	movs	r2, #24
 8001da6:	2300      	movs	r3, #0
	time_buffer=time_buffer/60;
 8001da8:	4606      	mov	r6, r0
 8001daa:	460d      	mov	r5, r1
	pTime[1]=(uint8_t)(time_buffer%24);
 8001dac:	f7fe ff5c 	bl	8000c68 <__aeabi_uldivmod>
	time_buffer=time_buffer/24;
 8001db0:	2300      	movs	r3, #0
	pTime[1]=(uint8_t)(time_buffer%24);
 8001db2:	7062      	strb	r2, [r4, #1]
	time_buffer=time_buffer/24;
 8001db4:	4630      	mov	r0, r6
 8001db6:	2218      	movs	r2, #24
 8001db8:	4629      	mov	r1, r5
 8001dba:	f7fe ff55 	bl	8000c68 <__aeabi_uldivmod>
	pTime[0]=(uint8_t)time_buffer;
 8001dbe:	7020      	strb	r0, [r4, #0]
}
 8001dc0:	bd70      	pop	{r4, r5, r6, pc}
	...

08001dc4 <process_set_command>:

uint8_t process_set_command(rx_packet_t *rx_packet)
{
 8001dc4:	b508      	push	{r3, lr}
	uint8_t ret_val=1;
	switch(rx_packet->element)
 8001dc6:	7843      	ldrb	r3, [r0, #1]
 8001dc8:	2b44      	cmp	r3, #68	; 0x44
 8001dca:	d00c      	beq.n	8001de6 <process_set_command+0x22>
 8001dcc:	2b53      	cmp	r3, #83	; 0x53
 8001dce:	d10f      	bne.n	8001df0 <process_set_command+0x2c>
	{
		case ELEMENT_FAN_SPEED:
			if((rx_packet->value>='0')&&(rx_packet->value<'5'))
 8001dd0:	7883      	ldrb	r3, [r0, #2]
 8001dd2:	3b30      	subs	r3, #48	; 0x30
 8001dd4:	b2da      	uxtb	r2, r3
 8001dd6:	2a04      	cmp	r2, #4
 8001dd8:	d803      	bhi.n	8001de2 <process_set_command+0x1e>
			{
				TIM1->CCR4=(rx_packet->value-48)*25;
 8001dda:	2219      	movs	r2, #25
 8001ddc:	4353      	muls	r3, r2
 8001dde:	4a0a      	ldr	r2, [pc, #40]	; (8001e08 <process_set_command+0x44>)
 8001de0:	6413      	str	r3, [r2, #64]	; 0x40
	uint8_t ret_val=1;
 8001de2:	2001      	movs	r0, #1
 8001de4:	e005      	b.n	8001df2 <process_set_command+0x2e>
 8001de6:	7883      	ldrb	r3, [r0, #2]
			}
			break;
		case ELEMENT_DOOR:
			switch(rx_packet->value)
 8001de8:	2b30      	cmp	r3, #48	; 0x30
 8001dea:	d003      	beq.n	8001df4 <process_set_command+0x30>
 8001dec:	2b31      	cmp	r3, #49	; 0x31
 8001dee:	d008      	beq.n	8001e02 <process_set_command+0x3e>
	switch(rx_packet->element)
 8001df0:	2000      	movs	r0, #0
		default:
			ret_val=0;
			break;
	}
	return ret_val;
}
 8001df2:	bd08      	pop	{r3, pc}
					HAL_GPIO_WritePin(DOOR_GPIO_Port, DOOR_Pin, GPIO_PIN_RESET);
 8001df4:	2200      	movs	r2, #0
					HAL_GPIO_WritePin(DOOR_GPIO_Port, DOOR_Pin, GPIO_PIN_SET);
 8001df6:	4805      	ldr	r0, [pc, #20]	; (8001e0c <process_set_command+0x48>)
 8001df8:	f44f 4180 	mov.w	r1, #16384	; 0x4000
 8001dfc:	f002 fd98 	bl	8004930 <HAL_GPIO_WritePin>
					break;
 8001e00:	e7ef      	b.n	8001de2 <process_set_command+0x1e>
					HAL_GPIO_WritePin(DOOR_GPIO_Port, DOOR_Pin, GPIO_PIN_SET);
 8001e02:	2201      	movs	r2, #1
 8001e04:	e7f7      	b.n	8001df6 <process_set_command+0x32>
 8001e06:	bf00      	nop
 8001e08:	40010000 	.word	0x40010000
 8001e0c:	40021800 	.word	0x40021800

08001e10 <process_get_command>:

uint8_t process_get_command(rx_packet_t *rx_packet)
{
 8001e10:	b510      	push	{r4, lr}
 8001e12:	b086      	sub	sp, #24
 8001e14:	4604      	mov	r4, r0
	uint8_t ret_val=1;
	char response_message[20];
	memset(&response_message[0], 0, 20);
 8001e16:	2214      	movs	r2, #20
 8001e18:	2100      	movs	r1, #0
 8001e1a:	a801      	add	r0, sp, #4
 8001e1c:	f019 fe90 	bl	801bb40 <memset>
	response_message[0]=PROTOCOL_PREAMBLE;
 8001e20:	232a      	movs	r3, #42	; 0x2a
 8001e22:	f88d 3004 	strb.w	r3, [sp, #4]
	switch(rx_packet->element)
 8001e26:	7863      	ldrb	r3, [r4, #1]
 8001e28:	2b55      	cmp	r3, #85	; 0x55
 8001e2a:	d80f      	bhi.n	8001e4c <process_get_command+0x3c>
 8001e2c:	2b43      	cmp	r3, #67	; 0x43
 8001e2e:	d90f      	bls.n	8001e50 <process_get_command+0x40>
 8001e30:	3b44      	subs	r3, #68	; 0x44
 8001e32:	2b11      	cmp	r3, #17
 8001e34:	d80c      	bhi.n	8001e50 <process_get_command+0x40>
 8001e36:	e8df f003 	tbb	[pc, r3]
 8001e3a:	0b4a      	.short	0x0b4a
 8001e3c:	0bc60b56 	.word	0x0bc60b56
 8001e40:	0b0b0b0b 	.word	0x0b0b0b0b
 8001e44:	0b0b0b0b 	.word	0x0b0b0b0b
 8001e48:	660d120b 	.word	0x660d120b
 8001e4c:	2b66      	cmp	r3, #102	; 0x66
 8001e4e:	d02d      	beq.n	8001eac <process_get_command+0x9c>
 8001e50:	2000      	movs	r0, #0
 8001e52:	e002      	b.n	8001e5a <process_get_command+0x4a>
	{
		case ELEMENT_TEMPERATURE:
			response_temperature();
 8001e54:	f7ff ff58 	bl	8001d08 <response_temperature>
	uint8_t ret_val=1;
 8001e58:	2001      	movs	r0, #1
		default:
			ret_val=0;
			break;
	}
	return ret_val;
}
 8001e5a:	b006      	add	sp, #24
 8001e5c:	bd10      	pop	{r4, pc}
			response_message[2]=(TIM1->CCR4/100)+48;
 8001e5e:	495d      	ldr	r1, [pc, #372]	; (8001fd4 <process_get_command+0x1c4>)
			response_message[1]='F';
 8001e60:	2346      	movs	r3, #70	; 0x46
 8001e62:	f88d 3005 	strb.w	r3, [sp, #5]
			response_message[2]=(TIM1->CCR4/100)+48;
 8001e66:	6c0a      	ldr	r2, [r1, #64]	; 0x40
 8001e68:	2064      	movs	r0, #100	; 0x64
 8001e6a:	fbb2 f2f0 	udiv	r2, r2, r0
 8001e6e:	3230      	adds	r2, #48	; 0x30
 8001e70:	f88d 2006 	strb.w	r2, [sp, #6]
			response_message[3]=((TIM1->CCR4%100)/10)+48;
 8001e74:	6c0b      	ldr	r3, [r1, #64]	; 0x40
 8001e76:	fbb3 f2f0 	udiv	r2, r3, r0
 8001e7a:	fb00 3312 	mls	r3, r0, r2, r3
 8001e7e:	220a      	movs	r2, #10
 8001e80:	fbb3 f3f2 	udiv	r3, r3, r2
 8001e84:	3330      	adds	r3, #48	; 0x30
 8001e86:	f88d 3007 	strb.w	r3, [sp, #7]
			response_message[4]=(TIM1->CCR4%10)+48;
 8001e8a:	6c0b      	ldr	r3, [r1, #64]	; 0x40
 8001e8c:	fbb3 f1f2 	udiv	r1, r3, r2
 8001e90:	fb02 3311 	mls	r3, r2, r1, r3
 8001e94:	3330      	adds	r3, #48	; 0x30
 8001e96:	f88d 3008 	strb.w	r3, [sp, #8]
			response_message[5]=PROTOCOL_POSAMBLE;
 8001e9a:	2323      	movs	r3, #35	; 0x23
 8001e9c:	f88d 3009 	strb.w	r3, [sp, #9]
			uart_driver_send(&uart_driver, (uint8_t *)response_message, 6);
 8001ea0:	2206      	movs	r2, #6
 8001ea2:	a901      	add	r1, sp, #4
 8001ea4:	484c      	ldr	r0, [pc, #304]	; (8001fd8 <process_get_command+0x1c8>)
 8001ea6:	f001 f86b 	bl	8002f80 <uart_driver_send>
 8001eaa:	e7d5      	b.n	8001e58 <process_get_command+0x48>
			response_message[1]=(char)ELEMENT_FAN_STATUS;
 8001eac:	f88d 3005 	strb.w	r3, [sp, #5]
			if(TIM1->CCR4==0)
 8001eb0:	4b48      	ldr	r3, [pc, #288]	; (8001fd4 <process_get_command+0x1c4>)
 8001eb2:	6c1b      	ldr	r3, [r3, #64]	; 0x40
				response_message[2]='1';
 8001eb4:	2b00      	cmp	r3, #0
 8001eb6:	bf0c      	ite	eq
 8001eb8:	2330      	moveq	r3, #48	; 0x30
 8001eba:	2331      	movne	r3, #49	; 0x31
 8001ebc:	f88d 3006 	strb.w	r3, [sp, #6]
			response_message[3]=PROTOCOL_POSAMBLE;
 8001ec0:	2323      	movs	r3, #35	; 0x23
			uart_driver_send(&uart_driver, (uint8_t *)response_message, 4);
 8001ec2:	2204      	movs	r2, #4
			response_message[3]=PROTOCOL_POSAMBLE;
 8001ec4:	f88d 3007 	strb.w	r3, [sp, #7]
			uart_driver_send(&uart_driver, (uint8_t *)response_message, 4);
 8001ec8:	eb0d 0102 	add.w	r1, sp, r2
 8001ecc:	e7ea      	b.n	8001ea4 <process_get_command+0x94>
			response_message[1]=(char)ELEMENT_DOOR;
 8001ece:	2344      	movs	r3, #68	; 0x44
 8001ed0:	f88d 3005 	strb.w	r3, [sp, #5]
			response_message[2]=48+HAL_GPIO_ReadPin(DOOR_GPIO_Port, DOOR_Pin);
 8001ed4:	f44f 4180 	mov.w	r1, #16384	; 0x4000
			response_message[2]=HAL_GPIO_ReadPin(HEATER_GPIO_Port, HEATER_Pin)+48;
 8001ed8:	4840      	ldr	r0, [pc, #256]	; (8001fdc <process_get_command+0x1cc>)
 8001eda:	f002 fd23 	bl	8004924 <HAL_GPIO_ReadPin>
 8001ede:	3030      	adds	r0, #48	; 0x30
 8001ee0:	f88d 0006 	strb.w	r0, [sp, #6]
 8001ee4:	e7ec      	b.n	8001ec0 <process_get_command+0xb0>
			response_message[1]='V';
 8001ee6:	2356      	movs	r3, #86	; 0x56
			strcat(response_message, FW_VERSION);
 8001ee8:	493d      	ldr	r1, [pc, #244]	; (8001fe0 <process_get_command+0x1d0>)
			response_message[1]='V';
 8001eea:	f88d 3005 	strb.w	r3, [sp, #5]
			strcat(response_message, FW_VERSION);
 8001eee:	a801      	add	r0, sp, #4
 8001ef0:	f01a fd26 	bl	801c940 <strcat>
			strcat(response_message, "#");
 8001ef4:	493b      	ldr	r1, [pc, #236]	; (8001fe4 <process_get_command+0x1d4>)
 8001ef6:	a801      	add	r0, sp, #4
 8001ef8:	f01a fd22 	bl	801c940 <strcat>
			uart_driver_send(&uart_driver, (uint8_t *)response_message, strlen(response_message));
 8001efc:	a801      	add	r0, sp, #4
 8001efe:	f7fe f977 	bl	80001f0 <strlen>
 8001f02:	4602      	mov	r2, r0
 8001f04:	e7cd      	b.n	8001ea2 <process_get_command+0x92>
			response_message[1]='C';
 8001f06:	2343      	movs	r3, #67	; 0x43
			get_runtime_DHMS(&timer[0]);
 8001f08:	4668      	mov	r0, sp
			response_message[1]='C';
 8001f0a:	f88d 3005 	strb.w	r3, [sp, #5]
			get_runtime_DHMS(&timer[0]);
 8001f0e:	f7ff ff2b 	bl	8001d68 <get_runtime_DHMS>
			response_message[2]=((timer[0]%100)/10)+48;
 8001f12:	f89d 2000 	ldrb.w	r2, [sp]
 8001f16:	2064      	movs	r0, #100	; 0x64
 8001f18:	fbb2 f1f0 	udiv	r1, r2, r0
 8001f1c:	fb00 2111 	mls	r1, r0, r1, r2
 8001f20:	230a      	movs	r3, #10
 8001f22:	b2c9      	uxtb	r1, r1
 8001f24:	fbb1 f1f3 	udiv	r1, r1, r3
 8001f28:	3130      	adds	r1, #48	; 0x30
 8001f2a:	f88d 1006 	strb.w	r1, [sp, #6]
			response_message[3]=(timer[0]%10)+48;
 8001f2e:	fbb2 f1f3 	udiv	r1, r2, r3
 8001f32:	fb03 2211 	mls	r2, r3, r1, r2
 8001f36:	3230      	adds	r2, #48	; 0x30
 8001f38:	f88d 2007 	strb.w	r2, [sp, #7]
			response_message[5]=((timer[1]%100)/10)+48;
 8001f3c:	f89d 2001 	ldrb.w	r2, [sp, #1]
 8001f40:	fbb2 f1f0 	udiv	r1, r2, r0
 8001f44:	fb00 2111 	mls	r1, r0, r1, r2
 8001f48:	b2c9      	uxtb	r1, r1
 8001f4a:	fbb1 f1f3 	udiv	r1, r1, r3
 8001f4e:	3130      	adds	r1, #48	; 0x30
 8001f50:	f88d 1009 	strb.w	r1, [sp, #9]
			response_message[6]=(timer[1]%10)+48;
 8001f54:	fbb2 f1f3 	udiv	r1, r2, r3
 8001f58:	fb03 2211 	mls	r2, r3, r1, r2
 8001f5c:	3230      	adds	r2, #48	; 0x30
 8001f5e:	f88d 200a 	strb.w	r2, [sp, #10]
			response_message[8]=((timer[2]%100)/10)+48;
 8001f62:	f89d 2002 	ldrb.w	r2, [sp, #2]
 8001f66:	fbb2 f1f0 	udiv	r1, r2, r0
 8001f6a:	fb00 2111 	mls	r1, r0, r1, r2
 8001f6e:	b2c9      	uxtb	r1, r1
 8001f70:	fbb1 f1f3 	udiv	r1, r1, r3
 8001f74:	3130      	adds	r1, #48	; 0x30
 8001f76:	f88d 100c 	strb.w	r1, [sp, #12]
			response_message[9]=(timer[2]%10)+48;
 8001f7a:	fbb2 f1f3 	udiv	r1, r2, r3
 8001f7e:	fb03 2211 	mls	r2, r3, r1, r2
			response_message[11]=((timer[3]%100)/10)+48;
 8001f82:	f89d 1003 	ldrb.w	r1, [sp, #3]
			response_message[9]=(timer[2]%10)+48;
 8001f86:	3230      	adds	r2, #48	; 0x30
 8001f88:	f88d 200d 	strb.w	r2, [sp, #13]
			response_message[11]=((timer[3]%100)/10)+48;
 8001f8c:	fbb1 f2f0 	udiv	r2, r1, r0
 8001f90:	fb00 1212 	mls	r2, r0, r2, r1
 8001f94:	b2d2      	uxtb	r2, r2
 8001f96:	fbb2 f2f3 	udiv	r2, r2, r3
 8001f9a:	3230      	adds	r2, #48	; 0x30
 8001f9c:	f88d 200f 	strb.w	r2, [sp, #15]
			response_message[12]=(timer[3]%10)+48;
 8001fa0:	fbb1 f2f3 	udiv	r2, r1, r3
 8001fa4:	fb03 1112 	mls	r1, r3, r2, r1
			response_message[4]=':';
 8001fa8:	243a      	movs	r4, #58	; 0x3a
			response_message[12]=(timer[3]%10)+48;
 8001faa:	3130      	adds	r1, #48	; 0x30
			response_message[13]=PROTOCOL_POSAMBLE;
 8001fac:	2323      	movs	r3, #35	; 0x23
			response_message[4]=':';
 8001fae:	f88d 4008 	strb.w	r4, [sp, #8]
			response_message[7]=':';
 8001fb2:	f88d 400b 	strb.w	r4, [sp, #11]
			response_message[10]=':';
 8001fb6:	f88d 400e 	strb.w	r4, [sp, #14]
			response_message[12]=(timer[3]%10)+48;
 8001fba:	f88d 1010 	strb.w	r1, [sp, #16]
			response_message[13]=PROTOCOL_POSAMBLE;
 8001fbe:	f88d 3011 	strb.w	r3, [sp, #17]
			uart_driver_send(&uart_driver, (uint8_t *)response_message, 14);
 8001fc2:	220e      	movs	r2, #14
 8001fc4:	e76d      	b.n	8001ea2 <process_get_command+0x92>
			response_message[1]=(char)ELEMENT_HEATER;
 8001fc6:	2348      	movs	r3, #72	; 0x48
 8001fc8:	f88d 3005 	strb.w	r3, [sp, #5]
			response_message[2]=HAL_GPIO_ReadPin(HEATER_GPIO_Port, HEATER_Pin)+48;
 8001fcc:	f44f 5100 	mov.w	r1, #8192	; 0x2000
 8001fd0:	e782      	b.n	8001ed8 <process_get_command+0xc8>
 8001fd2:	bf00      	nop
 8001fd4:	40010000 	.word	0x40010000
 8001fd8:	20001768 	.word	0x20001768
 8001fdc:	40021800 	.word	0x40021800
 8001fe0:	0801eb48 	.word	0x0801eb48
 8001fe4:	0801eb55 	.word	0x0801eb55

08001fe8 <parse_command>:

void parse_command(uint8_t *data)
{
 8001fe8:	b508      	push	{r3, lr}
	rx_packet_t *packet = (rx_packet_t *)data;
	if(packet->operation == OPERATION_GET)
 8001fea:	7803      	ldrb	r3, [r0, #0]
 8001fec:	2b47      	cmp	r3, #71	; 0x47
 8001fee:	d109      	bne.n	8002004 <parse_command+0x1c>
	{
		if(!process_get_command(packet))
 8001ff0:	f7ff ff0e 	bl	8001e10 <process_get_command>
 8001ff4:	b978      	cbnz	r0, 8002016 <parse_command+0x2e>
		{
			uart_driver_send(&uart_driver, (uint8_t *)nack_message, sizeof(nack_message)-1);
 8001ff6:	4908      	ldr	r1, [pc, #32]	; (8002018 <parse_command+0x30>)
 8001ff8:	2206      	movs	r2, #6
			uart_driver_send(&uart_driver, (uint8_t *)nack_message, sizeof(nack_message)-1);
		}
	}else{
		uart_driver_send(&uart_driver, (uint8_t *)nack_message, sizeof(nack_message)-1);
	}
}
 8001ffa:	e8bd 4008 	ldmia.w	sp!, {r3, lr}
			uart_driver_send(&uart_driver, (uint8_t *)ack_message, sizeof(ack_message)-1);
 8001ffe:	4807      	ldr	r0, [pc, #28]	; (800201c <parse_command+0x34>)
 8002000:	f000 bfbe 	b.w	8002f80 <uart_driver_send>
	}else if(packet->operation == OPERATION_SET){
 8002004:	2b53      	cmp	r3, #83	; 0x53
 8002006:	d1f6      	bne.n	8001ff6 <parse_command+0xe>
		if(process_set_command(packet))
 8002008:	f7ff fedc 	bl	8001dc4 <process_set_command>
 800200c:	2800      	cmp	r0, #0
 800200e:	d0f2      	beq.n	8001ff6 <parse_command+0xe>
			uart_driver_send(&uart_driver, (uint8_t *)ack_message, sizeof(ack_message)-1);
 8002010:	4903      	ldr	r1, [pc, #12]	; (8002020 <parse_command+0x38>)
 8002012:	2205      	movs	r2, #5
 8002014:	e7f1      	b.n	8001ffa <parse_command+0x12>
}
 8002016:	bd08      	pop	{r3, pc}
 8002018:	0801eb5d 	.word	0x0801eb5d
 800201c:	20001768 	.word	0x20001768
 8002020:	0801eb57 	.word	0x0801eb57

08002024 <SPI5_Write>:
/**
  * @brief  Writes a byte to device.
  * @param  Value: value to be written
  */
static void SPI5_Write(uint16_t Value)
{
 8002024:	b507      	push	{r0, r1, r2, lr}
  HAL_StatusTypeDef status = HAL_OK;

  status = HAL_SPI_Transmit(&hspi5, (uint8_t*) &Value, 1, Spi5Timeout);
 8002026:	4b06      	ldr	r3, [pc, #24]	; (8002040 <SPI5_Write+0x1c>)
{
 8002028:	f8ad 0006 	strh.w	r0, [sp, #6]
  status = HAL_SPI_Transmit(&hspi5, (uint8_t*) &Value, 1, Spi5Timeout);
 800202c:	681b      	ldr	r3, [r3, #0]
 800202e:	4805      	ldr	r0, [pc, #20]	; (8002044 <SPI5_Write+0x20>)
 8002030:	2201      	movs	r2, #1
 8002032:	f10d 0106 	add.w	r1, sp, #6
 8002036:	f003 ffa9 	bl	8005f8c <HAL_SPI_Transmit>
  if(status != HAL_OK)
  {
    /* Re-Initialize the BUS */
    SPI5_Error();
  }
}
 800203a:	b003      	add	sp, #12
 800203c:	f85d fb04 	ldr.w	pc, [sp], #4
 8002040:	20000010 	.word	0x20000010
 8002044:	20001590 	.word	0x20001590

08002048 <SystemClock_Config>:
{
 8002048:	b530      	push	{r4, r5, lr}
 800204a:	b095      	sub	sp, #84	; 0x54
  RCC_OscInitTypeDef RCC_OscInitStruct = {0};
 800204c:	2210      	movs	r2, #16
 800204e:	2100      	movs	r1, #0
 8002050:	a80a      	add	r0, sp, #40	; 0x28
 8002052:	f019 fd75 	bl	801bb40 <memset>
  RCC_ClkInitTypeDef RCC_ClkInitStruct = {0};
 8002056:	2214      	movs	r2, #20
 8002058:	2100      	movs	r1, #0
 800205a:	a803      	add	r0, sp, #12
 800205c:	f019 fd70 	bl	801bb40 <memset>
  __HAL_RCC_PWR_CLK_ENABLE();
 8002060:	2400      	movs	r4, #0
 8002062:	4b1d      	ldr	r3, [pc, #116]	; (80020d8 <SystemClock_Config+0x90>)
 8002064:	9401      	str	r4, [sp, #4]
 8002066:	6c1a      	ldr	r2, [r3, #64]	; 0x40
 8002068:	f042 5280 	orr.w	r2, r2, #268435456	; 0x10000000
 800206c:	641a      	str	r2, [r3, #64]	; 0x40
 800206e:	6c1b      	ldr	r3, [r3, #64]	; 0x40
 8002070:	f003 5380 	and.w	r3, r3, #268435456	; 0x10000000
 8002074:	9301      	str	r3, [sp, #4]
 8002076:	9b01      	ldr	r3, [sp, #4]
  __HAL_PWR_VOLTAGESCALING_CONFIG(PWR_REGULATOR_VOLTAGE_SCALE1);
 8002078:	4b18      	ldr	r3, [pc, #96]	; (80020dc <SystemClock_Config+0x94>)
 800207a:	9402      	str	r4, [sp, #8]
 800207c:	681a      	ldr	r2, [r3, #0]
 800207e:	f442 4240 	orr.w	r2, r2, #49152	; 0xc000
 8002082:	601a      	str	r2, [r3, #0]
 8002084:	681b      	ldr	r3, [r3, #0]
 8002086:	f403 4340 	and.w	r3, r3, #49152	; 0xc000
 800208a:	9302      	str	r3, [sp, #8]
  RCC_OscInitStruct.HSEState = RCC_HSE_ON;
 800208c:	2201      	movs	r2, #1
  __HAL_PWR_VOLTAGESCALING_CONFIG(PWR_REGULATOR_VOLTAGE_SCALE1);
 800208e:	9b02      	ldr	r3, [sp, #8]
  RCC_OscInitStruct.HSEState = RCC_HSE_ON;
 8002090:	f44f 3380 	mov.w	r3, #65536	; 0x10000
 8002094:	e9cd 2308 	strd	r2, r3, [sp, #32]
  RCC_OscInitStruct.PLL.PLLSource = RCC_PLLSOURCE_HSE;
 8002098:	2502      	movs	r5, #2
 800209a:	f44f 0380 	mov.w	r3, #4194304	; 0x400000
 800209e:	e9cd 530e 	strd	r5, r3, [sp, #56]	; 0x38
  RCC_OscInitStruct.PLL.PLLN = 336;
 80020a2:	2108      	movs	r1, #8
 80020a4:	f44f 73a8 	mov.w	r3, #336	; 0x150
 80020a8:	e9cd 1310 	strd	r1, r3, [sp, #64]	; 0x40
  if (HAL_RCC_OscConfig(&RCC_OscInitStruct) != HAL_OK)
 80020ac:	a808      	add	r0, sp, #32
  RCC_OscInitStruct.PLL.PLLQ = 4;
 80020ae:	2304      	movs	r3, #4
 80020b0:	9313      	str	r3, [sp, #76]	; 0x4c
  RCC_OscInitStruct.PLL.PLLP = RCC_PLLP_DIV2;
 80020b2:	9512      	str	r5, [sp, #72]	; 0x48
  if (HAL_RCC_OscConfig(&RCC_OscInitStruct) != HAL_OK)
 80020b4:	f003 fa38 	bl	8005528 <HAL_RCC_OscConfig>
  RCC_ClkInitStruct.ClockType = RCC_CLOCKTYPE_HCLK|RCC_CLOCKTYPE_SYSCLK
 80020b8:	230f      	movs	r3, #15
  RCC_ClkInitStruct.SYSCLKSource = RCC_SYSCLKSOURCE_PLLCLK;
 80020ba:	e9cd 3503 	strd	r3, r5, [sp, #12]
  RCC_ClkInitStruct.APB2CLKDivider = RCC_HCLK_DIV2;
 80020be:	f44f 50a0 	mov.w	r0, #5120	; 0x1400
 80020c2:	f44f 5380 	mov.w	r3, #4096	; 0x1000
 80020c6:	e9cd 0306 	strd	r0, r3, [sp, #24]
  if (HAL_RCC_ClockConfig(&RCC_ClkInitStruct, FLASH_LATENCY_5) != HAL_OK)
 80020ca:	2105      	movs	r1, #5
 80020cc:	a803      	add	r0, sp, #12
  RCC_ClkInitStruct.AHBCLKDivider = RCC_SYSCLK_DIV1;
 80020ce:	9405      	str	r4, [sp, #20]
  if (HAL_RCC_ClockConfig(&RCC_ClkInitStruct, FLASH_LATENCY_5) != HAL_OK)
 80020d0:	f003 fc08 	bl	80058e4 <HAL_RCC_ClockConfig>
}
 80020d4:	b015      	add	sp, #84	; 0x54
 80020d6:	bd30      	pop	{r4, r5, pc}
 80020d8:	40023800 	.word	0x40023800
 80020dc:	40007000 	.word	0x40007000

080020e0 <main>:
{
 80020e0:	e92d 4880 	stmdb	sp!, {r7, fp, lr}
 80020e4:	b09b      	sub	sp, #108	; 0x6c
  HAL_Init();
 80020e6:	f002 f943 	bl	8004370 <HAL_Init>
  SystemClock_Config();
 80020ea:	f7ff ffad 	bl	8002048 <SystemClock_Config>
  GPIO_InitTypeDef GPIO_InitStruct = {0};
 80020ee:	2214      	movs	r2, #20
 80020f0:	2100      	movs	r1, #0
 80020f2:	a80d      	add	r0, sp, #52	; 0x34
  __HAL_RCC_GPIOE_CLK_ENABLE();
 80020f4:	2400      	movs	r4, #0
  GPIO_InitTypeDef GPIO_InitStruct = {0};
 80020f6:	f019 fd23 	bl	801bb40 <memset>
  __HAL_RCC_GPIOE_CLK_ENABLE();
 80020fa:	4bc5      	ldr	r3, [pc, #788]	; (8002410 <main+0x330>)
 80020fc:	9400      	str	r4, [sp, #0]
 80020fe:	6b1a      	ldr	r2, [r3, #48]	; 0x30
  HAL_GPIO_WritePin(SC_BMP280_GPIO_Port, SC_BMP280_Pin, GPIO_PIN_RESET);
 8002100:	48c4      	ldr	r0, [pc, #784]	; (8002414 <main+0x334>)
  hi2c3.Instance = I2C3;
 8002102:	4dc5      	ldr	r5, [pc, #788]	; (8002418 <main+0x338>)
  __HAL_RCC_GPIOE_CLK_ENABLE();
 8002104:	f042 0210 	orr.w	r2, r2, #16
 8002108:	631a      	str	r2, [r3, #48]	; 0x30
 800210a:	6b1a      	ldr	r2, [r3, #48]	; 0x30
 800210c:	f002 0210 	and.w	r2, r2, #16
 8002110:	9200      	str	r2, [sp, #0]
 8002112:	9a00      	ldr	r2, [sp, #0]
  __HAL_RCC_GPIOF_CLK_ENABLE();
 8002114:	9401      	str	r4, [sp, #4]
 8002116:	6b1a      	ldr	r2, [r3, #48]	; 0x30
 8002118:	f042 0220 	orr.w	r2, r2, #32
 800211c:	631a      	str	r2, [r3, #48]	; 0x30
 800211e:	6b1a      	ldr	r2, [r3, #48]	; 0x30
 8002120:	f002 0220 	and.w	r2, r2, #32
 8002124:	9201      	str	r2, [sp, #4]
 8002126:	9a01      	ldr	r2, [sp, #4]
  __HAL_RCC_GPIOH_CLK_ENABLE();
 8002128:	9402      	str	r4, [sp, #8]
 800212a:	6b1a      	ldr	r2, [r3, #48]	; 0x30
 800212c:	f042 0280 	orr.w	r2, r2, #128	; 0x80
 8002130:	631a      	str	r2, [r3, #48]	; 0x30
 8002132:	6b1a      	ldr	r2, [r3, #48]	; 0x30
 8002134:	f002 0280 	and.w	r2, r2, #128	; 0x80
 8002138:	9202      	str	r2, [sp, #8]
 800213a:	9a02      	ldr	r2, [sp, #8]
  __HAL_RCC_GPIOC_CLK_ENABLE();
 800213c:	9403      	str	r4, [sp, #12]
 800213e:	6b1a      	ldr	r2, [r3, #48]	; 0x30
 8002140:	f042 0204 	orr.w	r2, r2, #4
 8002144:	631a      	str	r2, [r3, #48]	; 0x30
 8002146:	6b1a      	ldr	r2, [r3, #48]	; 0x30
 8002148:	f002 0204 	and.w	r2, r2, #4
 800214c:	9203      	str	r2, [sp, #12]
 800214e:	9a03      	ldr	r2, [sp, #12]
  __HAL_RCC_GPIOA_CLK_ENABLE();
 8002150:	9404      	str	r4, [sp, #16]
 8002152:	6b1a      	ldr	r2, [r3, #48]	; 0x30
 8002154:	f042 0201 	orr.w	r2, r2, #1
 8002158:	631a      	str	r2, [r3, #48]	; 0x30
 800215a:	6b1a      	ldr	r2, [r3, #48]	; 0x30
 800215c:	f002 0201 	and.w	r2, r2, #1
 8002160:	9204      	str	r2, [sp, #16]
 8002162:	9a04      	ldr	r2, [sp, #16]
  __HAL_RCC_GPIOB_CLK_ENABLE();
 8002164:	9405      	str	r4, [sp, #20]
 8002166:	6b1a      	ldr	r2, [r3, #48]	; 0x30
 8002168:	f042 0202 	orr.w	r2, r2, #2
 800216c:	631a      	str	r2, [r3, #48]	; 0x30
 800216e:	6b1a      	ldr	r2, [r3, #48]	; 0x30
 8002170:	f002 0202 	and.w	r2, r2, #2
 8002174:	9205      	str	r2, [sp, #20]
 8002176:	9a05      	ldr	r2, [sp, #20]
  __HAL_RCC_GPIOG_CLK_ENABLE();
 8002178:	9406      	str	r4, [sp, #24]
 800217a:	6b1a      	ldr	r2, [r3, #48]	; 0x30
 800217c:	f042 0240 	orr.w	r2, r2, #64	; 0x40
 8002180:	631a      	str	r2, [r3, #48]	; 0x30
 8002182:	6b1a      	ldr	r2, [r3, #48]	; 0x30
 8002184:	f002 0240 	and.w	r2, r2, #64	; 0x40
 8002188:	9206      	str	r2, [sp, #24]
 800218a:	9a06      	ldr	r2, [sp, #24]
  __HAL_RCC_GPIOD_CLK_ENABLE();
 800218c:	9407      	str	r4, [sp, #28]
 800218e:	6b1a      	ldr	r2, [r3, #48]	; 0x30
 8002190:	f042 0208 	orr.w	r2, r2, #8
 8002194:	631a      	str	r2, [r3, #48]	; 0x30
 8002196:	6b1b      	ldr	r3, [r3, #48]	; 0x30
 8002198:	f003 0308 	and.w	r3, r3, #8
 800219c:	9307      	str	r3, [sp, #28]
  HAL_GPIO_WritePin(SC_BMP280_GPIO_Port, SC_BMP280_Pin, GPIO_PIN_RESET);
 800219e:	4622      	mov	r2, r4
 80021a0:	2110      	movs	r1, #16
  __HAL_RCC_GPIOD_CLK_ENABLE();
 80021a2:	9b07      	ldr	r3, [sp, #28]
  HAL_GPIO_WritePin(SC_BMP280_GPIO_Port, SC_BMP280_Pin, GPIO_PIN_RESET);
 80021a4:	f002 fbc4 	bl	8004930 <HAL_GPIO_WritePin>
  HAL_GPIO_WritePin(GPIOC, GPIO_PIN_2, GPIO_PIN_RESET);
 80021a8:	489c      	ldr	r0, [pc, #624]	; (800241c <main+0x33c>)
 80021aa:	4622      	mov	r2, r4
 80021ac:	2104      	movs	r1, #4
 80021ae:	f002 fbbf 	bl	8004930 <HAL_GPIO_WritePin>
  HAL_GPIO_WritePin(GPIOD, GPIO_PIN_12|GPIO_PIN_13, GPIO_PIN_RESET);
 80021b2:	489b      	ldr	r0, [pc, #620]	; (8002420 <main+0x340>)
 80021b4:	4622      	mov	r2, r4
 80021b6:	f44f 5140 	mov.w	r1, #12288	; 0x3000
 80021ba:	f002 fbb9 	bl	8004930 <HAL_GPIO_WritePin>
  HAL_GPIO_WritePin(GPIOG, LED2_Pin|LED1_Pin, GPIO_PIN_RESET);
 80021be:	4622      	mov	r2, r4
 80021c0:	4898      	ldr	r0, [pc, #608]	; (8002424 <main+0x344>)
 80021c2:	f44f 41c0 	mov.w	r1, #24576	; 0x6000
 80021c6:	f002 fbb3 	bl	8004930 <HAL_GPIO_WritePin>
  GPIO_InitStruct.Mode = GPIO_MODE_OUTPUT_PP;
 80021ca:	2601      	movs	r6, #1
 80021cc:	f04f 0910 	mov.w	r9, #16
  HAL_GPIO_Init(SC_BMP280_GPIO_Port, &GPIO_InitStruct);
 80021d0:	4890      	ldr	r0, [pc, #576]	; (8002414 <main+0x334>)
 80021d2:	a90d      	add	r1, sp, #52	; 0x34
  GPIO_InitStruct.Speed = GPIO_SPEED_FREQ_HIGH;
 80021d4:	2702      	movs	r7, #2
  GPIO_InitStruct.Pin = GPIO_PIN_2;
 80021d6:	f04f 0804 	mov.w	r8, #4
  GPIO_InitStruct.Mode = GPIO_MODE_OUTPUT_PP;
 80021da:	e9cd 960d 	strd	r9, r6, [sp, #52]	; 0x34
  GPIO_InitStruct.Speed = GPIO_SPEED_FREQ_LOW;
 80021de:	e9cd 440f 	strd	r4, r4, [sp, #60]	; 0x3c
  HAL_GPIO_Init(SC_BMP280_GPIO_Port, &GPIO_InitStruct);
 80021e2:	f002 fab9 	bl	8004758 <HAL_GPIO_Init>
  HAL_GPIO_Init(GPIOC, &GPIO_InitStruct);
 80021e6:	488d      	ldr	r0, [pc, #564]	; (800241c <main+0x33c>)
  GPIO_InitStruct.Pull = GPIO_NOPULL;
 80021e8:	940f      	str	r4, [sp, #60]	; 0x3c
  HAL_GPIO_Init(GPIOC, &GPIO_InitStruct);
 80021ea:	a90d      	add	r1, sp, #52	; 0x34
  GPIO_InitStruct.Mode = GPIO_MODE_OUTPUT_PP;
 80021ec:	e9cd 860d 	strd	r8, r6, [sp, #52]	; 0x34
  GPIO_InitStruct.Speed = GPIO_SPEED_FREQ_HIGH;
 80021f0:	9710      	str	r7, [sp, #64]	; 0x40
  HAL_GPIO_Init(GPIOC, &GPIO_InitStruct);
 80021f2:	f002 fab1 	bl	8004758 <HAL_GPIO_Init>
  GPIO_InitStruct.Pin = GPIO_PIN_12|GPIO_PIN_13;
 80021f6:	f44f 5340 	mov.w	r3, #12288	; 0x3000
  HAL_GPIO_Init(GPIOD, &GPIO_InitStruct);
 80021fa:	4889      	ldr	r0, [pc, #548]	; (8002420 <main+0x340>)
 80021fc:	a90d      	add	r1, sp, #52	; 0x34
  GPIO_InitStruct.Mode = GPIO_MODE_OUTPUT_PP;
 80021fe:	e9cd 360d 	strd	r3, r6, [sp, #52]	; 0x34
  GPIO_InitStruct.Speed = GPIO_SPEED_FREQ_HIGH;
 8002202:	e9cd 470f 	strd	r4, r7, [sp, #60]	; 0x3c
  HAL_GPIO_Init(GPIOD, &GPIO_InitStruct);
 8002206:	f002 faa7 	bl	8004758 <HAL_GPIO_Init>
  HAL_GPIO_Init(GPIOG, &GPIO_InitStruct);
 800220a:	a90d      	add	r1, sp, #52	; 0x34
  GPIO_InitStruct.Pin = LED2_Pin|LED1_Pin;
 800220c:	f44f 43c0 	mov.w	r3, #24576	; 0x6000
  HAL_GPIO_Init(GPIOG, &GPIO_InitStruct);
 8002210:	4884      	ldr	r0, [pc, #528]	; (8002424 <main+0x344>)
  GPIO_InitStruct.Mode = GPIO_MODE_OUTPUT_PP;
 8002212:	e9cd 360d 	strd	r3, r6, [sp, #52]	; 0x34
  GPIO_InitStruct.Speed = GPIO_SPEED_FREQ_LOW;
 8002216:	e9cd 440f 	strd	r4, r4, [sp, #60]	; 0x3c
  HAL_GPIO_Init(GPIOG, &GPIO_InitStruct);
 800221a:	f002 fa9d 	bl	8004758 <HAL_GPIO_Init>
  hcrc.Instance = CRC;
 800221e:	4882      	ldr	r0, [pc, #520]	; (8002428 <main+0x348>)
 8002220:	4b82      	ldr	r3, [pc, #520]	; (800242c <main+0x34c>)
 8002222:	6003      	str	r3, [r0, #0]
  if (HAL_CRC_Init(&hcrc) != HAL_OK)
 8002224:	f002 f936 	bl	8004494 <HAL_CRC_Init>
  hi2c3.Init.ClockSpeed = 100000;
 8002228:	4a81      	ldr	r2, [pc, #516]	; (8002430 <main+0x350>)
 800222a:	4b82      	ldr	r3, [pc, #520]	; (8002434 <main+0x354>)
  hi2c3.Init.NoStretchMode = I2C_NOSTRETCH_DISABLE;
 800222c:	622c      	str	r4, [r5, #32]
  hi2c3.Init.ClockSpeed = 100000;
 800222e:	e9c5 2300 	strd	r2, r3, [r5]
  if (HAL_I2C_Init(&hi2c3) != HAL_OK)
 8002232:	4628      	mov	r0, r5
  hi2c3.Init.AddressingMode = I2C_ADDRESSINGMODE_7BIT;
 8002234:	f44f 4380 	mov.w	r3, #16384	; 0x4000
  hi2c3.Init.DualAddressMode = I2C_DUALADDRESS_DISABLE;
 8002238:	e9c5 3404 	strd	r3, r4, [r5, #16]
  hi2c3.Init.OwnAddress1 = 0;
 800223c:	e9c5 4402 	strd	r4, r4, [r5, #8]
  hi2c3.Init.GeneralCallMode = I2C_GENERALCALL_DISABLE;
 8002240:	e9c5 4406 	strd	r4, r4, [r5, #24]
  if (HAL_I2C_Init(&hi2c3) != HAL_OK)
 8002244:	f002 fd56 	bl	8004cf4 <HAL_I2C_Init>
  if (HAL_I2CEx_ConfigAnalogFilter(&hi2c3, I2C_ANALOGFILTER_DISABLE) != HAL_OK)
 8002248:	4649      	mov	r1, r9
 800224a:	4628      	mov	r0, r5
 800224c:	f002 ff92 	bl	8005174 <HAL_I2CEx_ConfigAnalogFilter>
  if (HAL_I2CEx_ConfigDigitalFilter(&hi2c3, 0) != HAL_OK)
 8002250:	4621      	mov	r1, r4
 8002252:	4628      	mov	r0, r5
 8002254:	f002 ffad 	bl	80051b2 <HAL_I2CEx_ConfigDigitalFilter>
  hspi5.Instance = SPI5;
 8002258:	4877      	ldr	r0, [pc, #476]	; (8002438 <main+0x358>)
  hspi5.Init.Mode = SPI_MODE_MASTER;
 800225a:	4978      	ldr	r1, [pc, #480]	; (800243c <main+0x35c>)
  hsdram1.Instance = FMC_SDRAM_DEVICE;
 800225c:	4d78      	ldr	r5, [pc, #480]	; (8002440 <main+0x360>)
  hspi5.Init.CRCCalculation = SPI_CRCCALCULATION_DISABLE;
 800225e:	6284      	str	r4, [r0, #40]	; 0x28
  hspi5.Init.Mode = SPI_MODE_MASTER;
 8002260:	f44f 7382 	mov.w	r3, #260	; 0x104
 8002264:	e9c0 1300 	strd	r1, r3, [r0]
  hspi5.Init.BaudRatePrescaler = SPI_BAUDRATEPRESCALER_16;
 8002268:	2218      	movs	r2, #24
  hspi5.Init.CRCPolynomial = 10;
 800226a:	230a      	movs	r3, #10
  hspi5.Init.BaudRatePrescaler = SPI_BAUDRATEPRESCALER_16;
 800226c:	f44f 7b00 	mov.w	fp, #512	; 0x200
  hspi5.Init.CRCPolynomial = 10;
 8002270:	62c3      	str	r3, [r0, #44]	; 0x2c
  hspi5.Init.BaudRatePrescaler = SPI_BAUDRATEPRESCALER_16;
 8002272:	e9c0 b206 	strd	fp, r2, [r0, #24]
  hspi5.Init.DataSize = SPI_DATASIZE_8BIT;
 8002276:	e9c0 4402 	strd	r4, r4, [r0, #8]
  hspi5.Init.CLKPhase = SPI_PHASE_1EDGE;
 800227a:	e9c0 4404 	strd	r4, r4, [r0, #16]
  hspi5.Init.TIMode = SPI_TIMODE_DISABLE;
 800227e:	e9c0 4408 	strd	r4, r4, [r0, #32]
  if (HAL_SPI_Init(&hspi5) != HAL_OK)
 8002282:	f003 fe27 	bl	8005ed4 <HAL_SPI_Init>
  hsdram1.Instance = FMC_SDRAM_DEVICE;
 8002286:	4a6f      	ldr	r2, [pc, #444]	; (8002444 <main+0x364>)
  hsdram1.Init.MemoryDataWidth = FMC_SDRAM_MEM_BUS_WIDTH_16;
 8002288:	f8c5 9010 	str.w	r9, [r5, #16]
  hsdram1.Init.SDBank = FMC_SDRAM_BANK2;
 800228c:	e9c5 2600 	strd	r2, r6, [r5]
  hsdram1.Init.CASLatency = FMC_SDRAM_CAS_LATENCY_3;
 8002290:	2040      	movs	r0, #64	; 0x40
 8002292:	f44f 72c0 	mov.w	r2, #384	; 0x180
 8002296:	e9c5 0205 	strd	r0, r2, [r5, #20]
  hsdram1.Init.SDClockPeriod = FMC_SDRAM_CLOCK_PERIOD_2;
 800229a:	f44f 6200 	mov.w	r2, #2048	; 0x800
  hsdram1.Init.ReadBurst = FMC_SDRAM_RBURST_DISABLE;
 800229e:	e9c5 2408 	strd	r2, r4, [r5, #32]
  hsdram1.Init.ReadPipeDelay = FMC_SDRAM_RPIPE_DELAY_1;
 80022a2:	f44f 5200 	mov.w	r2, #8192	; 0x2000
  SdramTiming.WriteRecoveryTime = 3;
 80022a6:	f04f 0a03 	mov.w	sl, #3
  hsdram1.Init.ReadPipeDelay = FMC_SDRAM_RPIPE_DELAY_1;
 80022aa:	62aa      	str	r2, [r5, #40]	; 0x28
  if (HAL_SDRAM_Init(&hsdram1, &SdramTiming) != HAL_OK)
 80022ac:	a90d      	add	r1, sp, #52	; 0x34
  SdramTiming.ExitSelfRefreshDelay = 7;
 80022ae:	2207      	movs	r2, #7
  if (HAL_SDRAM_Init(&hsdram1, &SdramTiming) != HAL_OK)
 80022b0:	4628      	mov	r0, r5
  Command->CommandTarget           = FMC_SDRAM_CMD_TARGET_BANK2;
 80022b2:	f04f 0908 	mov.w	r9, #8
  hsdram1.Init.RowBitsNumber = FMC_SDRAM_ROW_BITS_NUM_12;
 80022b6:	e9c5 4802 	strd	r4, r8, [r5, #8]
  SdramTiming.SelfRefreshTime = 4;
 80022ba:	e9cd 280e 	strd	r2, r8, [sp, #56]	; 0x38
  SdramTiming.RPDelay = 2;
 80022be:	e9cd a711 	strd	sl, r7, [sp, #68]	; 0x44
  hsdram1.Init.WriteProtection = FMC_SDRAM_WRITE_PROTECTION_DISABLE;
 80022c2:	61ec      	str	r4, [r5, #28]
  SdramTiming.RowCycleDelay = 7;
 80022c4:	9210      	str	r2, [sp, #64]	; 0x40
  SdramTiming.LoadToActiveDelay = 2;
 80022c6:	970d      	str	r7, [sp, #52]	; 0x34
  SdramTiming.RCDDelay = 2;
 80022c8:	9713      	str	r7, [sp, #76]	; 0x4c
  if (HAL_SDRAM_Init(&hsdram1, &SdramTiming) != HAL_OK)
 80022ca:	f003 fd0f 	bl	8005cec <HAL_SDRAM_Init>
  HAL_SDRAM_SendCommand(hsdram, Command, SDRAM_TIMEOUT);
 80022ce:	f64f 72ff 	movw	r2, #65535	; 0xffff
 80022d2:	a909      	add	r1, sp, #36	; 0x24
 80022d4:	4628      	mov	r0, r5
  Command->AutoRefreshNumber       = 1;
 80022d6:	e9cd 960a 	strd	r9, r6, [sp, #40]	; 0x28
  Command->CommandMode             = FMC_SDRAM_CMD_CLK_ENABLE;
 80022da:	9609      	str	r6, [sp, #36]	; 0x24
 __IO uint32_t tmpmrd =0;
 80022dc:	9408      	str	r4, [sp, #32]
  Command->ModeRegisterDefinition  = 0;
 80022de:	940c      	str	r4, [sp, #48]	; 0x30
  HAL_SDRAM_SendCommand(hsdram, Command, SDRAM_TIMEOUT);
 80022e0:	f003 fd24 	bl	8005d2c <HAL_SDRAM_SendCommand>
  HAL_Delay(1);
 80022e4:	4630      	mov	r0, r6
 80022e6:	f002 f86f 	bl	80043c8 <HAL_Delay>
  HAL_SDRAM_SendCommand(hsdram, Command, SDRAM_TIMEOUT);
 80022ea:	f64f 72ff 	movw	r2, #65535	; 0xffff
 80022ee:	a909      	add	r1, sp, #36	; 0x24
 80022f0:	4628      	mov	r0, r5
  Command->CommandTarget           = FMC_SDRAM_CMD_TARGET_BANK2;
 80022f2:	e9cd 7909 	strd	r7, r9, [sp, #36]	; 0x24
  Command->ModeRegisterDefinition  = 0;
 80022f6:	e9cd 640b 	strd	r6, r4, [sp, #44]	; 0x2c
  HAL_SDRAM_SendCommand(hsdram, Command, SDRAM_TIMEOUT);
 80022fa:	f003 fd17 	bl	8005d2c <HAL_SDRAM_SendCommand>
  HAL_SDRAM_SendCommand(hsdram, Command, SDRAM_TIMEOUT);
 80022fe:	f64f 72ff 	movw	r2, #65535	; 0xffff
 8002302:	a909      	add	r1, sp, #36	; 0x24
 8002304:	4628      	mov	r0, r5
  Command->CommandTarget           = FMC_SDRAM_CMD_TARGET_BANK2;
 8002306:	e9cd a909 	strd	sl, r9, [sp, #36]	; 0x24
  Command->ModeRegisterDefinition  = 0;
 800230a:	e9cd 840b 	strd	r8, r4, [sp, #44]	; 0x2c
  HAL_SDRAM_SendCommand(hsdram, Command, SDRAM_TIMEOUT);
 800230e:	f003 fd0d 	bl	8005d2c <HAL_SDRAM_SendCommand>
  tmpmrd = (uint32_t)SDRAM_MODEREG_BURST_LENGTH_1          |
 8002312:	f44f 720c 	mov.w	r2, #560	; 0x230
 8002316:	9208      	str	r2, [sp, #32]
  Command->ModeRegisterDefinition  = tmpmrd;
 8002318:	9a08      	ldr	r2, [sp, #32]
 800231a:	920c      	str	r2, [sp, #48]	; 0x30
  HAL_SDRAM_SendCommand(hsdram, Command, SDRAM_TIMEOUT);
 800231c:	a909      	add	r1, sp, #36	; 0x24
 800231e:	f64f 72ff 	movw	r2, #65535	; 0xffff
 8002322:	4628      	mov	r0, r5
  Command->CommandTarget           = FMC_SDRAM_CMD_TARGET_BANK2;
 8002324:	e9cd 8909 	strd	r8, r9, [sp, #36]	; 0x24
  Command->AutoRefreshNumber       = 1;
 8002328:	960b      	str	r6, [sp, #44]	; 0x2c
  HAL_SDRAM_SendCommand(hsdram, Command, SDRAM_TIMEOUT);
 800232a:	f003 fcff 	bl	8005d2c <HAL_SDRAM_SendCommand>
  HAL_SDRAM_ProgramRefreshRate(hsdram, REFRESH_COUNT);
 800232e:	f240 516a 	movw	r1, #1386	; 0x56a
 8002332:	4628      	mov	r0, r5
 8002334:	f003 fd11 	bl	8005d5a <HAL_SDRAM_ProgramRefreshRate>
  LTDC_LayerCfgTypeDef pLayerCfg = {0};
 8002338:	2234      	movs	r2, #52	; 0x34
 800233a:	4621      	mov	r1, r4
 800233c:	eb0d 0002 	add.w	r0, sp, r2
 8002340:	f019 fbfe 	bl	801bb40 <memset>
  hltdc.Instance = LTDC;
 8002344:	4d40      	ldr	r5, [pc, #256]	; (8002448 <main+0x368>)
 8002346:	4a41      	ldr	r2, [pc, #260]	; (800244c <main+0x36c>)
  hltdc.Init.Backcolor.Blue = 0;
 8002348:	86ac      	strh	r4, [r5, #52]	; 0x34
  hltdc.Init.HSPolarity = LTDC_HSPOLARITY_AL;
 800234a:	e9c5 2400 	strd	r2, r4, [r5]
  hltdc.Init.HorizontalSync = 9;
 800234e:	2209      	movs	r2, #9
  hltdc.Init.VerticalSync = 1;
 8002350:	e9c5 2605 	strd	r2, r6, [r5, #20]
  hltdc.Init.AccumulatedHBP = 29;
 8002354:	221d      	movs	r2, #29
  hltdc.Init.AccumulatedActiveH = 323;
 8002356:	f240 1c0d 	movw	ip, #269	; 0x10d
  hltdc.Init.AccumulatedVBP = 3;
 800235a:	e9c5 2a07 	strd	r2, sl, [r5, #28]
  hltdc.Init.AccumulatedActiveH = 323;
 800235e:	f240 1243 	movw	r2, #323	; 0x143
 8002362:	e9c5 c209 	strd	ip, r2, [r5, #36]	; 0x24
  hltdc.Init.TotalHeigh = 327;
 8002366:	f240 1e17 	movw	lr, #279	; 0x117
 800236a:	f240 1247 	movw	r2, #327	; 0x147
  if (HAL_LTDC_Init(&hltdc) != HAL_OK)
 800236e:	4628      	mov	r0, r5
  hltdc.Init.TotalHeigh = 327;
 8002370:	e9c5 e20b 	strd	lr, r2, [r5, #44]	; 0x2c
  hltdc.Init.DEPolarity = LTDC_DEPOLARITY_AL;
 8002374:	e9c5 4402 	strd	r4, r4, [r5, #8]
  hltdc.Init.PCPolarity = LTDC_PCPOLARITY_IPC;
 8002378:	612c      	str	r4, [r5, #16]
  hltdc.Init.Backcolor.Red = 0;
 800237a:	f885 4036 	strb.w	r4, [r5, #54]	; 0x36
  if (HAL_LTDC_Init(&hltdc) != HAL_OK)
 800237e:	f002 ffbd 	bl	80052fc <HAL_LTDC_Init>
  pLayerCfg.Alpha = 255;
 8002382:	20ff      	movs	r0, #255	; 0xff
  pLayerCfg.WindowX1 = 240;
 8002384:	21f0      	movs	r1, #240	; 0xf0
  pLayerCfg.WindowY1 = 320;
 8002386:	f44f 72a0 	mov.w	r2, #320	; 0x140
  pLayerCfg.Alpha0 = 0;
 800238a:	e9cd 0412 	strd	r0, r4, [sp, #72]	; 0x48
  pLayerCfg.BlendingFactor2 = LTDC_BLENDING_FACTOR2_CA;
 800238e:	f44f 6880 	mov.w	r8, #1024	; 0x400
 8002392:	2005      	movs	r0, #5
  pLayerCfg.WindowY0 = 0;
 8002394:	e9cd 140e 	strd	r1, r4, [sp, #56]	; 0x38
  pLayerCfg.PixelFormat = LTDC_PIXEL_FORMAT_RGB565;
 8002398:	e9cd 2710 	strd	r2, r7, [sp, #64]	; 0x40
  pLayerCfg.BlendingFactor2 = LTDC_BLENDING_FACTOR2_CA;
 800239c:	e9cd 8014 	strd	r8, r0, [sp, #80]	; 0x50
  pLayerCfg.ImageWidth = 240;
 80023a0:	e9cd 4116 	strd	r4, r1, [sp, #88]	; 0x58
  pLayerCfg.ImageHeight = 320;
 80023a4:	9218      	str	r2, [sp, #96]	; 0x60
  if (HAL_LTDC_ConfigLayer(&hltdc, &pLayerCfg, 0) != HAL_OK)
 80023a6:	a90d      	add	r1, sp, #52	; 0x34
 80023a8:	4622      	mov	r2, r4
 80023aa:	4628      	mov	r0, r5
  pLayerCfg.WindowX0 = 0;
 80023ac:	940d      	str	r4, [sp, #52]	; 0x34
  LcdDrv = &ili9341_drv;
 80023ae:	4d28      	ldr	r5, [pc, #160]	; (8002450 <main+0x370>)
  pLayerCfg.Backcolor.Blue = 0;
 80023b0:	f8ad 4064 	strh.w	r4, [sp, #100]	; 0x64
  pLayerCfg.Backcolor.Red = 0;
 80023b4:	f88d 4066 	strb.w	r4, [sp, #102]	; 0x66
  if (HAL_LTDC_ConfigLayer(&hltdc, &pLayerCfg, 0) != HAL_OK)
 80023b8:	f003 f86b 	bl	8005492 <HAL_LTDC_ConfigLayer>
  LcdDrv = &ili9341_drv;
 80023bc:	4a25      	ldr	r2, [pc, #148]	; (8002454 <main+0x374>)
 80023be:	602a      	str	r2, [r5, #0]
  LcdDrv->Init();
 80023c0:	6812      	ldr	r2, [r2, #0]
  huart1.Init.BaudRate = 115200;
 80023c2:	f8df 90a4 	ldr.w	r9, [pc, #164]	; 8002468 <main+0x388>
  htim7.Init.Prescaler = 8400-1;
 80023c6:	f8df a0a4 	ldr.w	sl, [pc, #164]	; 800246c <main+0x38c>
  LcdDrv->Init();
 80023ca:	4790      	blx	r2
  LcdDrv->DisplayOff();
 80023cc:	682a      	ldr	r2, [r5, #0]
  hdma2d.Instance = DMA2D;
 80023ce:	4d22      	ldr	r5, [pc, #136]	; (8002458 <main+0x378>)
  LcdDrv->DisplayOff();
 80023d0:	68d2      	ldr	r2, [r2, #12]
 80023d2:	4790      	blx	r2
  hdma2d.Instance = DMA2D;
 80023d4:	4a21      	ldr	r2, [pc, #132]	; (800245c <main+0x37c>)
  hdma2d.LayerCfg[1].InputColorMode = DMA2D_INPUT_RGB565;
 80023d6:	e9c5 470a 	strd	r4, r7, [r5, #40]	; 0x28
  hdma2d.LayerCfg[1].InputAlpha = 0;
 80023da:	e9c5 440c 	strd	r4, r4, [r5, #48]	; 0x30
  if (HAL_DMA2D_Init(&hdma2d) != HAL_OK)
 80023de:	4628      	mov	r0, r5
  hdma2d.Init.Mode = DMA2D_M2M;
 80023e0:	e9c5 2400 	strd	r2, r4, [r5]
  hdma2d.Init.OutputOffset = 0;
 80023e4:	e9c5 7402 	strd	r7, r4, [r5, #8]
  if (HAL_DMA2D_Init(&hdma2d) != HAL_OK)
 80023e8:	f002 f8ba 	bl	8004560 <HAL_DMA2D_Init>
